:100000000C94750F0C94940F0C94940F0C94940F03
:100010000C9446290C94940F0C94940F0C94A12AE0
:100020000C94940F0C94940F0C94940F0C94940FC4
:100030000C94940F0C94940F0C94940F0C94940FB4
:100040000C94940F0C94940F0C94940F0C94940FA4
:100050000C94940F0C94940F0C9483300C94940F84
:100060000C94940F0C94940F0C94940F0C94940F84
:100070000C94940F0C94940F0C94940F0C94AC214A
:100080000C94940F0C94940F0C94940F0C94940F64
:100090000C94940F0C94940F0C94940F0C94940F54
:1000A0000C94940F7F13471514152C1549127C15C9
:1000B000051506153511C211171E61150515051513
:1000C000201FAA134410471514152C1549127C152E
:1000D00099140615EC13C211171E61159711051519
:1000E000201FAA130515471514152C1549127C1548
:1000F000621206153812C211171E61159D110515E1
:10010000201FAA130515471514152C1549127C1527
:10011000C41206153B12C211171E6115F514051500
:10012000201FAA135711471514152C1549127C15B9
:10013000051506153F12C211171E6115A6130515E8
:10014000201FAA135711471514152C1549127C1599
:100150008B110615D813C211171E6115AF150515A1
:10016000201FAA135711471514152C1549127C1579
:10017000911106151B14C211171E611537110515B3
:10018000201FAA1357110515051505154912051548
:10019000941505154811C211171E051505150515ED
:1001A000201F05150515471514152C1549127C152A
:1001B000051506154E13C211171E611549130515B5
:1001C000201FAA130515471514152C1549127C1567
:1001D000F81106158013C211171E6115A31105151C
:1001E000201FAA130515471514152C1549127C1547
:1001F000001206158413C211171E61150515051589
:10020000201FAA130515471514152C1549127C1526
:1002100005120615A10FC211171E611569140515E7
:10022000201FAA130515471514152C1549127C1506
:1002300005150615960FC211171E611588130515B1
:10024000201FAA130515471514152C1549127C15E6
:10025000CD110615A415C211171E6115D11505156E
:10026000201FAA130515471514152C1549127C15C6
:10027000D91106155E14C211171E6115DA14051581
:10028000201FAA130515CA11BB14591349121E12B7
:10029000E4112A122E11C211171E0515B4110515ED
:1002A000201F05159CACCCB6F400C111214191A1D1
:1002B00031B171F19CACCCB6F4367491A1C111216D
:1002C0004131F17100030205000305010406020437
:1002D000C0C1C2FFC4C5C618808182C38485868719
:1002E0007071728374757677303132733435363786
:1002F00010111213141516170304050A08060BFF34
:100300000209070D010C00FF464B3A3A494A483AA8
:100310003A3A3A3A4C4F3A3A3A3A3A3A3A3A3A3A16
:100320003A3A3A3A3A4D3A3A66304E745A00000038
:1003300000000000000000000000000000000000BD
:1003400000000000000000000001540003FC000257
:10035000A80550000FF0000AA000000550000FF0A3
:10036000000AA00000000000000000000015470087
:100370003FFE002AA0005FFF07A0057807FEF03EC1
:1003800000F03FFFBD2AAA0AFFFFFFD400502B4018
:10039000BFC2F007C0BCFF007CABC0A0FF80006FF5
:1003A000FFF9F6AA8FFC000FFC000FFC000FF955B7
:1003B0004F9FFFF6BFFFE0CAAA00C00000C00000C8
:1003C000C00000C555007FFFD0400000F40000FFD2
:1003D000FFF4FEAAA7FC000FF9554F9FFFF600009F
:1003E0000400007C7FFFFC6AAAFCC000FCC555BC71
:1003F0007FFFD86FFFF8F6AA80FC0000FC0000FC2D
:100400000000FC0000E00000BFFFE40AAA7C00003E
:10041000FC0000FC0000FC0000FC00002C40000080
:10042000F40000FFFFF4FEAAA0FC0000F955409F75
:10043000FFF400000400007C7FFFFC2AAAFC0000FF
:10044000FC0555BC7FFFD86FFFF9F6AA8FFC000FA3
:10045000FC000FFC000FF8000F800002BFFFE4CA91
:10046000AA7CC000FCC000FCC000FCC000BC0000B6
:10047000086FFFF9F6AA8FFC000FFC000FFC000FBD
:10048000F8000F800002BFFFE0CAAA00C00000C051
:100490000000C00000C000000000006FFFF8F6AAD6
:1004A00080FC0000FC0007FC000FF8000F80000239
:1004B000BFFFE40AAA7C0000FC4000FCC000FCC5B1
:1004C00055BC7FFFD82FFFF902AA8F00000F000054
:1004D0000F00000F01554F1FFFF6BFFFE0CAAA0033
:1004E000C00000C00000C00000C555007FFFD04024
:1004F0000000F40000FD5550FFFFF8FC0000F8007C
:100500000080000000000400007C1555FCBFFFFCCB
:100510000000FC0000BC000008000000000000001B
:1005200000000000000000000155401FFFF4BFFF65
:10053000E40AAA7C0000FC0000FC0000FC0555BC9D
:100540007FFFD82FFFF902AA8F00000F000056018D
:100550005FE00AAA00000000BFFFE0CAAA00C000D6
:10056000005400002FD50000AA800000002FFFF8E3
:1005700002AA80000000000000000000000000004F
:100580000000BFFFE40AAA7C0000FC0000FC0000A1
:10059000FC0000BC0000082FFFF802AA8000BF503A
:1005A0000003FF007FA00155401FFFF4BFFFE00ADA
:1005B000AA000000000000000000000555007FFFB9
:1005C000D02FFFF802AA8002BF50000AA800000046
:1005D0000155401FFFF4BFFFE00AAA0000000055CC
:1005E00000000BF4000555007FFFD06FFFF8F6AA5E
:1005F00080FC0000FC0000FC0000F955409FFFF467
:10060000BFFFE40AAA7C0000FC0000FC0000FC051F
:1006100055BC7FFFD86FFFF9F6AA8FFC000FFC00D6
:100620000FFC000FF9554F9FFFF6BFFFE0CAAA006D
:10063000C00000C00000C00000C000000000006F4B
:10064000FFF8F40000FC0000FC0000FC0000F9557D
:10065000409FFFF4BFFFE400007C0000FC1540FC5D
:100660000BF4FC0555BC7FFFD86FFFF9F4AA8FFC93
:10067000000FFC0007FC000FF9554F9FFFF6BFFF6E
:10068000E0CAAA00C00000455000C2BF40C00280BE
:100690000000006FFFF9F6AA8FFC000FFC000FFCB2
:1006A000000FF8000F800002000004C0007CC000B2
:1006B000FCC000FCC000FCC555BC7FFFD84000005A
:1006C000F40000FD5550FFFFF8FC0000FC0000E0C6
:1006D0000000000000000000155500BFFF000000F2
:1006E000000000000000002FFFF802AA80000000B8
:1006F0000000000000000155401FFFF4BFFFE40AA6
:10070000AA7C0000FC0000FC0000FC0555BC7FFF3B
:10071000D82FFFF802AA80000000000000005FFA56
:1007200002AA00000000BFFFE00AAA0005FE00AA1E
:1007300080000000000000000000002FFFF802AA67
:10074000800000000000000000000155401FFFF481
:10075000BFFFE00AAA0005FE00FFC0000AFD000579
:1007600055007FFFD000000001550000AAF40000F2
:10077000540057E002AA00000000000000015500EC
:100780007EA8005400002F540002AA0000000000C0
:10079000000002FF400002FD0000550057E802AAD9
:1007A00000000000000000000000155500BFFF0021
:1007B000000000000000000000400000F40000FC09
:1007C0000000FC0015FC1FE8F8AA008000000000F3
:1007D0000400547C17E0FCA800FC0000FC0000BCF6
:1007E000000008FFFFFFFFFFFFFF0000FF0000FF0A
:1007F0000000FF0000FF0000FFFFFCFFFFFC000304
:10080000FC0003FC0003FC0003FC0003FC140000DC
:100810003FD4002BFFD4002BFF00002B0000000072
:100820000000000000000000000000D40000FFD421
:10083000002BFFC0002BC0FF0000FF0000FF0000E6
:10084000FF0000FF0000FFFFFFFFFFFF0003FC00B1
:1008500003FC0003FC0003FC0003FCFFFFFCFFFFA4
:10086000FC400000F40000FC0000FC07F8FC7E00E7
:10087000F955409FFFF400000005F8007E8000005D
:100880000000000000000000000000000000000068
:100890000000000000000000000000000000000058
:1008A00000000400007C0000FC0000FC0000FC00D4
:1008B00000BC000008000000000000000000000074
:1008C0000000000000000000000000000000000028
:1008D0000000000000000000000000000000000018
:1008E0000000000000555555FFFFFFAAAAAA00000E
:1008F00000000000000000000000554154FFC3FC50
:10090000AA82A8000000000000555500FFFF00AAC1
:10091000AA00000000000000FFFF00FFFF00000031
:1009200000000000000000000000000000000000C7
:1009300000000000000100000F00555B02FFF900FD
:10094000000F01554F1FFFF6000004C0007C9554B6
:10095000FCBFFEFCC000FCC555BC7FFFD81BFFFEE2
:100960003DAAA33F55563FFFFE3F00033E00032034
:100970000000400001F0001FE5557F6BFFFFF00015
:100980003FF1556F9FFFF60BFFFE00FEA3002F53B4
:10099000000151001F8302A803000000400000F086
:1009A0000550F1FE00D15000F0BD00F15FC09FFF87
:1009B000F400000101551F1FFFFF3E03FF3FDFE072
:1009C0000AFA00000003FFFD40EAAFF04002FCF528
:1009D00000FCBFF5F802FFD0FFFAB00000000000F5
:1009E0000420555022FFF800000000000000000025
:1009F00000000000000000000000000000000000F7
:100A000000000000000000000000000100000000E5
:100A100000000000000000000000000000F40000E2
:100A20002F400002F4000000000000000000000061
:100A3000000000BD00000BD00000BC000000000062
:100A40000000000000000001F8001F8000F8000016
:100A5000000000000000000000001501000BCF01A5
:100A6000555B03FFFB00014F001F8F00A8020054DD
:100A700000C7E000955500BFFF00C50000CBD000C7
:100A800000A80000000100000F01555F03FFFF00F8
:100A9000000F00000F000002000000C00000D5554C
:100AA00000FFFF00C00000C00000000000000001C7
:100AB00000000F00000F0001E7005F8F02A00F0091
:100AC0000002000000C00000C000006D0000CBD498
:100AD00000C02A0000000000000100000F00000F0D
:100AE00000000F00000F00000F000002000000C017
:100AF0000000C00000C00000C00000C000000000F6
:100B00000000000102F50F000BCF0000A700000F4E
:100B100000000F000002000000C17E00CF800068CE
:100B20000000C00000C00000000000000000000045
:100B3000000000000000150007F8007E0000000023
:100B400000000000540017E000AA000000000000B0
:100B500000000000006FFFF8F6AA80FC0000FC0017
:100B600054FC5FA0F955409FFFF4BFFFE40AAA7C44
:100B700017E8FCA800FC0000FC0555BC7FFFD8006E
:100B8000000000000000000000000000000001550F
:100B9000401FFFF400000000000000000000000003
:100BA0000000000555007FFFD0400001F4000FFC5D
:100BB000000FFC000FFC000FF9554F9FFFF6BFFF21
:100BC000E4CAAA7CC000FCC000FCC000FCC000BCA1
:100BD000000008400001F4000FFC000FFC000FFCB7
:100BE000000FF9554F9FFFF6000004C0007CC000C5
:100BF000FCC000FCC000FCC555BC7FFFD82FFFF92E
:100C000002AA8F00000F00000F00000F01554F1FB8
:100C1000FFF6000000C00000C00000C00000C000DF
:100C200000C555007FFFD0400000F45500FCAFF434
:100C3000FC00A7FC000FF8000F8000020000040079
:100C4000007C0000FC4000FCC000FCC555BC7FFFE0
:100C5000D86FFFF9F6AA8FFC000FFC000FFC000F05
:100C6000F8000F800002BFFFE4CAAA7CC000FCC0ED
:100C700000FCC000FCC555BC7FFFD8400000F4005C
:100C800000FC0000FC0000FC0000F955509FFFFC38
:100C9000000000000000000000000000000000054F
:100CA00055007FFFD06FFFF9F6AA8FFC000FFC0004
:100CB0000FFC000FF9554F9FFFF6BFFFE4CAAA7C57
:100CC000C000FCC000FCC000FCC555BC7FFFD86F55
:100CD000FFF9F6AA8FFC000FFC000FFC000FF9557E
:100CE0004F9FFFF6000004C0007CC000FCC000FC69
:100CF000C000FCC555BC7FFFD86FFFF9F6FE8FFC26
:100D00007F5BFEFFF9FC1F8FF9FD4F9FFFF6BFFFD2
:100D1000E4CBFA7C9FD4FCBFFEFCCBD0FCC5FDBC71
:100D20007FFFD800000100000F00000F00000B0043
:100D30000000000000000000000000C01500C7E82F
:100D4000009E000000000000000000000000000005
:100D50000000000000000000000007F8007E000016
:100D6000000000000400547C17E0FCAA00FC000016
:100D7000FC0000BC00000800000100000F00000F94
:100D800000000F00000F00000F000002000004C070
:100D9000007CC000FCC000FCC000FCC000BC000027
:100DA0000800000000BD00000BF40000000000007F
:100DB00000000000000000000400007C0000FC5562
:100DC00000FC2BD0FC00A8BC0000086FFFF8F6AABE
:100DD00080FC0000FC0001FC000FF9554F9FFFF65E
:100DE000000000000000155400BFFE00C00000C05D
:100DF00000000000002FFFF902AA8F00000F000082
:100E00000B000000000000000000BFFFE0CAAA00C5
:100E1000C000008000000000000000000000000092
:100E2000000100000F00000B0000000000000000A7
:100E300000000000BFFF90CAA9F08003F0BD03F0DE
:100E40000BD3F00556F07FFF602FFFF902AA8F0049
:100E5000000F00000F00000F00000F000002BFFF96
:100E6000E4CAAA7CC000FCC000FCC000FCC555BCA4
:100E70007FFFD800000100000F00000F00000F00EE
:100E8000000F00000F000002BFFFE4CAAA7CC000F0
:100E9000FCC000FCC000FCC000BC00000800000159
:100EA00000000F00000F00000F00000F01554F1F42
:100EB000FFF6BFFFE4CAAA7CC000FCC000FCC00073
:100EC000FCC555BC7FFFD800000100000F00000FDB
:100ED000000002000000000000000000BFFFE4CAA4
:100EE000AA7CC1F8FC7E80FC0000FC0000BC000075
:100EF00008400000F40000FC0000FC0000FC0000C2
:100F0000FC0000E000000000000000000000000005
:100F10000000000000000000000000400000F4009D
:100F200000FC0000FDFFF4FCAAA0FC0000E00000B3
:100F300000000000000000000000000000000000B1
:100F40000000000000400000F40000FC0000FDFF75
:100F5000FDFCAAA8FC0000E0000000000000150055
:100F600007E800AA000000000000000000000040A8
:100F70000000F40000FC0000FDFFFDFCAAA8FC003E
:100F800000E0000000000000150007E800AA0000D3
:100F9000AF400002BD00000000400001F4000FFC63
:100FA000000FFDFFF7FCAAA0FC0000E0000000001D
:100FB00000C01500C7E8002A0000AF400002BD00D5
:100FC000000000400001F4000FFC000FFDFFF7FCE3
:100FD000AAA7FC000FE0000B000000C01500C7E846
:100FE000002A00006F4000C2BD0080000000000029
:100FF00000000000555002FFF900000F01554F1F7F
:10100000FFF60000000150001F8000A80000C00093
:1010100000C0000000000000000100000F00000FF1
:1010200000054F007E0F00000F000002000004C00A
:10103000547CC7E0FCC000FCC000FCC000BC000049
:1010400008400000F44000FCFD40FC2BF4FC002CA8
:10105000F8000080000000000400047C05FCFC7F18
:10106000A0FCE000FC0000BC000008000000000044
:10107000000000000000070001FE007F800FE0007C
:1010800000001C0057FC1FE8FC9500FC0BD0FC0086
:10109000BFFC00002C00000100000F00003F00001A
:1010A0003F00003F00003F00003EF001F0C17FF034
:1010B000DFFA00E00550DFFFF0EA03F0000A00006D
:1010C000000500007F0003FF0003F80003FD00019E
:1010D000FF0003FAFFFF40FFFFF0A00FF0001FE04A
:1010E00057FF50FFFFF0AA03F017FFFF3FEAAAFEE9
:1010F0000054FC00FCFF01FD3FFFFF0BFE8FFFFFD4
:10110000FFABFEAA00FF0000FF0001FF00FFFE0092
:10111000FFF80000000114001FFC007FFC00FCFD34
:10112000403F3FFFFF0ABFFF5FF500FFFFF0800277
:10113000FC0003F8517FE0FFFE00EA8000001FD4AE
:1011400001FFFD07F82F0FF00F0FF00F0FF00A024D
:10115000FC001FFD00FFFFD0F00BF4E003FCC00318
:10116000FC8003FC000FF000001500003F07FFFFAC
:101170003FFFFFFE003FFC002ABF00000003FC0110
:101180005FFCFFFFFCFEA3FC0003FC0003FC00036C
:10119000FC0000FC005FFF0FFEFE3F80FCFE00FC39
:1011A000FD00FC3F4000FC0000FFD400FEFFC0FC3F
:1011B0000BF0FC02FCFC01FC0007E0000014000145
:1011C000F80013F007F3C0FE83F0A002FF00000A4E
:1011D0000155001FFFD07E02FCFC00FCFC07E0FF75
:1011E000FFFCAAAAA800001F0001FE0173F05FE344
:1011F000F0F803F50000BF00000AFFFF40FEAFF467
:10120000FC02FCFC00FCFC01FCFC03F0A80000005C
:1012100000500000F0007CF51FE0FF3E00000000E1
:10122000000000000000FC0000FC5555FCFFFFFC26
:101230000000FC0000FC00000000005F0001FE0157
:10124000F3F05FA3F0F802FF00002B000000FFFDA9
:1012500040AAAFF40002FC0001FC555FF8FFFE80DD
:101260000000000003FF0010AA05F0003F800028E6
:1012700001FF0002AA000000FFFFD0AAABFC0000A3
:10128000FC0005F8FFFFFCAAAAA80000000000006F
:1012900000000005FFFF3FFFFFFE00003C000000D4
:1012A000000000001F00003FFFFFFFFFFFE80000FD
:1012B00000000000000000001FE0003FC0003FD021
:1012C000000FF00003FC0003FC001FF07F8000FF14
:1012D0000000FF00003FC0000FF0000FF0007F8013
:1012E000000000FF07F0FF0F007E0BD3F007F3FDB7
:1012F0000F80FF00002FFFFFFCFFFFFC000000003D
:101300000000000000FFFFFCFFFFFC0017FF01FFD3
:10131000EA0FE8000FC0000FD40002FFD5002BFF3A
:10132000FF50FCAFFDFC000BFC0000000007FC5F61
:10133000FEFCFA80FC400000F40000FC0000FDFF11
:10134000F4FCAAA0FC0000E0000000000000000087
:10135000000000000000000000000000000000008D
:10136000000100000F00000B000000000000000062
:1013700000000000BFFF90CAA9F08003F0BD03F099
:101380000BD3F00556F07FFF602FFFF902AA8F0004
:10139000000F00000F00000F00000F000002BFFF51
:1013A000E4CAAA7CC000FCC000FCC000FCC555BC5F
:1013B0007FFFD800000100000F00000F00000F00A9
:1013C000000F00000F000002BFFFE4CAAA7CC000AB
:1013D000FCC000FCC000FCC000BC00000800000114
:1013E00000000F00000F00000F00000F01554F1FFD
:1013F000FFF6BFFFE4CAAA7CC000FCC000FCC0002E
:10140000FCC555BC7FFFD800000100000F00000F95
:10141000000002000000000000000000BFFFE4CA5E
:10142000AA7CC1F8FC7E80FC0000FC0000BC00002F
:10143000080000000000000000000001F9001F8FFC
:1014400001F80F000002000000000000155500BF69
:10145000FF80C00000C0000000000000000000018C
:101460000000000000000700000F00000B0000005B
:1014700000001C0000FC5400FC6F40FCC2F4FC9F08
:10148000FF6CAAAAA003FFFF03FFFF0000070000F4
:101490000F00000F00000F000002FFFFFCFFFFFC29
:1014A000F80000F00000F40000FFFFFCFFFFFC006C
:1014B000000000000000001500FF3F00FF3F00009B
:1014C00000000000000000000000400000FFFFFCE2
:1014D000FFFFFC0000000000000000000000000012
:1014E000000000000000001500FF3F00FF3F000368
:1014F000F40003FF0000BF00003F40007FFFFFFF3C
:10150000FFFFF800FFFF00FFFF00000000000100E8
:10151000003F00003E000000FFFFFCFFFFFC1FF447
:1015200000FEBF40E00BFC0000BC0000000000001B
:10153000000000000000003FFF003FFF000000002F
:101540000000000000000000000000FFFFFCFFFFA3
:10155000FC00000000000000000700003F00003F0A
:1015600000000F00003F00003F00000BFFFFFCFAEF
:10157000AAA8D40000FFC000E80000F55554FFFF02
:10158000FC00003F00003F00001F00003F00003F44
:1015900000003F00000BFFFFFCFFFFFCE00000C06D
:1015A0000000C00000FFFFFCFFFFFC000007000080
:1015B0003F00003F00003F00003F00003F00000BE5
:1015C000FFFFD0FFFFFCE00BFCC003FCD007FCFFDB
:1015D000FFFCFFFFE0003FFF003FFF0007FE000FA2
:1015E000F0000FF4000FFF0002FFFFFFFCFFFFFC05
:1015F00002FD0000FF0001FF00FFFF00FFF80000F8
:10160000007F0007FF000FF8000FF0000BF4003F11
:10161000FF003FFFFFF400FFFF0002FF0000FF009C
:1016200001FE00FFFFFCFFFFFC00003F00003F0049
:10163000000700003F00003F00003F00000BFFFFDD
:10164000FCFFFFFCFE0000E00000D00000FC0000FA
:10165000FC000000001F0000FF0000FE0000FC0076
:1016600000FC0000FF0000BFFD0FD0FFCFFC2FC229
:10167000FC0FC0FC0FD1FC0FFFFC02FFE0000003D9
:1016800001555703FFFF02AAAB0000030000000052
:101690000000FC0000FD5540FFFFF4FEABFCFC0128
:1016A000FC003FFC003FE000003F00003F00000066
:1016B00000000000000000003F00003FFFFFD0FFDF
:1016C000FFFC000BFC0003FC0007FCFFFFFCFFFF1E
:1016D000E000003F00003F000000000000000000AC
:1016E00000003F00003FFFD000FFFD0002FFD000E0
:1016F0003FFC01FFE0FFFE00FFE00000003F0000B4
:101700002A00000000000000000000001500003F5B
:10171000FFFFD0AAAFFC0007FC03FFF0000BFC5555
:101720005FFCFFFFE000003F00002B000000000016
:101730000000000000001700003F4001FCF41FE81B
:10174000BFFE000FF0007FFD00F82FD48002FC00E8
:10175000003F00003F0000000000000000150000F6
:101760003F00003FFD03F4FFC3FC2FC0BC1FC03C83
:10177000FF807CFFFFFCFFFFF800003F00003F0000
:10178000003F00003F00003F00003F00003FC0015D
:10179000FCC01FFCC1FFFCDFFFFCFFE3FCFE03FC01
:1017A000E003FC00000000000301400F7FFFFFFE8C
:1017B000AAA8F00000A00000000000C00000F00196
:1017C00040FFFFFD2AAABF00000F00000A00000032
:1017D000000000555555FFFFFFAAAAAA000000000F
:1017E0000000000000000000555554FFFFFCAAAAAD
:1017F000A8000000000000000000F00000FC000055
:10180000FFFFFD2BEAAF0000030000020000000014
:10181000000F00001F1FFFFFFAABE8E00000800090
:1018200000400000F44000FCFD40FC2BF4FC002CC8
:10183000F8000080000000000400047C05FCFC7F30
:10184000A0FCE000FC0000BC0000081FFFFFFFFF41
:10185000FFFF800FFF000FFF400FFFFFFF2FFFFF75
:10186000FFFFD0FFFFFCC00BFCC003FCC007FCFF68
:10187000FFFCFFFFE03000003000003000002000DF
:1018800000300418355D80300C902000083BAEBC61
:10189000359D9C318C9C2AAAA83BAEBC359D9C31C1
:1018A0008C9C2AAAA8300018355580300090200062
:1018B00008300418355D8030009020000830001892
:1018C0003555803000002000000057C007FFC402DB
:1018D000FFC000028000FFC005FFD402FFE0002E21
:1018E000000001F41557F82D1000028000300000B0
:1018F00030000030000020000007FFF40B503C05D2
:101900007FF40A00283FFFFC000F00157D402AAA43
:10191000800007FC00783C07897C280028003C00F8
:10192000557D55AABEAA003C00000000555555AA99
:10193000BEAA003C003FFFFC30000C30000C300021
:101940000C3FFFFC31554C32AA8C30000C3FFFFCA1
:1019500031554C32AA8C33FFCC30000C30000C30A7
:10196000000C35555C31554C32AA8C30000C355585
:101970005C31554C32AA8C33FFCC35555C2AFFA81C
:10198000000000000000000000000000555400AA04
:10199000BC00003C00003C00557C00AAA8000000F0
:1019A00000003C00003D55002AAA00000000000095
:1019B000001555003EAA003C00003C00003C000021
:1019C0003C00003C00003C00557C00AABC00003CF0
:1019D0000001414403C7E007E3C0228280003C00CD
:1019E000003D55003EAA003C00003C00557D55AA34
:1019F000AAAA000000000000000000000000000093
:101A0000000000003FFF3C0000000000003FC0005D
:101A10000000001540002A800017D7D42BEBE83FC8
:101A2000FFFC02828007F4D01F7DF40F3DF0020A14
:101A3000803C0078001E8007A0142800281F47F46F
:101A40003C343C2F8AF80002080000001440002AB1
:101A5000000000000007FFD03E00BC20000800008E
:101A60000034001C2F55F802AA80000000024C60D0
:101A7000017F50006E40020820003C0003FFC000C0
:101A80003C000000000000000003D800000000003F
:101A900000003C00003C00003C000028000000006A
:101AA0000000F0000000000000000078001E800729
:101AB000A0002800001FFFF43C1E3C3DF57C0AAA54
:101AC000A005003C3FFFFC00003C0000001F01FCA3
:101AD0003C1FBC3DF83C0A80281F00F43C143C3DF0
:101AE0007D7C0A82A0007F00078F003FFFFC000A78
:101AF000003FF0F43CF03C3CF57C282AA01FFFF4AA
:101B00003C3C3C3C3D7C280AA03C00003C1FFC3D8A
:101B1000F8002A80001FD7F43C3C3C3D7D7C0A82C3
:101B2000A01FF4F43C3C3C3D7D7C0AAAA0000000D0
:101B30000141400282800000000000000141440297
:101B400082A0000000001D0001E2D00E002C000069
:101B50000001414003C3C003C3C0000000040004EF
:101B60000B407800B7800008001F00003C1F3C3D80
:101B700078000A800006AAA431AA4C24AA4C02AA22
:101B80000007FFFC3E0F002F5F5402AAA83FFFFC96
:101B90003C3C3C3D7D7C0A82A01FFFF43E00BC3DE6
:101BA000007C0A00A03FFFFC3C003C2F55F802AA35
:101BB000803FFFFC3C3C3C3C283C2800283FFFFC8D
:101BC0003C3C003C28002800001FFFF43C003C3C4B
:101BD0000F7C080AA03FFFFC003C00157D542AAA98
:101BE000A83C003C3FFFFC3C003C0000001400F41B
:101BF0003C003C3FFFF82800003FFFFC003C001782
:101C0000C3D42800283FFFFC00003C00003C00003B
:101C1000283FFFFC0B40001F55542AAAA82FFFFCA9
:101C200002D000157D542AAAA81FFFF43C003C3DB9
:101C3000557C0AAAA03FFFFC3C3C003D7C000AA06A
:101C4000001FFFF43C053C3D57FC0AAAA03FFFFCE7
:101C50003C3D003D7EF40AA0281FF4343C3C3C3C53
:101C60003D7C080AA03C00003FFFFC3C0000000057
:101C7000003FFFF400003C15557C2AAAA03FFF401E
:101C80000000B41555E02AAA003FFFF800078015B0
:101C900057D02AAAA83D417C02BE8017EBD4280069
:101CA000283FD400003FFC3FE8000000003C01FC5E
:101CB0003C1E3C3DE03C2A00281555543EAABC3C45
:101CC000003C0000002D000002B400000AD000001B
:101CD000281400143C003C3FFFFC00000001E00021
:101CE0001E00000B400000A00000003C00003C0073
:101CF000003C0000282D000002D000000000000081
:101D0000000051F400F33C00F774002AA83FFFFCE8
:101D100000F03C00F57C002AA0007FF400F03C00BD
:101D2000F03C002020007FF400FC3C157D7C2AAABA
:101D3000A8007FF400F33C00F73C002A20057D5406
:101D40003EBEA83D28000A0000007D1400F33C00C0
:101D5000F77C002AA03FFFFC00780000F554002A21
:101D6000A80050003CFFFC0000000000000000F450
:101D700000503C3CFFF80000000FFFFC0007D000C3
:101D8000382C0000081400003FFFFC000000000099
:101D90000000FFFC002D00007D5400AAA800BFFC3D
:101DA00000F80000BD54002AA8007FF400F03C00B9
:101DB000F57C002AA000FFFC007AD000F5F0002A94
:101DC00080007FD000F0F0007FD400AAA800FFFCC4
:101DD00000780000F400002800007D3C00F33C0087
:101DE000F37C00A0A015F5502AFABC00007C00008E
:101DF000A000FFF400003C00557C00AAA000FF40BA
:101E00000000B40055E000AA0000FFFC0001E00063
:101E100055F400AAA800F47C002BA0007EF400A0DA
:101E20002800FD14000F3C005F7C00AAA000F07C9D
:101E300000F3BC00FE3C00A028000000057D503AE5
:101E400082AC000000000000555555AAAAAA000067
:101E50000000000035415C0ABEA00000003F41FCCC
:101E60003CBE3C3D007C2A00A83FFFFC003C00003B
:101E70003C0000280003D6170202D10103C0080A63
:101E800005C11919191905C23131313105C41919A2
:101E9000191905C52727272702B20209B405467775
:101EA000777777764502B71302B03F02C900011178
:101EB000FF023620023A1102B92002B82902D0FFEF
:101EC00001390129FF0000000000010101020203A5
:101ED000030405060708090A0B0C0E0F101214154F
:101EE00017191B1D1F212325272A11241FBECFEFE1
:101EF000CDBFDFE7DEBF10E4A0E0B0E4E0E8FFE73D
:101F000000E00BBF02C007900D92AE30B107D9F7C9
:101F10002DE7AEE0B0E401C01D92AA3EB207E1F7A2
:101F20000E94833C0C94BE3F0C9400009091347D41
:101F300081E098279093347D8093074080930640FA
:101F400008951092347D81E080930740809305408E
:101F500080930640089581E08093E97D10927B4252
:101F600010927C428093D169E2E3F2E411921586EB
:101F7000138E11A617AA82E4E034F807B9F710927D
:101F80008742109288421092894210928B4210929E
:101F90008C421092CA691092CB69109278421092CA
:101FA000794210927A4280E180938A421092F769D6
:101FB0001092CF69089580917A42813019F088E7B4
:101FC00092E4089589E792E408958031910508F03C
:101FD000C09747E0489F9001499F300D1124C901E7
:101FE0008E5C9D4BFC01E55AFF4F20914F4230E142
:101FF000239FA001112420914E42242B208331964F
:102000002091514230E1239FA001112420915042A0
:10201000242B208331962091534230E1239FA0014D
:10202000112420915242242B208331962091554235
:1020300030E1239FA001112420915442242B2083BE
:1020400031962091574230E1239FA0011124209125
:102050005642242B208331962091594230E1239F10
:10206000A001112420915842242B20838F599F4F87
:1020700020915B42E0E12E9FA001112420915A4261
:10208000242BFC01208308950895CF93DF93DC0176
:10209000EB012EE049914D932A95E1F7DF91CF9125
:1020A0000895CF93DF93342F522FDC01EB01252FBE
:1020B000231B2395A30FB11DC30FD11D49914D9330
:1020C0002A95E1F7DF91CF910895DC01242F261B9B
:1020D0002395A60FB11D1D922A95E9F70895CF9378
:1020E000DF93EB01342F722FDC01272F231B239565
:1020F000A30FB11DC30FD11D4C9158815D9349931E
:102100002A95D1F7DF91CF910895CF93DF93DC012A
:10211000022E000C330B51E0E42FF0E02E173F07A6
:102120001CF4DF91CF91089580E06115710521F0D5
:10213000EB01CE0FDF1F8881EA0FFB1F9081C0915A
:10214000D1699C0F980F908380918A42981730F044
:10215000981B90835093D1694F5FDECF1092D16965
:10216000FBCF0F93FC0131E0021714F40F91089597
:1021700090E06115710531F0DB01A20FB11D27FD63
:10218000BA959C9180E04115510531F0DA01A20F1A
:10219000B11D27FDBA958C91981B8091D169981B30
:1021A00097FF0FC080918A42980F3093D169309782
:1021B00031F0DF01A20FB11D27FDBA959C932F5F6F
:1021C000D3CF1092D169F3CFCF93DF93242FEC01BB
:1021D000C60FD11D261B498149932A95E2F71A9211
:1021E000DF91CF910895CF93DF93DC011092D169F5
:1021F0002417A4F0E42F042E000CFF0B90E06115CF
:10220000710521F0EB01CE0FDF1F9881EA0FFB1F54
:102210008081891731F081E08093D169DF91CF917E
:1022200008954F5FE5CFAFE7B2E48D919C91119790
:10223000E1E8F2E4208131812D933C93A3E8B2E4FC
:102240002D913C91119720833183E5E8F2E42081C0
:1022500031812D933C931082118208950E941311B5
:1022600080937B4290937C4208950C9413110E94BA
:102270001311E2E3F2E4292F22952F7022A39F701D
:1022800091A3982F92959F7090A38F70878F089538
:10229000E2E3F2E482A1829591A1892B90A192952B
:1022A000278D922BEBE7F2E490838183089582954A
:1022B000837090E09C01220F331F227095958795C3
:1022C000822B90917E42292F22952F7030E096E14B
:1022D000929FF001939FF00D1124E55DFF4B9589CE
:1022E000EBE2F0E444E084029001112445894913B3
:1022F0000CC0DF01A20FB31F4D915D916D917C91D8
:10230000452B462B472B09F0848B769641E4EB381E
:10231000F40761F708956EE472E48CE592E40C949E
:1023200045106CE572E48EE492E40C9445106EE482
:1023300072E48AE692E40C9445106AE672E48EE454
:1023400092E40C944510E2E3F2E4968D858D82953B
:10235000807F248D822B8093F5699093F66910928B
:10236000A4411092A5410895E2E3F2E4858D20E1B5
:10237000829FC0011124248D822B8093A4419093CD
:10238000A541089582958F708093CC6985E08093F4
:10239000F769089510928B420895E2E3F2E4858D87
:1023A00090E1899F90011124848D822B80938B4230
:1023B0000895E2E3F2E480918B42982F9F70948F0E
:1023C00082958F70858F0895E2E3F2E4ABE8B2E482
:1023D0008C91958D40E1949F90011124948D922BC6
:1023E0009C93982F9F70948F82958F70858F0895FE
:1023F00080918B428093894280EA809307040895FC
:102400008091894280938B42089580918B42909174
:10241000894290938B428093894280EA809307049B
:1024200080910240811109C088ED9DE180930340B5
:102430009093044081E08093024008950E94DB0F56
:10244000FC019081911103C08DE08083089591502B
:10245000908308950E94DB0FFC0190819F5F908321
:102460000E94DB0FFC0120812E3008F010820895BD
:1024700010927A42089581E080937A420895909173
:10248000784280917942981303C081E08093D169AA
:102490000895CF93C82F0E94DB0FDC01EC91F0E090
:1024A000EE5CFD4BC295CF70C48F0E94DB0FFC0128
:1024B0009081911104C08DE08083CF910895915057
:1024C0009083FBCFCF93DF930E94DB0FDC01EC9175
:1024D000D0918842C0918742ED30B1F48091104094
:1024E000982F9F7B953B11F0873F49F4C0935B4247
:1024F000D0938742C0938842DF91CF910895D093C3
:102500005B42C0934E42F8CF80910F408D3079F5F9
:1025100080911040853F61F0982F9F70973039F57A
:1025200082958F70982F977F973009F18B30F9F053
:10253000D0938742C09388420E94DB0FDC01EC916C
:10254000F0E0EE5CFD4BC58F0E94DB0FDC01EC91EF
:10255000F0E0EE5CFD4BD48F0E94DB0FDC01EC91D0
:10256000F0E0EE5CFD4B858D80934E42C5CFF0E0F0
:10257000EE5CFD4BD58F0E94DB0FDC01EC91F0E0AF
:10258000EE5CFD4BC48FB8CFCF93DF930E94DB0F7F
:10259000DC018C91C09187428D3001F59091104003
:1025A00080915B42292F2F7B253B11F0973F49F407
:1025B0008093884280938742C0935B42DF91CF91A2
:1025C00008959091884220914E42209387428093B3
:1025D000884290935B42C0934E42F0CF20910F40CF
:1025E000D091884290E02D3099F520911040253F00
:1025F00061F0322F3F70373059F522952F70322F0E
:10260000377F373029F12B3019F18E5C9D4BFC015F
:10261000858D809388420E94DB0FDC01EC91F0E015
:10262000EE5CFD4B848D809387420E94DB0FFC01A2
:1026300090914E42E081F0E0EE5CFD4B958F0E9460
:10264000DB0FDC01EC91F0E0EE5CFD4BD48FC3CFEF
:102650008E5C9D4BFC01858D809388420E94DB0F30
:10266000DC01EC91F0E0EE5CFD4B848D80938742C1
:102670000E94DB0FDC01EC91F0E0EE5CFD4BD58FAE
:102680000E94DB0FDC01EC91F0E0EE5CFD4BC48FAF
:1026900095CF8091314280937B4208958091314261
:1026A000E2E3F2E4982F92959F7090A38F70878F4A
:1026B00008958091367D9091377D892B91F080919E
:1026C000367D9091377D01978093367D9093377D4D
:1026D00081E09091A341911101C080E08093D16984
:1026E00008958091CF69823099F71092CF69109246
:1026F000A341109231428091264290E0E5CF0895A7
:1027000080E180938A4208958AE080938A42089506
:10271000E2E3F2E482A1829591A1892B90A19295A6
:10272000278D922B9093294080932A4082E08093BA
:10273000F7690895E2E3F2E4968F982F92959F70DF
:10274000958F8F70848F1092F769089583E080933E
:10275000F7690895CF93DF93CDB7DEB72E97CDBF3E
:10276000DEBF82958F70E82FF0E0E850FD4FE491D6
:10277000DE0111969E01215F3F4FBD0181E08E0F6A
:102780000E2E000CFF0BEE5CFD4B948D9D93E0E054
:102790008E300CF4E82FA217B30781F78EE492E491
:1027A0000E9445102E96CDBFDEBFDF91CF910895D8
:1027B000809128422AE0829FC00111242091457D0A
:1027C0003091467D8217930720F081E08093D16994
:1027D00008951092D169089584E08093F76908956F
:1027E000F89480910A6A8823B9F0E091086AF0E0D1
:1027F000E850F64980819091086A9F5F9093086A3B
:102800009091086A9F709093086A90910A6A91501B
:1028100090930A6A7894089580E0FCCF9091240800
:1028200095FFFCCF8093220808952EE0FC011192C1
:102830002A95E9F7089582E392E40E94151480E452
:1028400092E40E9415148EE492E40C941514EDE8C1
:10285000F2E48DE397E2DF019C011D9221503040AC
:10286000E1F70895FC01DC011B966B3051F4838580
:102870009E9111969C931197AE17BF07C9F78C9341
:102880000895808191819193EA17FB07D9F780839E
:1028900008958031910580F09C0120543109203C3D
:1028A000314050F09E7F9C012150324081E02F3E0C
:1028B000310518F080E0089581E00895809130425C
:1028C000811106C00E94131180937B4290937C4239
:1028D0000895CF93DF938091A4419091A5410097F3
:1028E00031F08D3F910589F0DF91CF910895C0912E
:1028F000F569D091F669CE010E9449148823A1F3AD
:10290000CE01DF91CF910C94E50F20915042809140
:102910004F4230E1839FC0011124922B20914E42FF
:10292000822B80932F7D9093307D81E080930640B1
:10293000DBCF0E94DB0FDC01EC91ED30A1F4909134
:10294000104080915B42292F2F7B253B11F0973F50
:1029500039F49091884290938742809388420895F9
:1029600090914E42F8CFF0E0EE5CFD4B848D809369
:102970008742858DF2CF8091367D9091377D892B6E
:1029800051F08091367D9091377D01978093367D0F
:102990009093377D08958091CF698130D9F78091E8
:1029A000B3418111F7CF82E08093CF6980912642B5
:1029B00090E0ECCF8EE0815078F480913042882313
:1029C00051F08091CD698D3031F480914E428093E9
:1029D0005B4280933F420895E82FF0E0EE5CFD4BB0
:1029E000948D20819223948FE6CFCF93DF93AEE432
:1029F000B2E4CAE6D2E43EE04C9158815D9349933B
:102A00003A95D1F7DF91CF9108950895CF938295AC
:102A10008F70E82FF0E0E850FD4FC4910E94DB0F6B
:102A2000FC01C083CF91089582958F70E82FF0E06C
:102A3000E850FD4FE491ABE8B2E421E030E002C0A1
:102A4000220F331FEA95E2F78D919C911197822B0B
:102A5000932B8D939C93089582958F70E82FF0E0CF
:102A6000E850FD4FE49181E090E002C0880F991F8B
:102A7000EA95E2F720918B4230918C428223932396
:102A800021E0892B09F420E02093D16908958295F3
:102A90008F70E82FF0E0E850FD4FE491ABE8B2E42E
:102AA00081E090E002C0880F991FEA95E2F78095D7
:102AB00090952D913C911197822393238D939C9314
:102AC00008952091CA693091CB6982958F70E82F63
:102AD000F0E0E850FD4FE49181E090E002C0880F03
:102AE000991FEA95E2F78223932321E0892B09F4C9
:102AF00020E02093D1690895CF93C82F0E94DB0F67
:102B0000C295CF70EC2FF0E0E850FD4FE491DC016E
:102B10008C910E2E000CFF0B8E171F0619F481E00E
:102B20008093D169CF910895CF93DF93AEE4B2E45F
:102B3000CCE5D2E43EE04C9158815D9349933A95BF
:102B4000D1F7DF91CF91089580913042882331F001
:102B50000E94131180937B4290937C420895E2E39C
:102B6000F2E482A1829591A1892B90A19295278D63
:102B7000922BE3E8F2E42081318120938542309367
:102B80008642A1E8B2E42D913C91119720833183D4
:102B9000EFE7F2E4208131812D933C939083818390
:102BA00008958EE0815078F480913042882351F06E
:102BB0008091CD698D3031F480914E4280935B429B
:102BC00080933F420895E82FF0E0EE5CFD4B948D3A
:102BD0002081922B948FE6CFE0E4F4E081818D6038
:102BE0008183A0E0B4E011968C91119780641196D6
:102BF0008C93A0E6B9E084E811968C93119781E359
:102C00008C9388E0858308959091630995FFFCCFAC
:102C100090E490936309809364090895680F791F85
:102C20008617970709F408952091630925FFFCCFC3
:102C3000FC012191CF0120936409F2CF27E731E015
:102C4000829FF001839FF00D1124E55FF54920E09C
:102C5000818192819695969530E4839FA0011124FD
:102C6000942B928390818695869530E4939FA00162
:102C70001124842B81839695969590832F5F3396AC
:102C80002D3731F7089527E731E0829FF001839FC8
:102C9000F00D1124E55FF5492DE781819081990FB1
:102CA000990F382F3295369536953370932B908344
:102CB0009281880F880F392F32953695369533706B
:102CC000832B8183990F990F928321503396211181
:102CD000E4CF0895EBE0FAE68DE190E1DF019C019D
:102CE0001D9221503040E1F70895EBE0FAE6919112
:102CF000DF01119798279C939AE7E832F907B9F713
:102D0000089527E731E0829FF001839FF00D1124A1
:102D1000E55FF5499F0122513D4F8191DF011197F8
:102D200086768C93E217F307C1F7089527E731E021
:102D3000829FF001839FF00D1124E55FF549629FAA
:102D4000D001639FB00D1124A55FB549CF0189580B
:102D50009E4F21912D93E817F907D9F7089570E058
:102D600027E731E0482F429FC001439F900D112477
:102D700047E751E0855F95490C94B73FCF93DF93C8
:102D80008F773CE0839FC00111248B58974E362FDC
:102D90003695E7E7F1E04E9FD0014F9FB00D11242B
:102DA00043E0349FA00DB11D1124A55FB549AD01CD
:102DB000445F5F4F8A1B9B0B60FF26C0FC01EA0F3C
:102DC000FB1FE4912636F1F0E22713967C911397CE
:102DD0007575F0E03C913A7AEF01D595C795C575C8
:102DE0003C2B3C93EE0FFF1FEA7AE72B1396EC93F4
:102DF000139711964A175B0709F788E0860FDF9152
:102E0000CF910895E676E1CFFC01EA0FFB1FE49134
:102E1000263639F0E227EC931196A417B507A1F7EF
:102E2000ECCFE676F8CFFF920F931F93CF93DF930B
:102E30008C01D42FF22EC0E0F801EC0FF11D80813F
:102E4000811107C0862FDF91CF911F910F91FF90C5
:102E500008952F2D4D2F0E94BE16682FCF5FECCF07
:102E6000FF920F931F93CF93DF938C01D42FF22EF9
:102E7000C0E0F801EC0FF11D8491811107C0862F8D
:102E8000DF91CF911F910F91FF9008952F2D4D2F1E
:102E90000E94BE16682FCF5FECCF9C0180E0F90145
:102EA000E80FF11D9081992311F08F3F09F40895E7
:102EB0008F5FF5CFEF92FF920F931F93CF93DF9326
:102EC000CDB7DEB76097CDBFDEBF89839A836B83B2
:102ED0007C834D835E832F83388709871A87EAE3D3
:102EE000F7E7A2E8B7E781EB98E710821182128238
:102EF0001C9211961C92119712961C921297E55BE8
:102F0000FF4FA55BBF4F8E179F0779F76AE089E0F7
:102F10000E949616CE0101967C0110E000E0F701B8
:102F2000419151917F012FEF2F5F822F022E000CD4
:102F3000990BFC01E40FF51FE491ABE0B0E0AC0F9E
:102F4000BD1FA80FB91FEC93E111EECFB801675E6A
:102F50007F4F880F991F880F991F681B790B2FEFE0
:102F600049E0CE010B960E9413170E5C1F4F0A3FDB
:102F70001105A9F689E00E941E166096CDBFDEBF3E
:102F8000DF91CF911F910F91FF90EF90089599E1FC
:102F9000899F802D112461E0282F260F30E0A901A0
:102FA000440F551F240F351F255F3549F901E15D99
:102FB000F24F9081492F440F440FD901A05DB24FC9
:102FC0009C919295969596959370942B90839C9155
:102FD000492F440F440F329690819295969596957D
:102FE0009370942B9C93408194E0499FA0011124FD
:102FF000436040832A55314FF90110826F5F683179
:1030000059F60895CF93DF930E946A1680E090E806
:10301000A1E0BB279858AF4FBF4FCBE0DAE6ABBF7C
:10302000FC01279129930196A11DB11D22E7C9300A
:10303000D207A9F780E090E0A1E0BB27AC01BD0179
:1030400058586F4F7F4FC9E0D2E76BBFFA01279105
:1030500029934F5F5F4F6F4F7F4F28E7C13BD207E8
:10306000A1F788559148AF4FBF4FC1EBD8E7ABBF31
:10307000FC01279128830196A11DB11D23962AE703
:10308000C832D207A1F7DF91CF910895CF92DF9296
:10309000EF92FF920F931F93CF93DF939AE2899F52
:1030A000800111240B581C4F83E0689F700111248C
:1030B00087E791E0489FD001499FB00D1124AE0DE4
:1030C000BF1DA55FB549D0E0C0E090E087E7C82EFE
:1030D000DD24D394F801EC0FFD1FE491E227EC937B
:1030E0009F5F1196953159F44F5F4C9DD0014D9DD6
:1030F000B00D1124AE0DBF1DA55FB54990E021961E
:10310000CA32D10539F787E0860FDF91CF911F9141
:103110000F91FF90EF90DF90CF900895EF92FF9284
:103120000F931F93CF93DF9392E1899FE0011124C6
:10313000C35DDC4F83E0689F8001112487E791E045
:10314000489FD001499FB00D1124A00FB11FA55F6A
:10315000B54930E020E090E087E7E82EFF24F394C3
:10316000FE01E20FF31FE491EC939F5F11969930FB
:1031700059F44F5F4E9DD0014F9DB00D1124A00F0B
:10318000B11FA55FB54990E02F5F3F4F2231310558
:1031900039F783E0860FDF91CF911F910F91FF9058
:1031A000EF9008951F93CF93DF93EC01142FFE014E
:1031B0008491811105C0862FDF91CF911F910895D1
:1031C00020E0412F0E94461863E0680F2196EFCF60
:1031D000382F262F562F5695569543E0852F642F6E
:1031E0000E94633E982F990F990FE82FE91BE50F76
:1031F000A7E7B1E08A9FB0018B9F700D1124E60F05
:10320000F72FF11D832F8695849FE00DF11D11246A
:10321000E55FF549317087E0831B220F2670821B22
:1032200021E030E001C0220F8A95EAF78081822BED
:10323000808308959C01ABE7B4E10E94C83EDC01A5
:10324000CB0123E1B695A795979587952A95D1F758
:1032500008959C01AFE1B5E00E94C83EDC01CB01BE
:1032600023E1B695A795979587952A95D1F7089567
:10327000CF92DF92EF92FF92CF93DF93EC01862FF4
:103280008150990BFC01EC53FD4FE491633008F43D
:1032900021979E01ABE7B4E10E94C83E6B017C011F
:1032A000AFE1B5E00E94C83EAE2FA40FBB27BB1F05
:1032B0009D012C0F3D1FD695C795D695C7952C0F10
:1032C0003D1FDC01CB0153E1B695A79597958795F6
:1032D0005A95D1F7820F931F63E1F694E794D79440
:1032E000C7946A95D1F78C1991098730910540F4FC
:1032F0008F5FDF91CF91FF90EF90DF90CF90089597
:103300000797F3CF823021F4637081F48DE1089543
:103310008150990B67E070E00E94853E62E070E0AA
:103320000E94853E9FE1981B892F08958CE10895A6
:103330008D3010F08C500895811101C08CE00895FB
:10334000CF93DF931092347D85E080931942EDE1B5
:10335000F0E4C9E3DDE7A7EEB9E6119219921D92F8
:1033600080E4E932F807C9F710922F7D1092307D82
:10337000DF91CF9108950F931F93CF93DF938091A7
:10338000347D882331F103EF19E629E33DE7CDE1F0
:10339000D0E4EBE8F1E467EE79E6D9011B969C9165
:1033A000D8018E918D01B4E08B9FA0011124892F4B
:1033B0008370842B8295807F4B85840F868B9695B6
:1033C0009695978B21503109219732976017710795
:1033D00021F7DF91CF911F910F9108951F93CF9304
:1033E000DF93182F88E1EBE8F1E4A7E1BDE7019056
:1033F0000D928A95E1F7CBE8D1E485E020E0412FFA
:10340000682F8E890E944618412F682F8F890E944D
:103410008E18229791E4C337D90781F780912F7DC9
:103420009091307D83709927892B49F420E048E002
:1034300061E088E5DF91CF911F910C94BE16DF917A
:10344000CF911F910895DC011E96FB013E963E919F
:103450002291321305C0A817B907C9F781E0089572
:1034600080E00895FC01108211821282138214827E
:103470000895DC011596FB0135963E9122912317A4
:1034800028F0321728F0A817B907B9F781E0089596
:1034900080E008956F927F928F929F92AF92BF9239
:1034A000CF92DF92EF92FF920F931F93CF93DF9310
:1034B0008B01DB011D921D921D921C921397EC0152
:1034C00022963C01BEE06B0E711CC12CD12C760102
:1034D000C394A991B0E0A70196010E94DE3EF801D5
:1034E00080809180A280B380DC01CB01880D991D82
:1034F000AA1DBB1D80839183A283B383AAE0B0E0A1
:103500000E94DE3E6B017C016C167D0611F7DF9197
:10351000CF911F910F91FF90EF90DF90CF90BF90D0
:10352000AF909F908F907F906F900895AC0190E046
:1035300070E0292F092E000C330B261737070CF0EB
:103540000895240F351FF90110829F5FF2CF4F922B
:103550005F926F927F928F929F92AF92BF92CF9223
:10356000DF92EF92FF921F93CF93DF9300D000D0B2
:10357000CDB7DEB7F894BE016F5F7F4F85EC91E465
:103580000E944A1A7894F980AA80CB80DC806F2D43
:103590007A2DC6012CE330E040E050E00E94993ED5
:1035A000E22E1CE38F2D129F8019112480931F425D
:1035B0006F2D7A2DC60120E13EE040E050E00E94F0
:1035C000993EB22E129FE0181124E0921E426F2DF8
:1035D0007A2DC60120E831E541E050E00E94993E95
:1035E00069017A0188E1289FB0181124B0921D4228
:1035F00080911D420E94981980932B42C982DA82E1
:10360000EB82FC82C701B60122E0660F771F881F9C
:10361000991F2A95D1F7605771478E4F9F4F21EB25
:103620003AE342E050E00E94993E215F3F4F4F4F06
:103630005F4F82EAC80E8FEDD81E84E2E81EF11CAF
:10364000C20ED31EE41EF51E62E0569547953795CF
:1036500027956A95D1F7C21AD30AE40AF50AA4E1BC
:10366000B0E0A70196010E94DE3E6A5879408109C8
:10367000910929E83CE140E050E00E94993E49016F
:103680005A01ADE6B1E00E94DE3EC61AD70AE80A4A
:10369000F90ADA01C90172E0B695A7959795879561
:1036A0007A95D1F7C81AD90AEA0AFB0AA8EEB3E05C
:1036B000A70196010E94DE3E29E837E740E050E08E
:1036C0000E94993E29013A018EE1289FC0181124D9
:1036D000A9E5B2E00E94DE3E28EE33E040E050E093
:1036E0000E94993EC21AC09223428EE048165104AD
:1036F0006104710498F58CE6881A82E1980AA108A1
:10370000B10881E0481A510861087108809220428E
:103710009092214240922242409123426091224263
:1037200080912042909121420E94381980932C422E
:1037300081E0809314402496CDBFDEBFDF91CF910E
:103740001F91FF90EF90DF90CF90BF90AF909F9030
:103750008F907F906F905F904F9008958BE6881ABE
:1037600082E1980AA108B1088DE0481A5108610861
:103770007108CCCF2F923F924F925F926F927F92BF
:103780008F929F92AF92BF92CF92DF92EF92FF9271
:103790000F931F93CF93DF93CDB7DEB72997CDBF9C
:1037A000DEBFC0902042D09021420D2C000CEE08CC
:1037B000FF0820902242422C042C000C550849821C
:1037C0005A8292012330310548F4245F3F4F298308
:1037D0003A8331E0C31AD108E108F108109123427D
:1037E000ADE6B1E0A70196010E94DE3E4601570119
:1037F00022E0B694A794979487942A95D1F7860EE1
:10380000971EA81EB91EC701B60120E931E040E0AD
:1038100050E00E94993E820E931EA41EB51EC70161
:10382000B60124E630E040E050E00E94993E821A62
:10383000930AA40AB50A29813A812F5F3F4FC90133
:10384000880F991F820F931F65E070E00E94713E00
:103850002EE129803A80229DC001239D900D1124E4
:10386000810F911D17FD9A95FB01E80FF91F9F012C
:1038700050E040E060E070E0CB01E9833A834B83A5
:103880005C836D837E838F8398879401A50160E0BC
:1038900070E080E090E0A980BA80C12CD12CE12CAE
:1038A000F12C00E010E00E94A03F2A5E36494A4019
:1038B00051096109710981099109E0E8AE2EF1E52C
:1038C000BF2ECC24C3940E94E93E59016A017B01BA
:1038D0008C01A0911D4240911E4240901F420A2E31
:1038E000000CBB0B20E13EE00E94D73E042C000CF4
:1038F000550866087708DC01CB01840D951DA61DCF
:10390000B71D3CE34302A0011124840F951FA11DA4
:10391000B11D1C012D01612C712C43013A82AB8336
:103920005C826D827E828F8298869C01AD0160E010
:1039300070E080E090E00E94A03F29014A01698781
:1039400079831C01F8941092D069A7EC6A2EA1E447
:103950007A2E8AE0A82EB12CC12CD12CE12CF12C8E
:1039600000E010E09201A40169857981C1010E9403
:10397000413FF30121933F019201A40169857981BF
:10398000C1010E94433F29014A01698779831C01D3
:1039900023ED31E426153705E1F665EC71E48DEF92
:1039A00091E40E94451078942996CDBFDEBFDF9147
:1039B000CF911F910F91FF90EF90DF90CF90BF902C
:1039C000AF909F908F907F906F905F904F903F90BF
:1039D0002F900895FC0195E020E08191980FDF0180
:1039E00011979A3060F49C9390E0211101C09E5F82
:1039F0002F5F2E3011F09111F0CF892F08959A503A
:103A00009C9391E0F2CFCF93803108F04AC0E82F29
:103A1000F0E0E35FF24E0C94BB3E1D1D2A1D421DDB
:103A2000531D991DB01D511DC61DCC1DDF1DF01D60
:103A3000F81D001E081E101E141E8091C4412EE0A9
:103A4000829FC00111246EE472E48B539E4BCF9190
:103A50000C9445108091C441CEE08C9FC00111248C
:103A60006EE472E48B539E4B0E944510E091C4417A
:103A7000CE9FF0011124EC54FE4B118A128ACF9193
:103A80000C94A71A8091C4413EE0839FC001112489
:103A90006EE472E48F519E4B0E94451081E080934A
:103AA0001440CF9108958091C441811126C0909116
:103AB000B44120914F4280E1289F900111248091D0
:103AC0004E42806C822B89238093B4418091B44113
:103AD0008F7339F78091CA699091CB699F7D8093EC
:103AE000CA699093CB698091CA699091CB699F7E96
:103AF0008093CA699093CB69D4CF23E040E06FE410
:103B000072E486EB91E40E9451109091B94191705A
:103B10009093B9412091B8418091B7413AE0239FF9
:103B2000800D1124911103C08093317DBACF81950E
:103B3000FBCF8091C4412EE0829FC00111246EE42E
:103B400072E483509E4B0E94451080910C4282FD8E
:103B500004C081E080931C42A4CF10921C42A1CFEC
:103B600024E040E06EE472E48FEB91E40E94511097
:103B70008AEB91E40E94321A8091B4419091B54150
:103B800094608093B4419093B5418BCF8091B441C0
:103B90009091B5419B7FF5CF4091B4415091B54193
:103BA0002091C441255F81E090E002C0880F991FF9
:103BB0002A95E2F78095909584239523E2CF409152
:103BC000B4415091B5412091C441255F81E090E01E
:103BD00002C0880F991F2A95E2F7842B952BD1CF2D
:103BE0004091B4415091B5412091C441285FDBCF51
:103BF0004091B4415091B5412091C441285FE6CF36
:103C00004091B4415091B5412091C4412A5FCBCF3E
:103C10004091B4415091B5412091C4412A5FD6CF23
:103C200081E08093C4413DCF1092C4413ACF7F924E
:103C30008F929F92AF92BF92CF92DF92EF92FF92BC
:103C40000F931F93CF93DF93082F02950F70C02F10
:103C5000D0E0E090F569F090F66920EFE22223E0F1
:103C6000F222E02AFD2AE092F569F092F669C70196
:103C70000E944914182F882381F0C701DF91CF914A
:103C80001F910F91FF90EF90DF90CF90BF90AF907A
:103C90009F908F907F900C94E50F8091A44190911C
:103CA000A5418B3F910509F469C08D3F910541F510
:103CB000CC54DD4FFE01C49180E0C7FD8BE0FC2FAA
:103CC000FF709F2E00E02C2F2071822EDBE0D81B8E
:103CD00090E0FC01E35EFF4B7F01FC2FF0727F2E32
:103CE0009C01275C32486901C074FC01E951F64926
:103CF0005F01901213C081E08093074080930540DC
:103D0000DF91CF911F910F91FF90EF90DF90CF90B7
:103D1000BF90AF909F908F907F900895882069F01A
:103D20006D2F8DE190E40E943214E12FF0E0EE5C03
:103D3000FD4B848DF70180831F5F772069F06D2F25
:103D400089E39DE70E943214E12FF0E0EE5CFD4B29
:103D5000848DF60180831F5FCC2371F06D2F87EE79
:103D600099E60E943214E12FF0E0EE5CFD4B848D69
:103D70008170F50180831F5F0F5FBBCF802FDF91C4
:103D8000CF911F910F91FF90EF90DF90CF90BF9058
:103D9000AF909F908F907F900C94031D8230A1F084
:103DA00038F08430E9F1C8F0853009F442C0089554
:103DB0006091C4418EE0689FB00111246B537E4B2B
:103DC0008EE492E40C9445106091C4418EE0689FAB
:103DD000B00111246F517E4BF3CF8091C44181110A
:103DE00017C08091B4418F7080934E428091B4414E
:103DF00082958F7080934F428091B5418F708093F0
:103E000050428091B54182958170809351420895CE
:103E100023E040E066EB71E48FE492E40C945110EF
:103E20006091C4418EE0689FB001112463507E4BC5
:103E3000C7CF24E040E06FEB71E48EE492E4EECF74
:103E40006F927F928F929F92AF92BF92CF92DF92AA
:103E5000EF92FF920F931F93CF93DF93182F12953A
:103E60001F708EE492E40E9415148091A4419091F9
:103E7000A5418B3F910509F4B9C08D3F910509F427
:103E800040C0892B79F5112359F08091F569909103
:103E9000F669807F9370812B8093F5699093F66922
:103EA0000091F5691091F669C8010E9449148823B0
:103EB000C9F00031110510F00053110987E0809F0F
:103EC000E001819FD00D1124C357DD4BAEE4B2E475
:103ED00067E04991542F52955F704F704D935D93F9
:103EE0006A95B9F7DF91CF911F910F91FF90EF90F5
:103EF000DF90CF90BF90AF909F908F907F906F900A
:103F00000895153001F580912F7D9091307D90932B
:103F100050429C0194E0369527959A95E1F72F70D1
:103F200020934F428F7080934E428091347D88233E
:103F3000C9F21330B8F21530A9F281E0809307403E
:103F400080930540CFCFE12FF0E0EC55FD4FC491B9
:103F50000BE0C7FF00E02C2F2F70822ED0E0912CB9
:103F60003C2F3071732E802F90E0DC01A35EBF4B9D
:103F70007D01BC2FB0726B2E9C01275C3248690119
:103F8000C074DC01A951B6495D01891471F2772032
:103F900069F0ED2FF0E0EE5CFD4BD7018C91848F42
:103FA000DF5F602F8DE190E40E943214662069F09B
:103FB000ED2FF0E0EE5CFD4BD6018C91848FDF5F3E
:103FC000602F89E39DE70E943214CC2369F0ED2F26
:103FD000F0E0EE5CFD4BD5018C91848FDF5F602FAC
:103FE00087EE99E60E9432149394CFCF812FDF9110
:103FF000CF911F910F91FF90EF90DF90CF90BF90E6
:10400000AF909F908F907F906F900C94CE1E6EE03B
:1040100085EC91E40E94961A6EE081EE91E40E9494
:10402000961A6EE08DEF91E40E94961A6EE083ED91
:1040300091E40E94961A6EE08FEE91E40E94961A27
:104040006EE08BE092E40E94961A64E086EB91E4C5
:104050000E94961A8AEB91E40E94321AE4EBF1E492
:10406000108A808191818064808391838081918195
:104070009160808391834AE050E069E070E082EFD4
:1040800091E40E94B73F88E080930C420C94BA1BE5
:104090006F927F929F92AF92BF92CF92DF92EF92F8
:1040A000FF920F931F93CF93DF93EBE2F0E480E650
:1040B00091E0DF019C011D9221503040E1F7E7E4DF
:1040C000FDE782EADF011D928A95E9F740E058EFAB
:1040D000DF0120E066E0A62E00E014E176E1B72ED5
:1040E00099249394FA0134913196D4913196C491E4
:1040F0003196E49111963C9311971796CC931797AC
:104100001896EC931897303108F051C0822F6A2D21
:104110000E94573E909F6001919FD00C11240D2C5E
:10412000000CEE08FF08813009F456C0823009F413
:1041300058C060E070E880E09927C60ED71EE81EE0
:10414000F91E1296CD92DD92ED92FC921597632F97
:1041500070E06D2E712C2630D0F49C92B69E7001CA
:10416000B79EF00C1124C301880F991F880F991F67
:104170008E0D9F1D855D9F4B1296CD90DD90ED902D
:10418000FC901597FC01C082D182E282F3821696E0
:10419000DC931697B69EC001B79E900D1124855DE5
:1041A0009F4BF301E80FF91F208BFC01C58B2F5F9C
:1041B0004C5F5F4F1996223109F094CFDF91CF9178
:1041C0001F910F91FF90EF90DF90CF90BF90AF9035
:1041D0009F907F906F90089560E070E081E0992754
:1041E000ACCF60E070E881E09927A7CFE62FE69595
:1041F00027E0AC01249FC001259F900D11248E5C07
:104200009D4BE80FF92FF11DE55AFF4F808160FFAC
:1042100001C082958F700895CF92DF92EF92FF9246
:104220009C01892F992782958F7066E1689FA00174
:10423000699F500D1124FA01E55DFF4B948984E0DC
:10424000989FF0011124E40FF51FE55DFF4BC0803E
:10425000D180E280F38090E080E0C114D104E104D9
:10426000F10449F13F70D701C601820F931FA11DD0
:10427000B11DABBFFC01A791A90156954795569575
:10428000479570E060E0505F6F4F7F4F4C0D5D1DB4
:104290006E1D7F1D6BBFFA014791842F90E0220FA6
:1042A000331F2670332702C0959587952A95E2F72C
:1042B0008370982F8A2FFF90EF90DF90CF90089512
:1042C00080910A6A8823E1F30E94F01390ED980F21
:1042D0009A3030F09FE9980F963020F499EA980FC1
:1042E000892F08959FEB980F963010F499ECF7CF33
:1042F000803231F390E0F4CF8A3310F0875508957F
:1043000080530895F894E8EFF9E6108A118A128A2A
:1043100078940895F89490910A6A9031B1F0E09100
:10432000096AF0E0E850F64980838091096A8F5F5E
:104330008093096A8091096A803110F01092096AAD
:1043400080910A6A8F5F80930A6A789408958091B9
:10435000240886FFFCCF08951F920F920FB60F928C
:1043600011240BB60F928F93EF93FF93E091096A9C
:10437000F0E080912008E850F64980838091096A36
:104380008F5F8093096A8091096A8F708093096AB0
:1043900080910A6A8F3028F480910A6A8F5F809337
:1043A0000A6AFF91EF918F910F900BBE0F900FBE95
:1043B0000F901F901895CF93DF93EC01FE0184912D
:1043C000811103C0DF91CF9108950E940E142196B0
:1043D000F5CF813408F0875F8F70089547E0489FDC
:1043E0009001499F300D11242E5C3D4BBC016C5F48
:1043F0007F4F8617970710F080E0089550E040E067
:10440000FA01E55AFF4FE20FF31FE081E11109C005
:104410004F5F5F4F4730510599F70196295F3F4F36
:10442000E8CF81E0089590E047E0292F30E0205761
:104430003F4F429FF001439FF00D1124ED56FD4B7D
:1044400080818A3A31F09F5F8111EFCF80931140D4
:10445000089581E0FBCF9C01ADECBCEC0E94C83E0E
:10446000DC01CB0123E1B695A795979587952A9511
:10447000D1F70895482F282F392FADECBCEC0E94BE
:10448000C83E23E196958795779567952A95D1F74C
:10449000842F2AE0629F80191124089582EC809372
:1044A000314281E08093A3418093CF69809126427D
:1044B00090E08093367D9093377D089527E731E033
:1044C000829FD001839FB00D1124A55FB549629FE3
:1044D000F001639FF00D1124E55FF5498EEE92E047
:1044E00001900D920197E1F708950F931F93CF93D9
:1044F0008C01562F4423D9F06A30C8F4C0E022233F
:1045000019F0FC012083C1E0852F90E00E943A223F
:10451000F801EC0FF11D805D8083E1E0EC0FE00F0E
:10452000F12FF11D1082CF911F910F910895252F2A
:1045300030E0ADECBCEC0E94C83E23E19695879537
:10454000779567952A95D1F7605DF8016083DBCF99
:104550001F93CF93DF93CDB7DEB72597CDBFDEBFD7
:10456000182F6091234220E041E0CE0101960E9485
:10457000752280912C4224E08202C00111242FEF89
:1045800040E0612F895496400E9430172FEF40E0A1
:10459000682F8DE20E94BE16682F8091F24280FF44
:1045A00021C02FEF40E0CE0101960E9413172FEF9C
:1045B00040E0682F8DE20E94BE16E091224294E016
:1045C000E902F00111242FEF40E0682FCF01895755
:1045D00096400E9430172596CDBFDEBFDF91CF9168
:1045E0001F9108958091224224E08202C00111248B
:1045F0002FEF40E0895796400E9430172FEF40E0A0
:10460000682F8DE20E94BE162FEF40E0682FCE018A
:1046100001960E941317DFCF1F93CF93DF93CDB77F
:10462000DEB72597CDBFDEBF182F80911C428130A9
:1046300009F040C060912B4220E241E0CE0101969A
:104640000E9475222FEF40E0612FCE0101960E945B
:1046500013172FEF40E0682F8AE30E94BE16182F31
:1046600060911E4220E040E0CE0101960E9475223A
:104670002FEF40E0612FCE0101960E941317682FA3
:1046800080911C42813079F480911D422FEF40E0EF
:104690008C30ACF080E50E94BE162FEF40E0682F12
:1046A0008DE40E94BE162596CDBFDEBFDF91CF916F
:1046B0001F91089560911D4220E240E0BFCF81E448
:1046C000EACFCF92DF92EF92FF921F93CF93DF93C7
:1046D0007C01EB01142F0E943A22805D8A839701AE
:1046E000ADECBCEC0E94C83E6B017C0133E1F6945A
:1046F000E794D794C7943A95D1F7C6018A309105CB
:10470000D8F0A70196010E94DE3E23E19695879599
:10471000779567952A95D1F7605D6883C6010E94F9
:104720003A22805D89831B82DF91CF911F91FF9098
:10473000EF90DF90CF9008951883892B79F7198334
:10474000F2CF0F931F93CF93DF93EB0197FF2FC00F
:1047500000271127081B190B873F9F4F1CF58DE27F
:104760008883C8010E943A22805D8A832DEC3CEC4C
:10477000D8010E94D73EDC01CB0123E1B695A79575
:10478000979587952A95D1F7009721F00E943A22B4
:10479000805D898383E48B831C82DF91CF911F919D
:1047A0000F91089580E288838DE28983DACF20E239
:1047B000288329838C01D5CFCF92DF92EF92FF928D
:1047C000CF93DF937C01EB010E943A22805D8B83C3
:1047D0009701ADECBCEC0E94C83E6B017C0133E15B
:1047E000F694E794D794C7943A95D1F796012A3076
:1047F000310588F0A7010E94DE3E23E1969587955A
:10480000779567952A95D1F7605D6883C6010E9408
:104810003A22805D05C080E38883C114D104B1F7DA
:104820008A838EE2898386E58C831D82DF91CF9116
:10483000FF90EF90DF90CF90089585E08093A000E7
:104840001092A4008FEF8093850689E48093080678
:1048500081E08093000680930A0680910D0680FF18
:10486000FCCF209110063091110684E036952795F3
:104870008A95E1F750E040E060E070E686E090E085
:104880000E94993E1092000681E080930D06C901B6
:1048900008952091061130910711A0910411B09153
:1048A000051181E08093A00092E490930806809324
:1048B000000680930A0680910D0680FFFCCF809150
:1048C00010069091110644E0969587954A95E1F778
:1048D000281B390B0E94C83EDC01CB01985FAF4F0B
:1048E000BF4F109200065CE0B695A7959795879507
:1048F0005A95D1F70895E62FE69527E0829FC001EB
:1049000011248E5C9D4BE80FF92FF11DE55AFF4FE6
:10491000808160FD82958F70089527E0289FD001E7
:10492000299FB00D112430E020E0F901EA0FFB1FB0
:10493000E357FD4B9081492F4F70FB0140839295C7
:104940009F7091832F5F3F4F6E5F7F4F2730310500
:1049500061F708958F929F92BF92CF92DF92EF926C
:10496000FF920F931F93CF93DF93CDB7DEB7689776
:10497000CDBFDEBFD42E8E010F5F1F4FAE01435F50
:104980005F4F780120E2D7012D937D011B961C9289
:104990001B974A175B07B9F7382F4C0120E072E0EC
:1049A000CC24C39483E0B82E882D831B8617D8F4BB
:1049B000D401ED914D01822F90E0E7FD54C0E03627
:1049C00018F4E03488F1E054800F911FDC01EC937F
:1049D000F4018081982F9D7F9C3219F08A3309F071
:1049E00040C02C3008F385E020E04D2D682FD80121
:1049F0008D918D010E9446184D2D682FF8018385F9
:104A00000E948E180E151F0579F76896CDBFDEBF80
:104A1000DF91CF911F910F91FF90EF90DF90CF909A
:104A2000BF909F908F900895E03238F0EA3349F4B8
:104A3000840F951FDC017C9314C0F0E0E85FFC4F0D
:104A4000E491EE3251F0EA3B99F3EC3209F0BCCF3D
:104A5000840F951FFC01B08204C0840F951FFC01D8
:104A6000C0822F5FBECFEAE3AFCF2F923F924F922B
:104A70005F926F927F928F929F92AF92BF92CF92EE
:104A8000DF92EF92FF920F931F93CF93DF93CDB7F7
:104A9000DEB7AB97CDBFDEBF8C015B019E012F5F00
:104AA0003F4F79013E013DE0630E711C470180E2FA
:104AB000D4018D934D011B961C921B976A167B06A1
:104AC000B9F787E0809F9001819F300D1124F90193
:104AD000ED56FD4B8081803109F08BC085E090E080
:104AE000682FF901E80FF91FE357FD4B4081411191
:104AF00003C00197A8F76FEF6F5F90E0462F50E07B
:104B000087E0809FD001819FB00D1124AE5CBD4B2A
:104B1000292F092E000C330B241735070CF1043014
:104B2000110508F047C0402F440F4F5FCE01499652
:104B30000E94AA24AB96CDBFDEBFDF91CF911F911B
:104B40000F91FF90EF90DF90CF90BF90AF909F902C
:104B50008F907F906F905F904F903F902F9008952F
:104B6000FA01E21BF30BEA0FFB1FE65AFF4F8081AD
:104B700087FD1EC0803280F48823C1F07EEF780F5D
:104B80007230B0F079EF780F753090F072EF780FE7
:104B90007F3070F08E3160F4E9E1F0E0EC0FFD1F42
:104BA0002E0F3F1FF90180839F5FB2CF8AE0F4CFC1
:104BB00082E0F2CF8BE0D5018C9380E211968C934A
:104BC00020E0822F022E000C990BFC013296EA0D98
:104BD000FB1D8417950714F01082ACCF69E170E0DB
:104BE0006C0F7D1F860F971FDC018C9180832F5FD8
:104BF000E8CF6E01B9E1CB0ED11CB601C8010E940D
:104C00008D24E091F242EBA7E3FF33C05524539487
:104C1000F3E0FFA3E091F042E295EC706091F14285
:104C20006F70F62FA98D8A8D4A2F3AE0839F400D31
:104C300011245B8D552311F184E6841B482F51E02C
:104C4000E830F1F4282F880F330B862F90E001967F
:104C5000821793070CF456C051E02817390721F446
:104C60008DA151E0853018F0E8E04A304CF0E0E0EA
:104C700007C083E0582E21E02FA3CCCFE830A1F36A
:104C80008EA1882311F08DE28983E43009F43BC1C1
:104C9000E830D1F1E11175C05E86683008F012C1CC
:104CA000D601A61BB10961E01B968C91853008F4F2
:104CB00060E0772473947F0E2DE030E0872D072C81
:104CC000000C990BD901A81BB90BAC0DBD1D7C9133
:104CD000760F60E07A3010F070E061E08E0D9F1D7D
:104CE000705DDC017C937A947110E8CF613009F03B
:104CF000ECC081E38A83552309F4E9C041508DE279
:104D00008A87E5C051E0B3CF513009F083C06624F3
:104D10006394660E862D841BD601A81BB10987FDFE
:104D2000B395772473941C968C91853008F4712C7C
:104D30001EA2642F042E000C770B1701260E371EBF
:104D4000862D062C000C990B9C01261B370B37FD7A
:104D50000EC0ADE0B0E0A81BB90BA20DB31D589674
:104D60002C91270D712C2A3018F07724739420E0B1
:104D70008E0D9F1D205DDC012C936A946110E0CFA5
:104D80005E86433609F013C1D601CE010F961C96FC
:104D90002C911C97293009F024C111978A179B0781
:104DA000B1F721E08F2FFF0F990B019639E3622FA6
:104DB000022E000C770B861797070CF0F2C081E0EB
:104DC000E83009F4F6C09A81903309F0F2C08111FD
:104DD000F0C081E38A83552309F405C14150242F93
:104DE000042E000C330BADECBCEC0E94C83EDC0181
:104DF000CB0123E1B695A795979587952A95D1F78D
:104E000020E3280F2B87405DE6EF8E9F400D112495
:104E10004C87CFC0F1E0FA0FF60FFA30D4F561E01D
:104E2000D601AF1BB109F7FDB3951C968C91853067
:104E300008F460E08F2F0F2E000C990BD601A81BF1
:104E4000B90B9D01235F3F4F28A739A71C011816F6
:104E50001CF181E0613049F481E38A83DE01A20D17
:104E6000B31D80E312968C9382E0840FD301A80FC8
:104E7000B11D5C929BA592FF84CF835018160CF055
:104E800080CFD301A80FB11D87FDBA954FA04C92DA
:104E9000F4CF652FFAE0CECFA8A5B9A54D90A8A76D
:104EA000B9A7460E4AA6B42D652FBA3010F05AA7FE
:104EB00061E09701280F391F7AA5705DD9017C93B5
:104EC0000197C5CF60E0F7E0F4CE511118CF242F41
:104ED000042E000C330BADECBCEC0E94C83EDC0190
:104EE000CB0133E1B695A795979587953A95D1F77C
:104EF00020E3280F2B8720E3240F36EF839F200D1C
:104F000011242C873ECF683008F03EC0D601A61B86
:104F1000B10961E01B968C91853008F460E071E086
:104F20007F0F2DE030E0872F072E000C990BD90161
:104F3000A81BB90BAC0DBD1DAC91A60F60E0AA304B
:104F400010F061E0A0E08E0D9F1DB0E34B2E4A0EE5
:104F5000DC014C92715039F7613001F581E38A83AD
:104F60005523A1F04150141614F48DE28A874E5F48
:104F700023E0842F622F0E94633E291B491B620E8F
:104F8000711CD3015C92A3CFF7E0C8CF4F5F842F91
:104F900063E00E94633E21E0290FF0CF5523B9F36F
:104FA000E2CF6E0D7F1DDB013C932F5F00CF4111DF
:104FB00006CF04301105C8F4000F0F5F85E020E034
:104FC000402F682FD7018D917D010E944618402FF8
:104FD000682FF70183850E948E188E149F0479F73D
:104FE000A9CD80E0EDCE4F5FFACE80E09CE22EE2CC
:104FF000D7013D917D01F501E80FF11D3083E1E01E
:10500000E80F1B963C91351111C0EA0DFB2DF11DE7
:10501000B1E05B1209C020838E5F8E149F0441F7BC
:10502000A80EB11CF501D8CD9083F6CF8E2FF5CF09
:10503000CF93DF93CDB7DEB72E97CDBFDEBFBE01D6
:105040006F5F7F4F90E00E948D248E8581111AC082
:105050009B81911111C029818D85222369F09AE0ED
:105060003C85899F300D1124832F223028F02B8519
:10507000399F200D1124822F2E96CDBFDEBFDF91E8
:10508000CF91089580E0F8CFF894E6EAF1E4118634
:1050900010861286138614861586789408958F706C
:1050A0008A3010F0895A0895805D0895CF93C82FF3
:1050B00082958F700E944F280E940E148C2F8F7043
:1050C0000E944F28CF910C940E141F93CF93DF931F
:1050D00027E0289FE001299FD00D1124CC56DD4BFD
:1050E00016E08A9182958F700E944F280E940E14BC
:1050F00088818F700E944F280E940E14115088F7EB
:10510000DF91CF911F9108950F931F93CF93DF935A
:105110008C01EC012E968A918F700E944F280E947C
:105120000E140C171D07B9F7DF91CF911F910F9146
:1051300008950F931F93CF93DF938C01EC01259675
:105140008A918F700E944F280E940E140C171D0721
:10515000B9F7DF91CF911F910F910895CF93C82F89
:10516000892F0E944F28803311F00E940E148C2F3B
:1051700082958F700E944F280E940E148C2F0E94DF
:105180004F28CF910C940E141F93CF93DF93D82FF9
:10519000162FC42F82958F700E944F2820E04C2F2D
:1051A000612F0E94BE16182F8D2F0E944F2820E0DD
:1051B0004C2F612FDF91CF911F910C94BE161F933E
:1051C000CF93DF9320E046E060E689EC9AEF0E94FF
:1051D0003017CFE1D1E116E09881412F682F892F58
:1051E0000E94C428C03191E1D90721F4DF91CF9109
:1051F0001F910895C83111F41F5F88E72197ECCF04
:105200009091B0419830BCF4E091AE41F0E0EA55A5
:10521000FE4B80838091AE418F5F8093AE41809141
:10522000AE4187708093AE418091B0418F5F809393
:10523000B04181E0089580E00895E091AE41E81B1F
:10524000FF0B3197E770FF27EA55FE4B80810895E9
:10525000F8948091B0411816BCF4E091AF41F0E0B1
:10526000EA55FE4B80819091AF419F5F9093AF4193
:105270009091AF4197709093AF419091B041915010
:105280009093B041789408958FEFFCCF1F920F92C6
:105290000FB60F9211240BB60F922F933F934F939B
:1052A0005F936F937F938F939F93AF93BF93CF93AE
:1052B000DF93EF93FF938091D0698F5F8093D069E4
:1052C0008091D06983708093D0698091B44190912E
:1052D000B54186FF28C085EC91E40E94EA1C882332
:1052E00049F08091B4419091B54182608093B4417E
:1052F0009093B5418091B4419091B54190FF13C016
:1053000065EC71E481EE91E40E94231A882359F040
:105310008091B4419091B54181608093B441909364
:10532000B541109212408091B4419091B54187FFF0
:1053300028C083ED91E40E94EA1C882349F0809103
:10534000B4419091B54188608093B4419093B54148
:105350008091B4419091B54191FF13C063ED71E428
:105360008FEE91E40E94231A882359F08091B44172
:105370009091B54184608093B4419093B54110926F
:1053800012408091B4419091B54192FF19C08AEBCF
:1053900091E40E94EA1C6FEB71E48AEB91E40E94B5
:1053A000391A882369F08AEB91E40E94321A8091BD
:1053B000B4419091B54180618093B4419093B541DF
:1053C0008091B4418F73D9F08091CA699091CB6973
:1053D00090628093CA699093CB698091CA699091D9
:1053E000CB6990618093CA699093CB6981E0809387
:1053F000E97D80911240813011F410921240809129
:10540000D069811186C080911240823049F080912C
:10541000387D882329F08091387D81508093387DB4
:1054200080911F428F5F80931F4280911F428C3377
:105430000CF46FC081E08093144010921F42809161
:105440001E428F5F80931E420E944924E82F8FEEF8
:105450008E0FEA52893114F4E9E1E81B0E2E000C9C
:10546000FF0BEA53F14EE4918091317DE80FE09318
:10547000460180911E428C330CF44BC010921E42A8
:1054800080911D428F5F80931D4280911D42883123
:10549000D4F110921D42809123428F5F809323426A
:1054A000C09123426091204270912142809122421A
:1054B0000E9482190C2E000CDD0B8C171D06BCF40B
:1054C00091E090932342809122428F5F8093224209
:1054D000809122428D305CF0909322428091204254
:1054E00090912142019680932042909321424091D5
:1054F00023426091224280912042909121420E9459
:10550000381980932C4280911D420E9498198093F3
:105510002B4281E080935301FF91EF91DF91CF9176
:10552000BF91AF919F918F917F916F915F914F91BB
:105530003F912F910F900BBE0F900FBE0F901F90B9
:1055400018951F920F920FB60F9211242F933F932D
:105550004F938F939F9381E0809313408091B34149
:10556000813089F580910840815080930840809176
:105570000840811128C080912742809308404EB195
:105580008091327D9091337D880F991F21E030E02A
:105590004F3F11F430E020E0822B932B8093327D3B
:1055A0009093337D8091327D9091337D892B59F496
:1055B0001092B341109202408FEF8FB99DE090930B
:1055C0006B0480936C0481E080930B0A9F918F9110
:1055D0004F913F912F910F900FBE0F901F901895F4
:1055E000CF92DF92EF92FF920F931F93CF93DF93AF
:1055F0008091124081118CC0D12CC2E0CC2ED4E716
:10560000ED2ED4E0FD2E11E08091F7698230F1F5A6
:105610008091294090912A4080937D4290937E42D0
:10562000D09210400E94DB0FFC01808180930F40DC
:1056300080917D4290917E422091024021110AC0CA
:105640008C3FF1E19F0739F5E0920340F09204406E
:10565000109302400E940C219C01369527953695A7
:105660002795D22E7091D169709330421092D169F2
:105670004091F769423009F4FEC1A0F4442331F1AE
:10568000413009F49EC11092F7693EC080917B427F
:1056900090917C42C1CF883C20E19207D9F6C0921C
:1056A0000240D8CF443009F4F6C108F4E7C14530D0
:1056B00051F720917B4230917C422F5F3F4F2093E6
:1056C0007B4230937C4280FDDECF9ECF40917B4277
:1056D00050917C42FA013196E0937B42F0937C42F8
:1056E000682F6370623031F1633009F459C1613061
:1056F000C1F0F901FF27EE0FFF1FEC55FF4F459159
:105700005491822FFA0109958091F76981117CCF1C
:10571000DF91CF911F910F91FF90EF90DF90CF908D
:1057200008956093F7698093F3699093F469709397
:105730001C40EACFD22FD695D695D695C22FC770EA
:10574000EFEFEC0FE73078F4F0E0E755F44D0C9410
:10575000BB3EFA2BE32BB02BE82BF12BF42BF72BD2
:105760002DE060E005C00E94DB0FFC016081262F68
:105770002093CD69D150DF3108F03EC0ED2FF0E02D
:10578000EC53F44D0C94BB3E022C062C0A2C122C2C
:105790001A2C1E2C242C2A2C302C382C3C2C422C3D
:1057A0004C2C612C662C6B2C712C772C7F2C8A2C2A
:1057B000882C912C992C9F2CA82CAD2CB32CB72C79
:1057C000BD2CC12CC52C0E94DB0FFC012081C9CF50
:1057D000609178422091794226170CF0C9CF2DE0D4
:1057E000C7CF22E062E0C4CF2CE063E0C1CF2DE060
:1057F0006DE0BECF22E0B5CF422F82E392E40E945B
:10580000651082CF422F80E492E4F9CF422F8EE4DC
:1058100092E4F5CF462F60E472E482E392E40E94C2
:105820006F1072CF462F62E372E480E492E40E942C
:1058300051106ACF462F6EE472E4EFCF462F60E43A
:1058400072E48EE492E4F3CF462F6EE472E480E4D7
:1058500092E4E5CF462F6EE472E482E392E4E7CF70
:10586000462F60E472E482E392E40E9485104CCFFC
:10587000462F6EE472E4F7CF1093D169462F70E0A3
:1058800060E0F1CF022F262F40E452E462E372E49D
:10589000CB010E94B11038CF1093D169C73061F4A9
:1058A00080918A428A3041F480913F428B3020F0CF
:1058B000895080933F4228CF022F262F50E040E0AE
:1058C000E5CF022F262F4EE452E4E0CF462F6EE4C0
:1058D00072E4CB01CACF462F62E372E48EE492E415
:1058E000C4CF1093D169462F70E060E0F7CF022F4C
:1058F000262F4EE452E462E372E4CA01CACF109349
:10590000D169022F262F50E040E06EE472E4C0CF50
:105910001093D169022F262F4EE452E470E060E02C
:10592000ECCF462F70E060E080E492E40E94F31038
:10593000EBCE462F70E060E08EE492E4F7CF022FCA
:10594000262F4EE452E462E372E490E080E0A1CFBF
:10595000022F262F40E452E4F6CF462F70E060E09D
:1059600082E392E4E3CF462F6EE472E4F9CF422F54
:1059700082E392E40E94E410C7CE422F80E492E4D6
:10598000F9CF422F8EE492E4F5CFC2E3D2E4C20F06
:10599000D11D261B4A9149832A95E1F71882B4CE7E
:1059A000822F86958F7327FD805421702713B0CEE8
:1059B000480F511D87FD5A9540937B4250937C427E
:1059C000A3CE40917B4250917C424F5F5F4F40930A
:1059D0007B4250937C421092F76960911C409C017D
:1059E000217033276217130609F092CE2091F369D4
:1059F0003091F4693695279536952795BC01E6E0F8
:105A0000660F771FEA95E1F76627262B372B81FF74
:105A100005C020937B4230937C4276CE80918342B6
:105A200090918442809385429093864280918142F6
:105A300090918242809383429093844280917F42EE
:105A400090918042809381429093824240937F4222
:105A50005093804220937B4230937C42C9010E9444
:105A60000C21892B09F050CE0E94131180937B42A8
:105A700090937C4249CE0E949A1346CE20917B425D
:105A800030917C422F5F3F4F20937B4230937C428A
:105A90000E949A1339CE882351F080917B429091D5
:105AA0007C42019680937B4290937C42ECCD109295
:105AB0007B4210927C428091347D882319F01093B0
:105AC0001240E1CD1092E97D1093D169C09212404D
:105AD0001092387DD8CD0F931F93CF93DF93182F5B
:105AE000D62FC1E001E0DC1728F4DF91CF911F91A0
:105AF0000F910895111105C08091F042816080934B
:105B0000F0420E944E22109212400093E97D0E94C2
:105B1000F02A809112408130D1F7CF5FE4CF2091FD
:105B20002D42022E000C330B2F5F3F4FAC01249F00
:105B3000C001259F900D349F900D1124019708F40A
:105B40000895EFECF7E03197F1F700C00000F6CFD1
:105B50001F93CF93DF93C0E4D4E018E01E8382E06C
:105B600090E00E948F2D1D838AE090E0DF91CF911D
:105B70001F910C948F2D20912D42022E000C330B7F
:105B80002F5F3F4FAC01249FC001259F900D349F94
:105B9000900D1124019708F4089552E05A95F1F7F9
:105BA00000C0F8CF0F931F93CF93DF93082FC0E06F
:105BB000D4E010E41E8381E090E00E94BB2D802F92
:105BC0000E94041685E090E00E94BB2D1D83DF91AA
:105BD000CF911F910F91089581E00E94D22D85E011
:105BE00090E00E948F2D84E690E00C948F2DEF9230
:105BF000FF920F931F93CF93DF9385E7E82E8EE1FB
:105C0000F82EE7012196F7011491111107C0DF91D9
:105C1000CF911F910F91FF90EF9008951F3F31F4A6
:105C200084E690E00E948F2D7E01EBCFFE018491EF
:105C30000E94D22DE70122967E01012FF7018FEFFE
:105C4000E81AF80A013021F41150C10FD11DECCF30
:105C500084910E9404160150F1CF0C94F72DCF933C
:105C6000DF93C82FD62F8AE20E94D22D89E18C0FB4
:105C70000E94041689E18D0F8C0F0E9404168BE29E
:105C80000E94D22D80E00E9404168CE70E94041628
:105C90008CE20E94D22D27E731E0D29FB001D39F42
:105CA000700D1124C29FC001C39F900D1124855F08
:105CB0009549DF91CF910C940E1660E089E00E9427
:105CC000AF1680912F7D80FF07C020E049E060ED96
:105CD00086EC98EF0E94301780912F7D81FF07C0DE
:105CE00020E049E06AEA8CEC98EF0E94301780913E
:105CF0002F7D82FF06C020E049E06CE984E30E942A
:105D0000BE1680912F7D83FF06C020E049E064E944
:105D100083E30E94BE1680912F7D84FF06C020E0A1
:105D200049E06CE882E30E94BE1680912F7D85FFDA
:105D300006C020E049E064E881E30E94BE1680913D
:105D40002F7D86FF06C020E049E06CE780E30E94DB
:105D5000BE1680912F7D87FF07C020E049E06EE4EA
:105D600081ED98EF0E94301780912F7D9091307DCA
:105D700090FF07C020E049E060E387ED98EF0E94C4
:105D8000301780912F7D9091307D91FF06C020E0EB
:105D900049E068E287E40E94BE1680912F7D9091D1
:105DA000307D92FF07C020E049E062E08BED98EF84
:105DB0000E94301780912F7D9091307D88279370BD
:105DC000892B39F420E049E060E380EE98EF0E94EF
:105DD000301789E00E941E1661E089E00C942F2E96
:105DE0004F925F926F927F928F929F92AF92BF92EB
:105DF000CF92DF92EF92FF920F931F93CF93DF9397
:105E0000CDB7DEB72E97CDBFDEBF0091F74210E0D1
:105E1000102F002700271F708091F642082B4801A1
:105E200000931840109319404FEE642E42E4742EF4
:105E3000CE0101965C0107966501F3012191D6011F
:105E40002D936D01A817B907C9F7E0901640F0909F
:105E50001740E016F10668F5F801EE19FF097F0119
:105E600080E00E941D29823009F05AC0EA94EF2890
:105E700009F056C0043011050CF452C081E00E94B4
:105E80001D2963E08232C1F485E00E945E2261E058
:105E900083E00E945E2263E080E00E946B2D0E94FE
:105EA000BB1981E00E94EE1963E081E00E946B2D36
:105EB0000EC0E01AF10AD4CF81E00E945E2265E0B4
:105EC00083E00E945E226BE085E00E945E2269E032
:105ED00081E00E942F2ED5018D915D01F301819308
:105EE0003F01AC15BD05B9F780911840909119405C
:105EF00080931640909317402E96CDBFDEBFDF9162
:105F0000CF911F910F91FF90EF90DF90CF90BF90B6
:105F1000AF909F908F907F906F905F904F9008957B
:105F20008091F04281FF14C0809115408111CFCF44
:105F300063E081E00E945E2265E083E00E945E22D1
:105F40006BE085E00E945E2281E080931540BFCF28
:105F5000109215400430110534F511950195110981
:105F6000000F111F0A5F1F4FFF24F3948F2D0F2C7A
:105F7000000C990B0817190780F4552453944424F6
:105F8000439483E0E82EF12C052D052C000C110B19
:105F90008016910660F4682D88CF60E08F2D0E94F6
:105FA000AF16F394E3CF93E0892E912CE6CF809146
:105FB000F04281608093F0420E944E221092124083
:105FC0004092E97D0E94F02A809112408130D1F701
:105FD0000E94BB19C701801B910B880F8F5F0E9425
:105FE000EE195394D1CFCF93DF9300D000D0CDB72B
:105FF000DEB780911440813009F04EC00E941D240C
:106000002091457D3091467D820F931F969587950F
:106010008093457D9093467D209128424CE251E04B
:10602000BA01EAE02E9F6019710911249B0136958F
:10603000279536952795BA01621B730B6817790768
:1060400088F582E1898385E18A8386E18B831C82DE
:106050006FEF80E00E94AF1680911140882331F0ED
:106060002FEF40E062ED87E00E94BE162FEF40E088
:1060700062EECE0101960E94131781E00E94A822D1
:1060800080E60E940C2380E00E94431661E080E0DD
:106090000E942F2E109214402496CDBFDEBFDF91B8
:1060A000CF910895B901660F771FFA01E61BF70B30
:1060B000E817F90720F482E1898384E1C5CF620FF4
:1060C000731FFA01E61BF70BE817F90720F482E1CA
:1060D000898383E1B9CF220F331F220F331F421B65
:1060E000530B4817590710F481E1F2CF80E1F0CF4C
:1060F00084E690E00E948F2D80E10E94D22D85E001
:1061000090E00C948F2D1F920F920FB60F921124D6
:106110000BB60F92CF92DF92EF92FF920F931F93E5
:106120002F933F934F935F936F937F938F939F939F
:10613000AF93BF93CF93DF93EF93FF9380EA809366
:10614000010488E080936B048FEF80936C040FB19F
:106150008FB9002309F499C010E0C801019780238A
:106160009123892B09F091C0F12CE12CDFE1CC24A3
:10617000C394D12CCE2DD0930504C6010E2C01C0A2
:10618000880F0A94EAF78093060481E090E00E9469
:10619000BB2D8EB190E08095909580239123892B23
:1061A00041F48FEFE81AF80A85E0E816F10411F7D8
:1061B000C5E08FE180930604C8010E94C43ECC0F65
:1061C000CC0FCC0FC80F80911240823079F5C730C8
:1061D00049F4109212408DE080936B048FEF80930E
:1061E0006C0409C088E080936B048FEF80936C048B
:1061F0008DE080937704FF91EF91DF91CF91BF9174
:10620000AF919F918F917F916F915F914F913F914E
:106210002F911F910F91FF90EF90DF90CF900F90F3
:106220000BBE0F900FBE0F901F901895C83220F52F
:1062300016E900EA80911B428111009307048EE564
:1062400091E00E94BB2D1150A9F78C2F0E940029CC
:10625000882359F081E08093B34124E632E3209310
:10626000034030930440809302401092124080918A
:106270001A428093387DBFCF8FEF809369049DE0F1
:1062800090936B0480936C04F0CF8FEF809369043C
:106290009DE090936B04A3CFCF92DF92EF92FF9299
:1062A000CF93DF93A7E4BDE726E036E1D7964C9184
:1062B000D7974F3F61F150E0DC968C91DC9790E0EE
:1062C000D6966C91D697613069F5DD966C91DD9725
:1062D000EC01CC0FDD1FCC0FDD1F349FF001359F8B
:1062E000F00D1124CE0FDF1FC55DDF4BD896CD908A
:1062F000DD90ED90FC90DB97C882D982EA82FB8228
:10630000E55DFF4B8E0F9F1FEC01288B658B2F5F88
:106310001996223159F6DF91CF91FF90EF90DF90DF
:10632000CF900895349FB001359F700D1124EB017B
:10633000C55DDF4BC80FD91F48894213E8CFFC0168
:10634000EE0FFF1FEE0FFF1FE60FF71FE55DFF4B80
:106350001082118212821382DACF1F93CF93DF93C0
:10636000CDB7DEB76C97CDBFDEBF11E060E0812F07
:106370000E94AF161F5F1730C9F780912F7D81FDF6
:1063800037C080912E428230F1F1833069F0813044
:1063900079F520E046E061E089E50E94BE1670E0F4
:1063A00060E082E090E022C020E042E061E084E52D
:1063B0000E94BE1620E044E061E08AE50E94BE161D
:1063C00020E046E061E089E50E94BE1670E060E0F2
:1063D00082E090E00E94352570E060E081E090E08E
:1063E0000E94352570E060E090E080E00E94352555
:1063F00066E081E00E942F2E6C96CDBFDEBFDF915C
:10640000CF911F91089520E046E061E081E40E9471
:10641000BE16E8ECF2E467E18291811102C061509E
:10642000D8F76F5F89F420E045E065E08DEC9AEFE6
:106430000E94D21885E00E94811620E046E061E0CB
:1064400081E40E94BE16D4CFE62FF0E0E055FD4B6C
:10645000CE010196DC0122912D932A2F281B2617AD
:10646000D4F345E00E94AA24E8CF7F928F929F92B6
:10647000AF92BF92CF92DF92EF92FF920F931F9352
:10648000CF93DF93CDB7DEB76597CDBFDEBF4C01AD
:106490007A01CA0140968B01041B150B6817790716
:1064A00010F000E110E040E3BE016F5F7F4FC701D5
:1064B0000E9461238DE28C831D822FEF40E06EEB02
:1064C000CE0101960E94131740E3BE016F5F7F4F1C
:1064D000C7010197800F911F0E9461232FEF40E0B9
:1064E0006EEDCE0101960E9413178E0C9F1CC12CDD
:1064F0008AE3782EAC2CB12CA016B10688F06596F4
:10650000CDBFDEBFDF91CF911F910F91FF90EF9034
:10651000DF90CF90BF90AF909F908F907F90089525
:10652000BE016F5F7F4FC501880D991D0E94352503
:10653000DC2CD694D394C0FC21C040E2BE016F5E37
:106540007F4FC5018E0D9F1D0E9461237C8A1D8A8D
:1065500020E04D2D61E0CE0141960E94131720E00E
:106560004D2D62E2CE0101960E94131720E04D2DC1
:106570006AE88CE70E94BE16C394BCCF20E04D2D84
:1065800062E9CE0101960E941317F6CF8130A9F07F
:1065900028F08230F9F0833059F1089588ED94E1C4
:1065A00084BF909368008AE990E08093260A9093D4
:1065B000270A88E080930206089588ED9CE184BF55
:1065C0009093680085E391E08093260A9093270AD0
:1065D0008AE0F0CF88ED25E230E084BF20936800A8
:1065E00080ED91E08093260A9093270A8BE0E2CF1A
:1065F00088ED2DE230E084BF209368008BE692E0C6
:106600008093260A9093270A8CE0D4CF84EF91E000
:106610000E948F2D81E38093600980912D420C941C
:10662000C63283E00E94C632E0E2F8E087E594E0FB
:106630008087918783E087838681806C868380E86A
:10664000858384E690E00C948F2DCF93DF93109296
:1066500060090E9411338CE00E940E1483ED9AEFC2
:106660000E94DB21CBE0DAE6899182958F700E944F
:106670004F280E940E14FE01319780818F700E9476
:106680004F280E940E148AE7C832D80769F78AE0BB
:106690000E940E1489ED9AEF0E94DB2184E00E9493
:1066A0000E14DF91CF910C9406330F931F93CF9369
:1066B000DF93109260090E9411338CE00E940E1447
:1066C0008AE00E940E1487EF9AEF0E94DB21D0E04F
:1066D000C0E0CE010E94EE218823E1F0CE01C0315E
:1066E000D10508F0C0960E94AE2880E20E940E14E8
:1066F00010E000E0C8018C0F9D1F0E94652880E219
:106700000E940E140F5F1F4F0430110599F78AE0A5
:106710000E940E142496C03C43E0D407D1F681E4D5
:106720000E940E148AE30E940E1480E20E940E144E
:1067300082E392E40E94842880E20E940E1480E2A8
:106740000E940E1482E40E940E148AE30E940E142A
:1067500080E20E940E1480E492E40E94842880E289
:106760000E940E1480E20E940E1483E40E940E1414
:106770008AE30E940E1480E20E940E148EE492E4DA
:106780000E9484288AE00E940E1483E50E940E1461
:106790008AE30E940E1480E20E940E14CDE0D0E045
:1067A00001E010E020918B4230918C42C8010C2E08
:1067B00002C0880F991F0A94E2F782239323892B42
:1067C00009F055C080E30E940E14219758F78AE023
:1067D0000E940E148DE40E940E148AE30E940E148F
:1067E00080E20E940E148CE592E40E94842880E2EC
:1067F0000E940E1480E20E940E148EE40E940E1479
:106800008AE30E940E1480E20E940E148AE692E44B
:106810000E94842880E20E940E1480E20E940E14DE
:1068200087E40E940E148AE30E940E1480E20E9404
:106830000E14809188428F700E944F280E940E147F
:10684000809187428F700E944F280E940E148AE028
:106850000E940E1489ED9AEF0E94DB2184E00E94D1
:106860000E14DF91CF911F910F910C94063381E3A9
:10687000AACF82E390E00E948F2D8091B3418130B6
:1068800011F080E008957299F8CF81E20E94D22D34
:106890000E94253380E20E94D22D81E008952F923C
:1068A0003F924F925F926F927F928F929F92AF92A0
:1068B000BF92CF92DF92EF92FF920F931F93CF93ED
:1068C000DF93CDB7DEB76C97CDBFDEBF8091EA42D4
:1068D00020E1829FC00111242091E94222952F706E
:1068E000822B20E032E04901881A990AAC0140531A
:1068F00051094B8F5C8FD12CC12CF12CE12C512CE8
:1069000043EB642E4DE7742E2FEF31E0D901A81B25
:10691000B90BA98FBA8F0E946A166FEF80E00E94B0
:10692000AF166FEF89E00E94AF166FEF8AE00E940A
:10693000AF16B6E05B9EC00111242FEF40E061E08E
:10694000895296400E943017E1E1E51520F1E52DCE
:10695000F0E0E355FB4C0C94BB3EBF3415352B35B2
:10696000093613362236ED354F35FF349935593512
:10697000D636883655370A353B35CB34473706E3AC
:106980001BEF27E23BEF43E15BEF62E27BEF89E045
:106990009BEF0E945A176BE080E00E942F2E80EA46
:1069A0008093020480915000897F8460809350001E
:1069B00080915000816080935000889580915000B4
:1069C0008E7F809350008091387D811150C310924A
:1069D00012406C96CDBFDEBFDF91CF911F910F911A
:1069E000FF90EF90DF90CF90BF90AF909F908F90EF
:1069F0007F906F905F904F903F902F90089502E3AB
:106A00001BEF2FEF3BEF4DE15BEF6EE97BEF87ED87
:106A10009BEFBFCF02E31BEF2CED3BEF47E15BEFBA
:106A20006CE27BEF8EE09BEFB4CF02E31BEF2CE731
:106A30003BEF41E85BEF64E87BEF87E89BEF0E9468
:106A40005A1780912E420E94C71787E00E94EE19C4
:106A50000E94AD31A0CF02E31BEF23EC3BEFA90175
:106A600065E47BEF8AE49BEF0E945A1780911B42FA
:106A70000E94C71790CF02E31BEF26E13CEF40E1F5
:106A80005CEF62EE7BEF85EE9BEF0E945A178091E0
:106A900029420E94C71780912A428E5FE9CF02E304
:106AA0001BEF23EC3BEFA9016EE87BEF89E89BEF3E
:106AB00070CF02E31BEF23EC3BEFA901B901C90141
:106AC0000E945A1735EFA32E32E4B32E212C442412
:106AD0004394322C34E03E8B07E010E020E241E0AA
:106AE000632DCE0101960E947522D5018C9190E014
:106AF000002E02C0959587950A94E2F720E080FF6A
:106B000026E6442D6E89CE0101960E941317339418
:106B100001501109BE89B05EBE8B0F3F1007F1F620
:106B20004394F8E02F0E21E0A21AB1084F12D1CF02
:106B300032CF8114910409F449C081E040E1C416C8
:106B4000D1040CF480E09601215F3F4FA98DBA8DEE
:106B50002A173B0708F4826002E31BEF23EC3BEFAC
:106B6000A901823061F1833071F1B901813049F5B9
:106B700089E99BEF0E945A172FEF40E06CE583E410
:106B80009AEF0E94301740E2BE016F5F7F4FC40151
:106B90000E9461232FEF40E064E8CE0101960E943D
:106BA00013178114910431F0A601B4018B8D9C8DD3
:106BB0000E94353268E081E00E942F2EECCE64E91D
:106BC0007BEFC901D7CF64E97BEFD2CF02E31BEFA4
:106BD00023EC3BEFA901B901F4CF02E31BEF26E759
:106BE0003BEF41E75BEF6CE67BEF87E69BEF0E94B4
:106BF0005A1780911A42883751F0803F21F08C3328
:106C000021F480E035CF82E033CF83E031CF81E0E3
:106C10002FCF02E31BEF23EC3BEFA90160E47BEFF6
:106C20008BE39BEFB6CE02E31BEF21E63BEF4BE598
:106C30005BEF65E57BEF80E59BEF0E945A17809143
:106C40002D4216CF2FEF40E061E68DEA9AEF0E94C9
:106C5000301720E042E061E084EE98EF0E943017A8
:106C600020E043E061E084E099EF0E94301720E0EB
:106C700044E061E084E299EF0E94301720E045E0B3
:106C800061E084E499EF0E9430170E94DF280E949F
:106C90001D242091457D3091467D820F931F96954E
:106CA00087958093457D9093467DBE016F5F7F4FB2
:106CB0000E94DC232FEF40E062EDCE0101960E949E
:106CC00013170E944924BE016F5F7F4F815191408D
:106CD0000E94A1232FEF40E062EACE0101960E94BC
:106CE000131720E046E061E080E899EF0E9430173A
:106CF00020E048E061E084E699EF0E94301702E36B
:106D00001BEF23EC3BEFA901B9018FEA9BEF41CECA
:106D100020E042E04F0D61E088E00E94BE160CE6E4
:106D20001AEF82E0B82E20E04B2D69E0C8010E94E6
:106D30003017035F1F4FB394B7E0BB12F4CF0AE0E4
:106D400010E0B12CBAE0AB2EE4E0BE1223C080917B
:106D50002842BE016F5F7F4F8A9DC00111240E94AF
:106D6000DC2342E04B0D20E06CE6CE0101960E9450
:106D70001317B3940F5F1F4FF5E0BF12E5CF02E387
:106D80001BEF2FEB3BEF4BEB5BEF66EB7BEF83EB0C
:106D90009BEFFFCDF801E65EFD4B808140E3BE0135
:106DA0006F5F7F4F90E00E946123DBCF02E31BEF18
:106DB00023EC3BEFA90168EC7BEF89EA9BEFEE2027
:106DC00011F083EA9BEF0E945A1728E0E29EC0016F
:106DD000112426E1289F8001299F100D1124055DB3
:106DE0001F4B412C8E2D880F880F880F8150888F64
:106DF0004394888D840D0E944F2820E0442D62E04A
:106E00000E94BE1618013CE03E8BB12CA12C20E064
:106E1000442D6E898CE70E94BE16F10181919191FB
:106E2000A191B1911F01892B8A2B8B2B49F1F8017C
:106E3000EA0DFB1D808929E0289FF0011124E95B00
:106E4000F248908126E6911120E037E0839FC0014F
:106E50001124442D6E89665F885B97400E9430172D
:106E60004FEFA41AB40A5E89545C5E8B84E0A816C6
:106E7000B10469F60A5E1F4F98E04912B9CF8BCD75
:106E800026E6442D6E89645F80E59AEFE7CF02E342
:106E90001BEF23EC3BEFA9016AE07CEF84E09CEF61
:106EA0000E945A1780912F42E3CD43EC5BEFA7E499
:106EB000AA2EADE7BA2EF5019A0186A9882311F012
:106EC00029EE3BEF39966E167F06B9F78F2D0F2C02
:106ED000000C990B069669E0689FF001699FF00D20
:106EE0001124E95BF24881818F3F39F0808140E4D1
:106EF0005BEF882311F041ED5BEF02E31BEF66EBE4
:106F00007BEF83EB9BEF0E945A1720E041E068E0A3
:106F100085EB9AEF0E94301720E041E06AE885EBAC
:106F20009AEF0E9430171FE181E020E042E0682FD5
:106F30008BE10E94BE161150C1F720E042E068E7E5
:106F40008EE00E94BE1620E041E068E78CE70E94D8
:106F5000BE168F2D66E00E94633E9D5F988F8795D9
:106F6000882787958F5F8F8B02E718EF1E8AD501E0
:106F7000D6968C91412C813011F0F6E64F2EBE89C9
:106F8000B63088F53B2EE3E03E0E242D432D6AE01B
:106F9000C8010E943017D501D7968C91242D432D1E
:106FA00061E48F3FB1F10E944F28242D432D62E40C
:106FB0000E94BE16282EF50184AD8F5F0E944F28D7
:106FC0006FE0620D242D432D0E94BE16282ED501A0
:106FD000DE968C910E944F2860E1620D242D432D96
:106FE0000E94BE161AC03E88BDEF3B0E20E0432D26
:106FF00068E78CE70E94BE16242D432D6AE8C8017D
:107000000E943017F50187A98F3FC9F4242D432D25
:1070100063EC87E59AEF0E94301720E0488D6F8976
:1070200088E00E94BE16FE89FF5FFE8B29E0A20E5B
:10703000B11C095F1F4FFC3009F099CFACCC0E9406
:107040004F28242D432D64EC0E94BE16282ED50116
:10705000DC968C918F5F0E944F286EE0620D242D8C
:10706000432D0E94BE16282EF50186ADB3CF809128
:10707000B441857029F48091B341882309F492CCFE
:107080000E942829182F0E943934813009F41FEFFB
:107090000E94442831E1351508F1E52DF0E0ED5A64
:1070A000F74C0C94BB3E65389038AC382539603AC3
:1070B0007D3AFE38D638323AE238E638CA3A863A6D
:1070C000E63A493ABB386E38D73A103109F450C322
:1070D00000F5112339F0183009F463C2133011F0B0
:1070E000173081F50E946A166BE080E00E942F2E17
:1070F00081E0809314400E94F32F0E94BB1987E027
:107100000E94EE1962E087E00E942F2E0E94AD31AE
:1071100060CC183109F429C3103201F711E09BC08B
:107120001031C1F048F4112309F495C083E0183000
:10713000A9F680932E4206C0183151F0103271F634
:1071400010922E428091B441857009F4E4CBCACFED
:1071500081E0EFCF82E0EDCF183149F0103221F01D
:107160001111BCCF1EE077C010921B42EBCF81E023
:1071700080931B42E7CF1031B1F048F4112391F313
:10718000183009F0ABCF81E080932A42DBCF183171
:1071900031F0103209F0A2CF10922942D3CF81E012
:1071A00080932942CFCF10922A42CCCF183139F0A8
:1071B000103209F4E6C2111191CF512CC3CFEAE08D
:1071C0005E2EC0CF183171F0103221F0111186CF30
:1071D00017E041C040E1C41AD108D7FEB3CFD12C8B
:1071E000C12CB0CFC6010F96A98DBA8D8A179B0707
:1071F00008F0A8CFB0E1CB0ED11CA4CF1031C9F05C
:1072000048F41123F9F01830B1F080911A428093BC
:10721000387D64CF183159F08CE31032B1F7809388
:107220001A428091F042877F8093F042EECF88E748
:10723000F6CF80EFF4CF8FEF80931A428091F04227
:107240008860F2CF7EE0572EE0CF183149F010323F
:1072500021F0111143CF512E75CF0E94553372CFBB
:1072600020E044E062E08FE59AEF0E94301761E091
:1072700084E00E942F2E85E0E9E0F0E4DE015196E3
:1072800001900D928A95E1F7109260090E941133E6
:107290000E9427148AE00E940E148EED9AEF0E943D
:1072A000DB210E94822157E0652E7E01E1E1EE0E96
:1072B000F11C60E3762E10E080910A6A882361F069
:1072C0000E94F013F701E10FF11D9081891719F069
:1072D000123008F073C01F5F0E9428298F3F11F4FD
:1072E000143051F70E94F0138A3009F069C0DD2490
:1072F000D394798A7A8A7B8A00E010E080910A6AC6
:10730000882369F00E94F013082F80ED800F8A30E7
:1073100008F076C0F701E10FF11D00831F5F0E94A6
:1073200028298F3F31F4003249F7F3E0DF1609F4E2
:1073300094C0012F10E05701A00EB11ED12CC12C1A
:107340008501AE14BF0409F070C0B0E1CB16D104C2
:1073500018F0E0E3CE1AD1086C9C80016D9C100DF2
:1073600011240E5C1D4B94E0B92E85E0C82ED12C63
:107370000E946021A82EA29420EFA2220E946021E8
:10738000F601E45AFF4FE00FF11F8A298083F1E0F4
:10739000CF1AD1082EEFC2162FEFD20649F7BA94B2
:1073A000095F1F4FB110E1CF0E94F0138A3009F43A
:1073B0009ECF0E9428298F3FB9F399CF10E08CCF40
:1073C0000E9428298F3F09F48DCF82E09BEF0E9415
:1073D000DB210E9427140E94AB0F83EF9AEF0E94DB
:1073E000DB210E9406330E946A166BE080E00E9457
:1073F0002F2E81E08093144083E00E940029E9CA87
:107400008FE9800F863008F485CF8FEB800F8630B0
:1074100038F4F701E10FF11D80E2800F80837ECF09
:107420000A3309F07CCFD52C7ACFD5018E914D014E
:107430000E947C2190E098012A193B09220F331FFA
:10744000220F331F02C0880F991F2A95E2F7C82A1E
:10745000D92A540176CF0E94F01380910A6A8111D3
:10746000FACFB9CF103109F486C148F4112309F4D9
:10747000A4CE183009F032CEB1E15B2E63CE1831C4
:1074800021F0103209F46ECE29CEE12C1BE0512EF2
:1074900059CE103109F472C148F4112309F481C0A6
:1074A000183009F01BCEFFE05F2E4CCE183129F0CA
:1074B000103209F013CE12E0CECEA6E05A2E42CE04
:1074C0001031B1F050F41123A9F083E0183069F0C5
:1074D00080912D420E94C63201CE183129F010321F
:1074E000B9F710922D42F4CF81E080932D42F0CF76
:1074F00082E0FBCFEEE05E2EEBCF112309F451C00A
:10750000103209F0EBCDF12C1CE0A5CE103171F159
:10751000D8F4112309F439C1183009F0DFCD8F2DCB
:107520000F2C000C990BFC01EC5DFD4B20812150D0
:107530002083209128422F3108F404CE8D5D9D4B8D
:107540002EE1FC012083FECD183149F0103209F004
:10755000C5CDFA94F7FEF6CD94E0F92EF3CDF39471
:1075600034E03F150CF0EECDF12CECCD8F2D0F2C2F
:10757000000C990BFC01EC5DFD4B20812F5F2083FB
:10758000209128422F3108F4DDCD8D5D9D4BDC012B
:107590001C92D8CD183109F4FAC0103229F011111B
:1075A0009DCD88E0582ECECD81E0E826CBCD183198
:1075B00049F0103221F0111191CD18E04CCE10920B
:1075C0002F42C0CD81E080932F42BCCD103109F411
:1075D0006EC078F4112309F4DDC0E7E4FDE718304C
:1075E00009F07CCD16AA3996BDE7E33BFB07D1F73E
:1075F000A9CD1831C1F1103209F070CDFA94F7FE1F
:1076000002C07BE0F72E8F2D0F2C000C990B0197F9
:1076100010F48BE090E049E02F2D0F2C000C330B81
:107620002A5F3F4F429FD001439FB00D1124A95BB9
:10763000B2489C012A5F3F4F429FF001439FF00DEB
:107640001124E95BF24818963C91208532137ACDDB
:10765000019797FF02C08BE090E0FA94F7FEDCCF31
:107660006BE0F62ED9CF8F2D0F2C000C990B0696C0
:1076700029E0289FF001299FF00D1124E95BF248D1
:10768000208539E0F3944BE04F150CF4F12C8F2D4D
:107690000F2C000C990B0696389FF001399FF00DC6
:1076A0001124E95BF2488085821761F34BCD8F2D61
:1076B0000F2C000C990B069629E0289FF001299FBA
:1076C000F00D1124E95BF24840852081211139C079
:1076D00007E41DE7F80186AD841320C087E49DE729
:1076E000DC01DE965C91DE975417A1F037A9D7969E
:1076F0002C9132130FC027E43DE7D901DE966C913F
:10770000DE97561302C0D6961C92275F3F4F621633
:10771000730699F709966816790611F739966E1669
:107720007F06C9F681E0D801DE969C91DE9794131E
:1077300002C0D6968C93075F1F4FE017F10799F7A9
:1077400001CDE7E4FDE726AD241301C016AA399662
:107750006E167F06C1F729E0289FF001299FF00DE2
:107760001124E95BF2481082EDCC57E0552EEACCAB
:1077700043E0542EE7CC35E0532EE4CC24E0522EE7
:10778000E1CCD12CC12C19E066CD15E064CDF12CF3
:107790001DE061CDE12CF12C1BE05DCD1F93CF935B
:1077A000DF9382E080932D4280912D420E94C63269
:1077B00080917C008E7F98ED94BF80937C008091B7
:1077C000630083FDFCCF90917C0088ED9B7F84BF9C
:1077D00090937C0090917C00926084BF90937C0099
:1077E00090917C00916084BF90937C0080914101D6
:1077F0008111FCCF82E08093470114E01093400197
:1078000010924601C1E0C093520181E6809350017D
:10781000C0930A0A1092010A8091090A8E7F809310
:10782000090A86E08093000A8091000A81608093B3
:10783000000ADFEFD093000480EC809304040E94E0
:10784000EC15D09362048DE080936B04D0936C04AC
:10785000D093690410930106109200060E944428F8
:1078600087E380931F428BE380931E4210921D4258
:107870008CE080932B42D5E0D093234283E0809329
:10788000224285EE97E080932042909321424091DE
:1078900023426091224280912042909121420E9495
:1078A000381980932C42C0931440C0932E421092FA
:1078B0002F421092D069C0931C4210921B4288E75D
:1078C00080931A4284E6809324428CE1809325427F
:1078D0008CE380932642D093274288E1809328420C
:1078E000C093294210922A420E941D248093457D14
:1078F0009093467D80911A428093387D7894DF91F1
:10790000CF911F9108950E94CE3B0E94A82D0E9406
:10791000F72D0E946A166BE080E00E942F2E0E94D5
:10792000F32F0E94AD310E9407200E9444280E943C
:1079300027140E94AB0F0E9448200BE811E480EA54
:10794000F82E92E0B92EC1E028E0E22EDFEF3DE014
:10795000D32E40E8C42EA090124081E0A81609F46E
:107960001DC1A81608F485C082E0A812F4CF1092B9
:10797000E97D1092387DEBE2F0E4148A769681E49A
:10798000EB38F807D1F7E0926B04D0936C04DFB9C1
:1079900080912942813071F40E9402186BE080E0EE
:1079A0000E942F2E90912A42990F990F80E09C5FA0
:1079B0000E948F2D0E946A166BE080E00E942F2E9D
:1079C0000E9478300E944428E0926B04D0936C04AB
:1079D000D0927704CFB880915000897F84608093E3
:1079E0005000809150008160809350008895809174
:1079F00050008E7F8093500080911240823059F366
:107A00000E94F72DC09204040E944C3182E390E062
:107A10000E948F2D739906C00E9427140E94AB0FFD
:107A20000E9448208091B341813009F4B2C0C093D4
:107A3000E97D10927B4210927C421092F769C093CC
:107A4000D1691092CF69C093347D0E94BB190E9406
:107A50005D2E0E94AD31C09314400E94F32F6BE065
:107A600080E00E942F2EDFB9D0926B04D0936C047B
:107A700072CF8091244290E080931A4090931B40F3
:107A800080911340813021F08091024081114AC0E1
:107A90008091CF69811116C00E9428298F3F91F0F3
:107AA000E82FF0E0E053FD4FE491E0933142C093C2
:107AB000A341C093CF698091264290E08093367DA8
:107AC0009093377D0E94F02A80910240813061F4CA
:107AD0008091034090910440009709F457C00197AA
:107AE000809303409093044080910540813079F465
:107AF0008091254220911A4030911B40820F932F94
:107B0000911D80931A4090931B40109205408091E4
:107B10001A4090911B40019780931A4090931B400C
:107B20001092134080911A4090911B40892B09F0CC
:107B3000A7CF809106408823B9F020912F7D309106
:107B4000307D80910040909101402817390751F015
:107B50000E945D2E80912F7D9091307D809300401A
:107B6000909301401092064080910740882359F07D
:107B70000E94BB1987E00E94EE1962E087E00E9434
:107B80002F2E109207400E94F32FE5CE1092024054
:107B9000ABCF82E390E00E948F2D44CF0E9413224E
:107BA000A09214400E94F32F10920240EBE2F0E406
:107BB000148A76960E171F07D9F780912F7D81FDC5
:107BC0004CC00E94AD310E94BB1987E00E94EE19A3
:107BD00062E087E00E942F2E67E08BE00E945E2229
:107BE000F092020480915000897F8460809350005D
:107BF0008091500081608093500088958091500062
:107C00008E7F809350000E94F32F8091387D8111E8
:107C100005C08091F04283FFB09212408091B34141
:107C20008130A1F410921240E091AF41F0E0EA55AA
:107C3000FE4B8081833041F40E9428290E94393410
:107C4000811102C00E944F340E945D2E809112402B
:107C5000813041F2F09201047ECE80912F42882340
:107C600009F4AFCF81E00E941D298332B9F482E08C
:107C70000E941D29823291F480E00E941D298D31DD
:107C800009F49FCF80E00E941D29853109F499CF26
:107C900080E00E941D298D3009F493CF80E00E947E
:107CA0001D29823209F498CF0E94F02E95CF991B9E
:107CB00079E004C0991F961708F0961B881F7A95E3
:107CC000C9F78095089587FB082E062687FD8195C4
:107CD00067FD61950E94573E0EF4919507FC8195D2
:107CE0000895AA1BBB1B51E107C0AA1FBB1FA61703
:107CF000B70710F0A61BB70B881F991F5A95A9F755
:107D000080959095BC01CD01089597FB072E16F440
:107D1000009407D077FD09D00E94713E07FC05D082
:107D20003EF4909581959F4F0895709561957F4F92
:107D30000895A1E21A2EAA1BBB1BFD010DC0AA1FAC
:107D4000BB1FEE1FFF1FA217B307E407F50720F0C4
:107D5000A21BB30BE40BF50B661F771F881F991F3F
:107D60001A9469F760957095809590959B01AC0188
:107D7000BD01CF010895EE0FFF1F0024001C0BBEB4
:107D80000790F691E02D09940E94A93F8A950895E5
:107D9000A29FB001B39FC001A39F700D811D11244C
:107DA000911DB29F700D811D1124911D08950E9497
:107DB000C83EB7FF0895821B930B08950E94C83EEA
:107DC000A59F900DB49F900DA49F800D911D11242F
:107DD0000895DF93CF931F930F939A9DF02D219FCA
:107DE000F00D8B9DF00D8A9DE02DF10D039FF00DA0
:107DF000029FE00DF11D4E9DE00DF11D5E9DF00D09
:107E00004F9DF00D7F936F93BF92AF925F934F930F
:107E1000D5010E94C83E8B01AC01D7010E94C83E2B
:107E2000EB01E80FF91FD6010E94383F2F913F91D7
:107E3000D6010E94C83EC60FD71FE81FF91FAF9199
:107E4000BF910E94383F2F913F910E94C83EC60FBC
:107E5000D71FE81FF91FD6010E94C83EE60FF71F83
:107E60009801BE01CF010F911F91CF91DF9108952D
:107E70000E94C83E460F571FC81FD91F08F43196ED
:107E80000895689401C0E8948F929F92CF93DF93F6
:107E90000E944F3FDF91CF919F908F90089588244B
:107EA0009924F401E401B0E49F93AA279A158B0466
:107EB0009C04ED05FE05CF05D007A10798F4AD2F72
:107EC000DC2FCF2FFE2FE92D982C892E982F872F6E
:107ED000762F652F542F432F322F2227B85031F79A
:107EE000BF9127C01B2EBF91BB27220F331F441FFA
:107EF000551F661F771F881F991F881C991CEE1F2E
:107F0000FF1FCC1FDD1FAA1FBB1F8A149B04EC059B
:107F1000FD05CE05DF05A007B10748F08A189B08CC
:107F2000EC09FD09CE09DF09A00BB10B21601A9401
:107F3000E1F62EF49401AF01BE01CD01000C0895CD
:107F40002A0D3B1D4C1D5D1D6E1D7F1D801F911F49
:107F50000895AA2781110C94B13FA8E0892BD9F785
:107F60000895A3958695E8F78A2F99270895DC014F
:107F700001C06D9341505040E0F70895F894FFCF51
:0E7F8000FF0001C80001010105505834310016
:108000000106B5064E70F858985684D84C5B8C4BD8
:108010004C3B1C427070384BAE783C0670B958CE61
:108020008CA08D08849B76761908AE58FC58F3997D
:108030009E990AB5960D9E1596BD966262C6CA5067
:108040001C231908AE58FC58E21BE2371100EE5C05
:10805000981C45028CA08411008D08580CA0B5A274
:108060007B9BCBC313E3DB4B43CB3B434B535BBD0E
:10807000B25100E30E1C5016B523110CAE0E93C482
:108080008370FA70A033F0B80E6150F86550C4F0F8
:108090007C30147C3050BCE0C8CCF73008C8CC66CB
:1080A000EBE0D5884FA550F0D44FA550D43FA8F0B1
:1080B000EECBA550AEB87C58AE8CA74C3344983C60
:1080C000A883B5BC84634C6100431300A550EED473
:1080D000D3B87C588C33A3B070E0A550EED433B83D
:1080E0007C588CC378A84E703868F828EEE8B5BC88
:1080F0008860A04E70B85860434C3748ED04711C3E
:10810000EC1F0C1B919CCC9BCCA3203C560630183A
:108110006621463087662F110C1D02C8CC5C5AD0F0
:108120007038CC9704624728707C3014FCE090666D
:10813000281C70381B2E28BC30EB33B898A8E00000
:10814000A383634323387C8338FC6B383C53387CEF
:108150003B387C2338083C8C1BADBC300670FCE0FF
:1081600048711C8C7F0C238914538C2B0441B02341
:10817000F8992C4C3F305166FB610044ED040CC76C
:108180000100D50CCC0F3008999C0CCFB83C580C92
:10819000D91C6000711CEB5924305006CC4F300CB8
:1081A000B19CA6CB091E201CE2153221460100E03D
:1081B000D50CCC3F300A999C0CBBB8F10C7CD80490
:1081C000884484D83C467CA8C46100CC4B30C306AC
:1081D000203C1C6ADB78EE30BF0E66267BA606705C
:1081E00038EE4B3EB75EF0FC56468B300770999CDC
:1081F00051844E7020B8BC588CC50284983CA8E0CD
:108200006D5820091EC8CC6046F070306906787C35
:10821000660FBC6670380EBAF038BA6EB7F04670AA
:10822000B858CCA03846BC30E660C4783C1C420A42
:10823000BD8E60A0587058585870707070E0DCA007
:10824000C44484C44404B1702DD91C610030FF0EB5
:108250004EF0E020F0AE70AEF0A6DB309C3C30A7D4
:108260003C309B685A2E28704E9C103020E84E708F
:108270009C90105C1010A8883006999C3069067894
:108280007CA63C68D5060ECC1F4CA038CC432E28CB
:10829000BC30B606E00C6B90662870387C1C0A1C5B
:1082A0004E70E06228E01908AE581C58F6BDBE4476
:1082B000F64348F62BF6603D02568C33841100B12C
:1082C0000EAE8E301EC63F4CC3301AC6A36E3008A9
:1082D000EE4E702E3C86F313EE66F3EEB8AE3D0222
:1082E000D588387E7E8953065E04467056607CA62B
:1082F0004708FCA627FCA64B3CED08E606E6E6464A
:1083000046FC06E01C8ECECC474C37784C1758E024
:10831000CC8338BC3AEEE2DFCE308E1A3C7E1E4E65
:108320001CAE3A30AEAA3CBECB133CEAF358AE6E5C
:108330001C53CE3A303C46FC6E1A3A3CEA38CA2806
:10834000E044E23349A459A41B49A4E5A43C1E4ED1
:10835000BE4F58E5A4D898D83CBB2550581CDD8C9E
:108360006EB858E065BC8C1BCCA0044841B0336D9E
:10837000BCCE992CF90C8C2F3C580C6765204670AC
:10838000B85888D3C4B83C5804987C58042B492466
:10839000B8587CD804D8FCD88404D87C8498A8E049
:1083A00085BC390C048CBBB85804ED04C4E0B01A89
:1083B00030E61B1C50BCAEC1B0AE4D14DDAC492440
:1083C00065205DBC651C4C752EB85888987C580893
:1083D000983CA81D02B85884987C5804A341B0F971
:1083E0000C3330A7C8CCF91E66DB2DAA8D08F681A8
:1083F0000B1C98B10A30FD70F0B8150A46A809BAEE
:108400008BA3ABDBB3ABA39B93FBA3F3032B23C9DE
:108410001230CFA663B51230903B1D140912309173
:108420000286061D146684E37330D04330CE0663A3
:1084300065169C021D1411B41DB4D884D81B30A835
:108440000629BF30AE06AF19B4D8D91C8C2330E052
:108450001B30D02D149388309C0613841D1411B446
:1084600006D91CA6D88C7384D884E6BD1C090E04DA
:10847000DD14661BD806163066066B1E7E8C177ED2
:10848000A1140CDDAC5D1E307006C7668B307466BF
:10849000D3069B3071463C301A7E3766EB305C4623
:1084A000E80B3065DB307A4636BB30689B301D0602
:1084B000CB3B301A06CF6667B8D8485CA2E2178873
:1084C000D8E88B266637DD1430053B302D23A61CFB
:1084D000D0E51411B46E5606D91C301D1C621F065F
:1084E000970C2B301FE5140912E6161D1411B46EFB
:1084F000060404CC13081C02A65A56BC1AD91CB890
:108500003007E8BAEF6E49241C0C2DB50CE5A46EBB
:1085100006D91CA675B0E9145B6E3DA41DB48E0689
:10852000D91C1C627330CF2D1449246E3DA46EAE4D
:10853000C512AA625830C02D14CCEF8CDBE0B8B85D
:108540003044E86914061ED91CA1143020E8F89CB8
:10855000E213A83060A820045330C848C8CCA066F5
:10856000E34404048449242DA806864C2BAD7043B3
:1085700093C1B01EA114C66FCC4F6914061ED91C3E
:10858000A11409123020E84924B80E41A41DB41CDE
:10859000EAE38E56063C3040FCE0BD1C2012050785
:1085A000204924785A0E43660E7038EE477A30C060
:1085B000661BAEA3AE3CE03020E80C57302006F836
:1085C000A85666A00879B2D91CA6063C30147C30A7
:1085D0001C50BC087A3056D84C1B36448C1B048483
:1085E000D8E80C8F3020E8E09E4EA0A60E3C266610
:1085F000EEEEEEEEE6A63C266606BEEEEEEEEE06ED
:10860000AEFC2E6E0E60DE77DC101E7CFE7FFCBEA4
:10861000FE5FFCBE437E9EBE1F3CEB7E3C1A9EFC72
:108620009CBE603003FCE8D34670CEED28041413E2
:1086300008AE58FECD7DE05CE0D460D0DC6202D7AD
:10864000629362E97CE0C2E223302C1B302ED4A07E
:10865000D57C33E97CE0D414030CA01C98E217D439
:10866000A03045D57C98F6CD7D7B1C38BC44137A70
:108670003076EF76DF7617483C0AE0CC1BAA7339D8
:1086800088E60952D5883ED74DA6251CD91C302036
:10869000E81538004C73B0E22F302DE813B8957C04
:1086A000D91C7B30C30E203C0A2365202B4E203C76
:1086B000D026E806303404661708B0C606C61CD0BB
:1086C0000C1BE21722E866F13A0E30410660304B8F
:1086D00006F3302506FCE61C0A301E6A23666A375C
:1086E000FC0E66813A30CD6A2F3C3E3EA366E030F8
:1086F000610660306606A0301ADBB03C0E660401ED
:10870000AC0C0F1CE22F0E16913E70012053AED818
:108710000C27B0B13E088BC1B0B1BC492444B0A114
:108720001CF93E589DBC981C1D88FC1EBEBEDDA4D5
:108730004E70E5A4D8B0D83CBEC32550704670B08A
:1087400068301E7CA11C0441EEB83CD844D8FCA87B
:10875000D91C78D884D8F04926410CA83080A6E6E8
:108760004EF070B858CC1F0C1B66664C17168C1355
:108770006E3C588C233080464C2F8C23767676BC0A
:10878000588C2B76767676BC56EE3C56EEEE4E3016
:10879000107030FDF0AEF046F070B858E07CD80CA8
:1087A000DD2F580C2B30844D320CDF890C4C3304F8
:1087B000B170434BF8E61F26E865144C19387DBCB0
:1087C000651CC8F84666E8B858F6F62B9DBC410C07
:1087D00004B898A859248C47C1B0302EA84924C1A8
:1087E000024E28E8A89868E0FC5C0AB8AAA8E0B0A5
:1087F00030E83AF6E3E030107030FDF0E0000000C1
:108800005AEEEEFCC6E6E6C63C06BC5CEA5A505C94
:1088100030662B22E399C63AC60E3006C3A6E67A26
:108820005ABC1A30F6F63C58FC0E3C3A301C0A3C56
:108830005AB03AE07AF30438BC585C98FE9526FCAE
:1088400010D0900EEE7E93EE0C31237EDBEE7EA3F5
:10885000FE13081C78221BDCEB1465238C27787E22
:108860006881228CAF88DB780EDC901E6F080CC705
:108870004E6E56DC5050087B0C5F0C1F0CE30C1F37
:1088800008330423780E561C561750DB7E63EE7EA9
:108890004B9C78221BDCEB9443E030D066FB20E05D
:1088A000D400980278A26838BC983C28E01CAE58E6
:1088B0000813044E6E56DC90688DB8B8580C2BC95E
:1088C0008C89B68CB551884EE80CDDB641A48A4936
:1088D00024DD20792419B46A1C0A301D623F0A2B5A
:1088E000AE9C58636E1DA4DD8CC1026E601CCB383B
:1088F000BC58780ED91CE9501C622B62BEDCDBA28E
:108900000C471437D4A250DCDC8C5BBE1FDCEB8C34
:108910001BD013D0DC4C9BD47F1EBE2F5467DCDBF6
:108920008C1BD013D0DC9BBE131EBE5EDC0C135020
:10893000BEE0DCA0760C831C6247A29C622FA222C0
:10894000230AA2501CE0169CE0D2D268AED2D228F4
:108950004EA846F070E0D91C78D808D8F0AB781C47
:10896000221BDCEB6206569C622BC6DC14DBA05695
:1089700013860EDC50BEDE774277FABEE3A6426F66
:108980007E07A6FAD31EBBBE2766EBE31E0C13BE02
:10899000AE0C83A550E854670CAD2355BC410C1DAB
:1089A000024EE860E078E05CA01E0C1B9C131C22C9
:1089B0002B62BEDCDB0C83144742F21F0404D00B95
:1089C0007676130456DBD45F8C2F543F3E63BE5340
:1089D0008483B8580C2B410CFD8A4EE8203077E098
:1089E000689D2244781CEA31B60EB8AAAE3C68F8FD
:1089F000AAAE3CA838AAAE3CE8387C4AFC2878FEEF
:108A00003B09B8B8D84C578C47D8DE3EFE31B8F396
:108A10004484D8063020665746F07038566637D9F9
:108A20001CA6E853D91C230841B0CE6DB81902B872
:108A30003C5806F804A0965C1427D4B6E30EF62B37
:108A40008C63DC541F66E333D4144FA6E32E8A3ABA
:108A50005B0E0A061C2A4F0E7E8E9C0ABA60E0AEA0
:108A600056E346A38C431B66239A3A370C1F4E737A
:108A700084762B0C4B069CA206BF1BEE608DB8CEF5
:108A800008D528EEE9502E0EA0B8BCEE7EE6C6FE54
:108A90001BDC508C752A5CF65B752C552CD4DABE29
:108AA00026E37B661FD4EB46BE3F752C552CD414B1
:108AB00047BEE3D4141FA2E39CE04C437E9EBE4716
:108AC000DCD4E3DCA07E83A28C1BD013D0DCA26BB1
:108AD000552C4C752DF3BEB6AE60EE5D1E5C4C930E
:108AE000063003562FC6FB462746FBC68606A6372A
:108AF000D4BEE31ED3752CD4143FBEE3A2D414EB32
:108B0000D61B1C501CA63033A6E00D2AC6A6C6A64E
:108B1000F306F6C70BE0DC201FD4EBA0E0A28C1B11
:108B2000D013D0DCA2E0A01E7E7E43ED28D91CEE3F
:108B30002526DC10FEE0DCD0D07C70D91CB07C7027
:108B4000061C4AD36A2775B0AB3020DE7E2320494D
:108B500026E8D309CA008CB3F12E461AAEBCFA1A25
:108B60003A30E63A303CC61C3CA2BC02F6F6DE6B5C
:108B7000F6277CD90E7CAE0819BCF90EF6CF75CA63
:108B8000AE5851000E389C0A983CBEAE2838FC26E0
:108B900084E6C67C287E7E677E01CBCDC63000EEA3
:108BA000CC4371CC66250E22C8EE66A30B000000F4
:108BB00000000000E55CBB6100A3E55C8838FC6652
:108BC000E6876B1CC4E666664B095010841CEE01F8
:108BD0003041A478901C8C476A550E4DA43DA49D4D
:108BE000A48C1F7CAAB18CC1B0041D1425FEA55015
:108BF000EED44B4670B87C588CED02B070EEF0E0CD
:108C00004EE8286AB3B83C58A020BC30C1FC1CE038
:108C100000105B504B903BF3D023BD8E103C064CB4
:108C200023308006708C83AE1CE2EEEEEEFC5C50CE
:108C3000303CE6E60E9CF83C5842A65844D91C301D
:108C40002006861CB86AF3AA6A37C6E8A8B8D3F823
:108C50007E60BEB03AE006B8588C233055737C581D
:108C60004C3305BCEEE91BB8580CDFB05A3C06305B
:108C7000667E679CD0FE431CD03EFE53FE470658DE
:108C80000ECD90EE87B00EB85830505E7C067C302A
:108C900076B1B5BCEEB85CCA46A80C2BE21B1C2210
:108CA0009C5858CEBC30147C301C50BC5870305985
:108CB000E2B858E0D8A686251CC1B030E02D1404D7
:108CC0001D1030E09C58BC0E66483D3A44251C1DE2
:108CD0003C984D14987A30F6453AF6F6167A3016E6
:108CE0003C5804D89CA298A2580C9321382B4C5184
:108CF000370C33BD386520A30CB5374CC9370CB7DA
:108D00008CCD378C8F5E7B3091AEFC9C425D1CAE6F
:108D10004D32C1B0711C9DBC110C1D028C1B0CB3DB
:108D20001538838C6B4CF53B0CF53B4CC9376520F3
:108D3000838C653BD32D38DB4C41370C3381346554
:108D400020A3203C0A30836A7F3031E82D383B0C69
:108D500081356520C3B8FB0C3B8C678C1B4924060E
:108D6000A6A6B8A6A803B8F8E806A6F13B4924B819
:108D70003C0E8CA730CD8C2FD91CD532AAAEBCA806
:108D80009858889858653A4C5330AEAAAEBCA80C97
:108D9000571B301E0C0B668CF39C98D844D8581C7B
:108DA0003001AAAEBCA8C1B030D02D14A83060E804
:108DB000D53649249C98D848D858D91CBD1C090ED2
:108DC000042021386B4C778C5F0C1BBD3865209BD1
:108DD0003030E81B30305E172EE83CBEFCE8953A98
:108DE000BEFCD056E82138430C1BBD386520BBB80B
:108DF000E04936BD1C1314201538BB3020A8A8A8A4
:108E00006D7CDC100E304C66CF21B0DDAC49249C6B
:108E10009858B81CD04C1B1CD0AE7CA2813A65205F
:108E20009B3057BE5E2B2666DF03305466E3834ECD
:108E3000BEFC1CD0E81538630C276520CB4EBEFC69
:108E4000D0E81BB8E0301F43301F23301FE8E8E8AC
:108E5000DDAC4924F81C98E8B83C58880898FC6DAB
:108E60001C61001106DCD01C0EB87E584CE706F8D9
:108E7000425646BE47A6E606E6E646A39C98584CF0
:108E80002330804686DDAC4924B80E8CA76686E682
:108E900083DDAC4924B80E30C8E0C8CC3B66E32083
:108EA0001938436D00C1B020492495BC110C9C9821
:108EB000D84C3B4C1FAEBCD1A6D84E5CD070AEBCDB
:108EC000FE6D076645023040E6C8CC6D0266DB04E5
:108ED000B1703C30E866FB59364924A5BCB8D88847
:108EE000D8A84E68D91C1538734CD13E957CB35D1B
:108EF0001C8498A84936492478EEAB7C4A68251C26
:108F0000D91CB81B0CCB6520E36D7C06251CB6BBB9
:108F10001C307F6A93303A6A73302E6A53302C6A61
:108F20003378EA1FAA0A3C68EED91C21B0B30000CE
:108F30000000000049248C931C78EE4B255068B843
:108F40005884986D1CB83C06300F6A291A86D91CC3
:108F5000DDAC492478E0DCA01CF2251866301E1C2C
:108F60006ACF78581598EE8FB858F83C9C580C5F2B
:108F7000B80E95BC110C810A4C37587C7048840C93
:108F80002B88B0A11C44B8D80C23584898589C583A
:108F90004C4B1D3C4924980E1DBCB80E86813A8C62
:108FA000537C560EB858AE444D32587CA11CB8586C
:108FB0001C98BC580C5B30E61BD03B3A30E617E0FF
:108FC0009010589C583532F8E6C1B04CA066664CFB
:108FD00013061EA1143020E8E060B0303360B030DA
:108FE0003A70EEEEDADADAEEEE7CE041A4584DA407
:108FF000EDA4D8E05CF84A0EBEBE175031020E8CCC
:109000002248E30130028C043EAEC242880480BE96
:10901000202C51C0202ECC0DA241A9AA84F902C453
:1090200050020D3384537FBC3F00000004DC78778E
:1090300077A50400DC4E0DC0AD804070097E441061
:10904000226323144F8CCCC30DC912942379D33FD0
:109050000030004100E45C480640200180840B3071
:109060003417E33B03614413D323C1903331FAF443
:10907000E4D2CA44F24DD4908823743880DFCFB351
:10908000F3BC6C759792E288CFD3CE4060C1562175
:109090001E168C74E8237655D4B87088323931D5D1
:1090A000D193F0E04D472E1FB82F2C89617420C258
:1090B00040844410A0363513834E847F64D84E55C7
:1090C000E88080D274124C1BE360A307800F28CC89
:1090D0001B31841C91DC3E01FC279EC001316D8256
:1090E0000FEEFF13DFCFFBFC27D90F9E1BC43013FD
:1090F00072813CF7F73CF743182F2EE388A4033C1A
:10910000000010D544483012D070C5713003B0173C
:10911000470C3C12C470CC030D8BCF8002470C4D22
:10912000F348CCC44C7888871F871EC715335F84EB
:109130008F2341C0084013CF4688CC00253840CD4E
:109140007512080A0D21334073C4044383C700F825
:10915000B1C44CFC72FC85BFDB87C4040C232031F6
:1091600023715CC00E193400C6848914C3703CD1CD
:10917000F3CF90E150CE6192DFF120A955A34A15BB
:10918000A82A166262403C8777F8480491C33833B6
:10919000C3400431F3B0F7C9C4E4C88DBBCB34700D
:1091A00038E013130741C43C7324232378D1C43D12
:1091B000215E141F13CAC53884C4AC737C7CC8B547
:1091C0001012024080D844C84417612520B33D20C6
:1091D000C623FCECD36EC8C1EC0B5420F944001537
:1091E0004F1534551823FBF73284FC4C018B8773E1
:1091F000E1F81727FF0113C760D19278AF17C603B4
:1092000094D754508F8FF450E4E5A41F659A3D8A9B
:109210006BDFCB3C02CA23A3CA8DC94D8842132001
:10922000668633F3ACFC18FE43A28D0B11A2CA83F1
:109230004813144140001733CC0C0CB26D33847DBD
:1092400003C74F3CC48314F3303D14CA20CED191E0
:1092500010CC3F3CC03EFD2EF2C6F1EE98127337A3
:10926000D673F4480C30CDC980CB3483D88F2072AC
:10927000CA2033DEF32003C48A6D1458608219A813
:10928000C5878C047931ACCCF07340CC1EC97667AD
:10929000F2355B43440B1D38CF7ED0C162733F0A69
:1092A00001630E80B8B3007C8E3C05B0F4D203108D
:1092B000BB0030CD0058885CC574351A37C3D2ED79
:1092C000E2D03010A2633C03F10C4D0CE1E8CF304A
:1092D000FD1107723C7012948ECB9025A18C23094E
:1092E0001C480F8A036AC214130FE30300A3388BD0
:1092F0002AA04C03C431CF0C0CC02C0200DE0AE2C1
:1093000038FC494000C0001D841057195F3DC44E11
:10931000C47FC3FF5DD64BD524CE0358C8CA19629B
:1093200081D117FB420808B2338443F5FC414CCC91
:10933000125328C634B952B9CE0350C400C846F2FD
:10934000CE7FE00932713233F100402233870C8C3A
:109350002CC5C40123EF0B0725F653843401339049
:10936000CC4C04E415AFCECC013931C710733303B4
:10937000188101C831313E1E080700F2C38071FC1C
:1093800063C5C8C4AC85332246E31F3B380720833E
:10939000DC0741FC13C33F6F88F8DDCC5050D57318
:1093A000444C18C04C58F8F883CC7132C3C10C0738
:1093B0000692BD78413BC4BD8F1304B3F810FA1870
:1093C000F3274ED1C7C7C7C7EBA48C080081ABE316
:1093D0007B48B13013223AC467233F437632168864
:1093E000C0F0303F32516308408F12F357B0804BCA
:1093F000F0CC0CD3C0C4DBD8567F5D34F2430503F8
:1094000041460000020103044247000027242120B6
:109410004348000028252200444900002926230053
:109420004540000F800000981E19B0456C63AB13D7
:109430000D08B0C964F0B8C9640EB01D6088C96475
:10944000CBAD130D08B0BEF053ABB063840F0DB0BD
:1094500071643BADB0BE001D606902AAB03560D337
:10946000A5A6A6B035603102B21E18B00EBBAFB0D3
:1094700061603B930201B05EE0930F030151848869
:1094800008080176008435928C031201595A860827
:109490001301215E8E0913015184338E1301A99E9D
:1094A0008F141301715E8E0114015184AB9705096D
:1094B0001601910E008883900505023007455A94E5
:1094C000130200418A940103012E8603355A810C50
:1094D000034E68A8E828E08F141398F0E0840C038A
:1094E000410C511E900C03318A87120C0308CD5E8B
:1094F000CE0C03C15294130C034E2868A82B980C71
:10950000034EE8090299100F039586922D04B005C9
:1095100066870504715E84011207995E84011289D1
:109520005E8C0504A18A0000BD8A8513047D5684E3
:109530000E05870E0548015A9E1205140E05B550FA
:10954000B8E81102981E05B0296A96040175BCE0BE
:1095500094030106B0B162BF0306AEAEAE2BB12DCF
:10956000181E0548B0296A833F030635586B9809D1
:109570000688015A940E098823831206B0ED66BF4F
:109580001306155A833F13063558C30065A68F147A
:10959000079208B0C966930D0888CB8713098481A8
:1095A000568C020C8E0CB0156E870F0C88CB96056E
:1095B000041341743B8E01050DF9709502902D1234
:1095C00051842574BB86060FE03009999C1508610B
:1095D000004106982F31B02D62922D105184080859
:1095E000D578CB8B0301100182880325BEBEBEB0A7
:1095F0001D606666B869603102851310CC2308EDE2
:1096000004B10E94100D0F1210810E842D12B03182
:1096100066900F1413A50E0000751E982B310E0CCA
:10962000B0CD6E981413010C38EE238C03128CB558
:10963000514E70EEE8B902930803B0FA1BBEE8B3CE
:109640008910A06964EE3A460BBE3C1898F01B8E58
:109650000412F552840E12BD2A8E14120D9E9E1213
:109660009552890313015A8613295AAB4E2172ADC4
:109670004E88DB8705124E655A930F0351846B8E1B
:1096800001145184438E091351848808E17A851AA4
:109690000913555E94121113B0F9629413130081EB
:1096A0008A8E0F4552AA14134950356043AB1413E8
:1096B00049501D60B92EAD141398A0BE589BAF142D
:1096C00013495061607B981E3031E16E850E0F1496
:1096D000795A97050916BD0EBF304D18455ABF1966
:1096E0004D18A55ABF303C18E956BF303D3C1825EF
:1096F0005ABF193D3C18055A993E3C18F8AEB8E8D7
:10970000AEA8B902BF193C18BD56BF303D18195A52
:10971000BF193D18515ABF303E18C556BF193E18E3
:10972000E156001D92910518830504482394030F08
:10973000B0E57E8E070913D13E8E0F0188ED0471CE
:109740001E86060F0184BB00009D7CAB0000201C20
:10975000E2E2E283B87CD84C1F481344D83C98A876
:109760004451064DBCE27F410C8C3B8498A8448553
:1097700006880CCB53410C04840C1F08830498A862
:1097800009B8634EE6BCAEB90C004A545C6FD6CA49
:10979000767D4D453C8C92989EA4AAB2BBC2C8CCA3
:1097A0003AD1E0E7EDF3F901097C0E2B14242D32B8
:1097B000353E4763545A6B717C82881A91993245C1
:1097C00093779E28A4A620ACB94F30C8A3DCE761EC
:1097D000EC4209FC600EC01F2E52575CB265696DE9
:1097E0007177883792989EB0B9A8C1DA1582D0D621
:1097F0000EDCE8EF1A14E208F6204CFC286B2A0075
:10980000C88C2409E71892C29EA3E7274DE0489E22
:10981000ECB83C5808987CA8E04E70F8E085B5E0BC
:10982000FFA0B0BE001D6070E0FA174EA05CF6A06D
:109830006636761B26E0F61B4E2B4A6A56D4D4E0D9
:109840004A545C6F0820F66D7132454F61ECDCC004
:10985000A66B982A3A47ACCA63887C82987DAA2B6B
:10986000D67654DC1A20E80E777C0E0E999357308A
:10987000F3FC42F96052280114E237EFB9B2B2E0CA
:10988000141F1A3E155CBBD192FCED453CC8094D36
:109890002EDAB0B9A8C19E2DD677A48C716535D0CB
:1098A000E7FDBCEEC10295BE69CC886B825A23F0FD
:1098B0009D585C0EAEF0AE6E70D494CBE0A55043D4
:1098C00032EC4E70783C0602E01CEA603CEB4CA4A3
:1098D00091EE6E98AE6150AEA0FEA03E337EE000E9
:1098E0002800D58818B550B902B550B5504E70381B
:1098F000AE7828B868F8A8AEE8E0A04E6E60EEE05A
:1099000047710E834140424348700E0078464567D8
:109910006075E00017141110534C0F00A8869C725C
:109920005259911C1815121A515CCF96A94E9D766A
:10993000565A901B19161305575DD085AC4F9E984B
:10994000505B08000C0C0C00555E07770C0C0C00EB
:1099500041460E4E5155593A617E0E5E2D2B2A2FEF
:1099600042474B0052565A2062257F00373431302F
:1099700043484C4F53573D2C631D9A0D3835322EBA
:1099800044494D5054583F05643C9B243936337E3E
:10999000454A08000C0C0C00653E07870C0C0C882F
:1099A000EE61501BDA26F6EF1D64989417D44AFA3C
:1099B000EE58AE0EF09C4A5CEA271C505C0E0A4A38
:1099C000EEEEEE5C262666421FFA06E247FC4626CD
:1099D000E21FFC468C13BE70981D60580E38A60618
:1099E000DA661FFAE7461AB160F08898AE8C5385A4
:1099F00050A0B0EED33E1BBB85508C97A0B03E7BF1
:109A0000CB8550EEAB630EB07BF8615070B0EE5377
:109A1000630EB0CBB8AEF86EB7CC6F4E70B8D84C02
:109A20003FD88C27AD7062C102B8AEF86E6760CCCB
:109A30004341A4E5A8BD8C834E70B8D84CA7D88C00
:109A40003FAD70641BCEB0EE8F2BEE702BCEAE0010
:109A5000B0A8AE58711C98AEE0B0A558B0AE4E702C
:109A600078BC46063C68E078BCAE300560061972EA
:109A7000EE38A02E6EFE433E2F385E3E537EF61B20
:109A800056765CE2174E60EE0EF0386E334C810B6A
:109A9000C90ACEF0AEE0CE7EFEBBA118CC60B858AD
:109AA0004C608CA00841B0B83C58084898FCA8E02D
:109AB00046705CA0D4D4542FCE58E09CD251B5A3AC
:109AC000983C98FC58B83CD88C132E0C1B2E2EBCFE
:109AD000F375583005755830087558300758B8BCBC
:109AE000D80CA0C4D8584E30FFD8BC0E7CA0BE60A5
:109AF000F1585B657387A1C90B3F8F15B01A30A66B
:109B00007E677E777E8F1ED8BEFBA6DBE0D8A6F3ED
:109B1000E0D800A6EBE0D80000A6E3E0A95C98BC82
:109B20006D1EA95C88CBA95C08ABB83C588404E0E6
:109B3000044E70783C5A70AE38EEAE0EF0386E605F
:109B4000EE0C134EF06EAE7BD55C542B1C52F0E045
:109B50004EF0D460AE7038DCDCDCDC93D55C544B6A
:109B60003CDC5010F070F03BD4C7AE7038DCAADC9F
:109B7000DC7C94E36B300870AEE0DCA05C38521CF7
:109B8000AEEE6FAE0E7038D494BB5CF260DCE09C3D
:109B9000D4D4F2EBE048A670851458C15C4E708EA8
:109BA000783CC6B0C67F08CEAE584E3CE6BCEE78D8
:109BB0005A7AAEC39806374C098348E07806BCEE63
:109BC0005A3AAE5878E62BBC1AEEF0EEAE0C3306DD
:109BD00033AE2E6366E3AE70FABC1A3CE638EE3C58
:109BE00070662FEEF098EE41A4CC17266E78063CF6
:109BF000063C063C686E4435BEB8584898A8E0005C
:109C00004E1B4EBE5C501B2E7AD898463E5ED81C2A
:109C1000D4763654E3EEEE6BD86EEE4B2687D86ED4
:109C200026DFAED80E23D8AE2BD8AED86E9E5E5BA4
:109C30008E1E263BD8FCD86EA66E264B66CEBE1E68
:109C4000D4D4C34EAE98EE2E76767600CB2E7AD84C
:109C500098463E5ED8065E139E0ED8DCDC8E132E30
:109C600062F354CB98AED898FE1B66CEAE5C4ABF6A
:109C7000EEAE5C0EE66B3A5BC62622DE6EFA604EF6
:109C80001EE0C6C36E63424F66EAE32EFAAE4ED8BC
:109C90004E5C50EEAED8AE332E7AD898463EFA23BC
:109CA000D8465E139ED85EAE6E2E2BD8EE66D85C7C
:109CB0004E13228EF32EEED4D4D3AE98C1622EFA78
:109CC000AE5E1BB5A23ECE6EEEEE0EEE5A0EEEE688
:109CD00013BA4E9C4217AE8E4E6EDC50CE5322CE3F
:109CE000F34EEE94C963D4CABBA63BC3FEB7F6A736
:109CF0000E8E1CEE8A5C4A9766061B36E04E22CE1C
:109D00003EEEC21BAA260EC223EE2EFBDE338A6E67
:109D1000262EFB6A626B7E5BEE865A5E2A4EBAE0A6
:109D20004E709ECE68B8A606A8E07E78EE68B8A60B
:109D30007EBB4E7078FED8B8DED8E01D648CB5626C
:109D400098941FD44AC9622EFAAEDCCED86ECEF6F5
:109D50006026E63B66EE1ED44ECF66E076FA3B36D2
:109D60007E13484623B6AE932EF0BEF01E06FA8E42
:109D7000FB2EEE66DB8EB0B5604CA0FAA00EF81D8F
:109D8000620E6964EEB03D60556469620E556435DB
:109D900060696475624E5C2650E04ED88564EECEF4
:109DA000E05C4ED01050D050105090D0D050D050D9
:109DB0005CE0FAA00E8E2626065C4647D4941BCEA5
:109DC000E066D34EDA8C93DCD4239D642BDC9D6457
:109DD000D4D49D640ECE95620E9564DCD417DC95C8
:109DE00064EE4EEE93CA0A0ACAEAEA4A8C330E06B9
:109DF0000E46E04ACAEAEFE0BE6E8ED8988E4E2735
:109E0000980EE026CB5C626EA5622EFAAE045E135D
:109E1000081E1A6ECEE673CE5E7FDCD494856B2668
:109E2000DBF568A3B9685C336E66AE333A8EF32E09
:109E3000EE66539CE22B62E24F225C23AEFAAEE266
:109E40006B4E5C6A0E1C500C13A66E0E4C1B096008
:109E50008C1BBE1E1162228EF32E543FEE66D4EE92
:109E60000BEE4C2B2968AE6EDC909CFA9BDCE23347
:109E7000628ED89883268E7E9BCECECE626E0E0CDE
:109E8000396153AE7EF32E7E982BD8988EEEEEEE8F
:109E90000E6ECEEE2798AEE066CB8ED82695626E1B
:109EA0005A5E0E0C1BE1644C1F0160416AEE5C902F
:109EB000D010905010501050905050100B4E54979E
:109EC0007A103AD4E7543F148F94CF54FF9CD05C5F
:109ED0006B9050D05010D050101050905CEEE000BD
:109EE000D0501050D050101010D0D09C8B1CD0D01F
:109EF000101050D0509010DC2B5CD0D0D01010D06F
:109F0000505CDB5CD0D0D0D0501C9B1CD0D0D09CFF
:109F10006B2EFAAE8964B861500EF85EBB06BAF6D5
:109F2000330D62E6EB66EE5ADFE64FBE1EFEFE1E06
:109F3000FE1388B85E2EFAAE08DA77D164FA1B9861
:109F4000FE072E11622EFAAE3E5EBFDAABA606E623
:109F500083461BA6080E5E5A5C8A62228ED8988BB6
:109F60005CCE62AE4E4D6E422766EEE3D8A5608BA6
:109F70000160B32EFA0EAE0E26E6B35E57AEE56470
:109F80005C4EA60E6E3B08CB54F7D43E26DB738E98
:109F90007EF3982EBE333E6EEED4940BAE8EEAEA7C
:109FA000EAAE9CD086C6E35C8EEEF568A56CFAE35B
:109FB000D4BB2E9C822E8EB5680C376E8E6E2E6EA4
:109FC0001CA56CFA3B8EDBEEDB8E235EEF665E0C2F
:109FD0001BBE00B5600CCBD164496098FE356AA603
:109FE000EEDB8E29686E5C1B2E62F34226DCE08C71
:109FF000A04ED8B968EE75620EB968B03D60EB004E
:10A00000000000B0094648167616810B70C15A014F
:10A010000C10080120040114010401140120051290
:10A02000120F120D050D0F1219200C0F13140E0F25
:10A030000E0518091314050E140E150C0C10120938
:10A04000160114050F1514200F062012010E070526
:10A050001001030B090E0714121920010701090E44
:10A060001905130E0F12010D120F0D08B060303AD2
:10A0700070BC5C50100EC1B0AE307A0656A856D3F4
:10A0800049240CA08DBCF10E2170B8F0B00E4C2309
:10A09000BD701BB57069708D70B00E356069704C05
:10A0A00023B9701BB17081704670F84C1F48EB0EDD
:10A0B000B835606970AD7081700E626970A9708D7D
:10A0C00070F04E70F8280D729D585CEE615060EE95
:10A0D0006670EE38D494B34E70138CA0BEBEBEE052
:10A0E00025601B1D60A550F05CE0D4D4D4D4D460AE
:10A0F0004E7078BC26DCD4EB667038A05CE0217032
:10A10000B5701D74F0BD700EA970EE4E70EE6162F8
:10A11000842170B1700EA970356081648C27B57090
:10A120001BBD700E3560BEBEC9643160A970696028
:10A130008164A9702EFA0E0960C9644D60FE89031E
:10A1400005608C60F088B9706BB0FA33FE238888A4
:10A150005EF00E35608964B80E3560D164316005FB
:10A1600060F00EB8AE6160FADF0ECB8C1F88E08421
:10A17000E0AE88FE13485EF0B0FAA00EEBAD74E3DB
:10A180002E0E7AFE4B480C338C238488445CA60642
:10A19000E6B177468FCECE235C62EE570C0785641E
:10A1A0000EA6AE3D7A0C0D633960AD746ECE5C5A6E
:10A1B0005E26E6433ED454D3EE3D7AD84E3ECE6B77
:10A1C000AED8221ED8AEAEBEEB1E2EAE8ECE93D82B
:10A1D0003ED86EEED454B3EEBD606ED8469CEEE130
:10A1E00078EE132E62F38E42FA1BDC9B0CE389643B
:10A1F0000160A9640960D16449601E0560B05ED841
:10A2000098464D60A606E6A176B176DC6654EB5E14
:10A21000B5608C3BBEBE696431608C2B6964316073
:10A220004C87696466660075608C3F4E5C66503D85
:10A23000604C13BE0C60F0E04E6E5E546F94EFD431
:10A2400027544F14679CD09CE0DC90901090509065
:10A2500010505050905CE09094F3631C5D789C50DB
:10A260005C109CE05C5D789C50DCE05C5D785CE0C0
:10A270001C5D781CE00808AE0E2EBAFE43880C1B4D
:10A280008C13485EEE4C457B8C2BAE0ECECE4E5CD6
:10A290001050EE66F62F661B268EEED898EEEEEE88
:10A2A000CEEEF69F8EFB2EEE66DB4EEE98EE4C1B4E
:10A2B0008ECEEE8E5B2EEE98EE4C0BE6F7EEEB8C30
:10A2C00047884C1F48734463840CC38C1B842B88C1
:10A2D0001B8564436E8E00AD743B26F6278EB32E2D
:10A2E0006600B5604C5F98EE66006960696449601D
:10A2F000D8AE0E263B6EEE3BD454B726E36E4EEE40
:10A30000E178EE133E8EF32ED4CEEE549BD88E8E93
:10A310004E5C50D89C90905B8A8ABEEB1ED8AE4EA5
:10A320002ED88E1E62ABAEFAAEFA0B7E661E8E9BE8
:10A33000980C4F8C3B396023B0D898464D60F0D1D3
:10A340006449608C13F08C13BEF00B5ED8AE98AEEF
:10A350000C1F8C1F866EDAC3D8A5600C7B8964D174
:10A36000644960016005600C8739604CA0BEE04E16
:10A370005C6A560E8E0CA02300ED64FA0D63B04C9F
:10A380009F0E1E4E5C66D01D604E5010D0D0D01077
:10A39000501090109C506960F60D62E01CA09C6EFD
:10A3A000138E26F34EAEEEEEEEEEFCA0A2E0CED47F
:10A3B00054AB139C42E60D63B0221FDAEBAEA24E03
:10A3C0002E5C105CEE22270D622EA2F3A637EEEE75
:10A3D000EEFA9BAEB04A1C5090B562B0064E3055B6
:10A3E0007C067C30E04924B83CD88C1F881384D884
:10A3F0007CA8E0302D9C58A051B698DCD0CB06C08C
:10A400001000000000800000000000048080042094
:10A410000020030001080CC41431000D320003CCED
:10A420002B28900210003314900130021028400CA9
:10A430004070A2015039980332900004800000005F
:10A44000C0000580000000005002420AC035003004
:10A45000300000DC000C8A04000068CC39000000E9
:10A460001AA031C1030230B9C040000C00008C00BA
:10A470001303C680088000B32100000850C80032D2
:10A480000800088000080800040001D9200C80C8DA
:10A49000A024933920000000C38D06083068000313
:10A4A0003000F30125000840009013900343A64DAF
:10A4B0008E0C307003190000000003000000000043
:10A4C0003000030000003000C3D0000004C0004290
:10A4D00000380C20153700F7CA89886FC8CB02F303
:10A4E00033840090D00300000240D95555555505DE
:10A4F00095657116695AAAA9EAAA2AAAABEFAE0312
:10A5000054285A3FEFFCE3C38B000BEE2A1E80FC5D
:10A5100000AF02542196A9C091EB95E5286ABB05CE
:10A52000550AC467A25A0A99872352F51188FE4F2B
:10A530008D13EF6E4D0CBA3833CCCC2000002CDAE2
:10A54000555555551500155515005555154055557A
:10A550001515551510001000000000000000100037
:10A5600000401040101560D50CEBD10C448A12123B
:10A57000FFDA8C88221341418B63680C8859206272
:10A58000800C302003C0083E2CC100AFC4C0F8BC12
:10A5900007B3CE204F11138087FC110AA08A8028B0
:10A5A000B820C938808C02FEECC17FFB38FF40C266
:10A5B000BBCFE3684E4C4CBCFF4E5CA80300953902
:10A5C0002292DDDB4B2FF470010F3FFFE12040F2C0
:10A5D00004C631E2C8C8FF310AC88CCCDF8720012D
:10A5E00009C9BFF3EF0B1220131124C40889E01B23
:10A5F000484322C4008F24003E46402C26233C3F83
:10A60000800314D0E76361134F1344343619314D7E
:10A610003B442A400129924FFE51D23C70212838F8
:10A62000CCFC3E400C04506029064CDB60F74E0128
:10A630000C002554D8F36063F7F187AAC1FF8DE3BE
:10A64000224BDC7136EE03C5084A8E288C927410BA
:10A65000CD0420812BCEEF8983040040B74FB00793
:10A660002010224988B04ED24F861258EFA11D0FFC
:10A670003BC0323C3F11CCF21C6F974072FB423D15
:10A68000B51F02300004E3844B12F4760BA2788CE1
:10A69000B30948006262173B0202862D52B8FF11CF
:10A6A000E25E5D50B2C46D0A100C403040866831E5
:10A6B0002658594D241452330029410718240720E5
:10A6C0002900A48002C0C4808CFB0B9522000B786B
:10A6D0008E00AC928400A75423CFF8092044F630B2
:10A6E00043C0B5EE5E298FF0735A2323CEB4001118
:10A6F0008C3CCC0B480C4442BC90393E9320082142
:10A7000000203D460000040040000010000004044A
:10A710000001000001400000410441B915376CFC04
:10A72000D1170304C3CC500C0C330860C4CCD0CC7C
:10A73000800411230A3FC6C80080FFBF78EE8A3F1D
:10A74000034C0322CC3401304C21002330108028EC
:10A75000C33062E2500005C01088C0FCA30438C5B5
:10A760008424B34DCDE02B2F043C123028DE40383A
:10A77000647D1374C6374208403EF6030000C140B2
:10A780002194C83E312220022085006B84CEC8046B
:10A79000599D5316097D7F71D8C532E1463B8038FB
:10A7A000133040C785224E5523DD0E054F4490CC13
:10A7B0001CDDBFB88B44A074125022129130970355
:10A7C00000767FF74C17DF8445CE98F2D949140202
:10A7D000C42012513222C900048C4A3B4BFC800336
:10A7E000050B0051482B0E31EC502DF0DF38C8130B
:10A7F000ECCCD8513D300451FBC73EF37F0CD00C5C
:10A80000441348AD7056390C51844E584488A18089
:10A8100095BCF0B3D5888A3E23E6D7ABAA0A704D23
:10A82000A47E7C81BC8D8CB0AA39887309504E5BA4
:10A830000CDF98EA2DBE0AFC4DA459A4AA0A582997
:10A84000A48A41A4CC57980647662F022762130AB0
:10A85000AEFCCA7004B00A8AB0CA70E5A47CE21FDC
:10A86000F6B362BF62ABF62BF61BF67F0C5B980A61
:10A87000468D8C59A498AA58081304B00A7C060F78
:10A88000662F02EF62DBF5A8B0AA70E5A4EA987023
:10A890001CA18C98622362626E6258B06A775582FE
:10A8A00046FC708A980A29A4BD8C6ADB20B07038F7
:10A8B0009C5898700E388E8E1CB63FB6DCDCDB02DE
:10A8C0007B4AF01C6A101C02BBA666700A4EF09808
:10A8D0007CAA698C70389C98F0467078A6682E66C1
:10A8E0000DBA6670EEF0EEC34670781C10701C0A4C
:10A8F00038E039883E37FEFEFEB183980A7CAA69AB
:10A900008CFC4DA4AA58B00A4DA4AA0A70E5A47CF8
:10A9100022DDAFE078E64E30C058708370383E9349
:10A920001CEA277CEA2371841B5584C606B0666F37
:10A93000E07EEEA0FEDC58B098701CB0FC6A6F7C24
:10A94000705584DE7985AB00000000000000000037
:10A950000000000000B0702E70380E3B55849870D7
:10A960002E58AEF0E07858EE8B1598EE810A4CEF39
:10A970000C27D588671CB1182BCCC3A918AEBC30E6
:10A9800076767627D588437AFA851406DA1A300661
:10A99000098366E64670787066BCFA38D884D8F0C9
:10A9A000BA3A301C62027CA23C0E3A300A7E27EE94
:10A9B000EECBEE3C7066EEAEF0EEBC663FEEAEDC8B
:10A9C000901C3B3C2606467078A6681C02C4BD8CD1
:10A9D00009B81D02B8463C584484B0E06259A66EDE
:10A9E000E0C461A4CAD844D885A43C0AED1ACCA01E
:10A9F000D5886A66A08CE746E000000000000000F1
:10AA0000386B3823380338E338C338A338FCE00008
:10AA100038E038933873385338333893387CE03C17
:10AA2000E07CE07CE03CE086EA667038CAE086E6DE
:10AA3000667038C64B42EAEAEA22E2E61FC61BC647
:10AA4000360A1B261B62620A707C3020FCE0AAC317
:10AA50007CD80CE92F758879A085140CCD071902D4
:10AA60007CD80CD12F758841A4F80C83E6DDA9654C
:10AA7000504C1346261366E8DD8CFBE61F26E8657E
:10AA8000144C1938655026E8E55C75067858EE8751
:10AA9000CC1F41A4A1A48584CDA8884E66480B157F
:10AAA000981CEE1B0C7B810AAE668F840C731B888E
:10AAB0004E704C47CCC98F41A4F8CD84E844B044D3
:10AAC00070198C4C27B066CB95A47CAAFC61A47C41
:10AAD0000A4CA9A76550E62398ADA01D0245BC11FC
:10AAE0000C711C2DA84CAFE0390C0860BC580CA0B0
:10AAF0000498DDD83BA188B030C570CC1F4C1B79C1
:10AB0000A055C42DA87BAA0A584888F5A898AA5829
:10AB1000334E59A48D8C986ACFE0AA8A700A7C3093
:10AB200083FCE0AE1C8A700E7C3080B31DA44BCC3D
:10AB30003F4E70F84666E8467038AA0ACC57E213D2
:10AB400022E21322E2132228E04CC98259A49DA4D8
:10AB5000AA0A29A4AA5839883E5F488C337EFEFE93
:10AB6000FEE3B0E098EE4DA4E5A41C6A4F06E64E65
:10AB70007005BC95BCCE581C0A59A43988FCEE98C7
:10AB80007C1D88EE7CEE6A461746363606277676BA
:10AB900013266A698C980A84F5AA584A174A4A23E8
:10ABA000666262E6E6E6E61322CA101C0A986D8C1D
:10ABB00098E0B9844C1187AE41A444F8E633E5A887
:10ABC0004C3748655026E8DD8E30DADADAEEEEE012
:10ABD000B02BB03A707A258CF3B02BB03A707A254E
:10ABE0008CA3B02BB03A707A258C53B02BB03A704E
:10ABF0007A258C3A3A3A7CEEEEE0B0703C467CE046
:10AC000066BC1C3A3076F6E7E23FEAC3666AAF03F9
:10AC1000222222227B9C229F224F3A3A301C22275A
:10AC20004E4C7F488EA9186EBCCB3A3066AF7A7A0C
:10AC30003C1CE044448641A4CC3FC6BC584C1B4D50
:10AC4000A4E5A47C82E2DFE237E2AFE223DDAC934D
:10AC5000F68384763CAEBC9C98161C66673C0E2935
:10AC6000A48C29A54E70AAE03C0EBB59A4A3E2E730
:10AC700036C736C739883EA74C2FED1848234C3BC2
:10AC800041A44DA4DD8C4E70E0E5A4884B7D9C98DA
:10AC9000CCBF4CAF4C9BCB5C42EE2B0E4E701C4A93
:10ACA00033AA7C8E8ED33C58681598EE9B0C1FC43B
:10ACB000934C7B8CA758B8E683B85898BC30E64BC9
:10ACC000E0C81C0A1DA4A37D9C8411007EFE4B8D50
:10ACD00008063064069B8D901C0AB8E6B38A636A46
:10ACE0008686A644D190EE60810A4670CC2FB85873
:10ACF0004C83B80A38AAFC0EF8FCAAE8AE0930ABBF
:10AD0000EA0130091E04CC7F4C6F06984C8D900CE4
:10AD1000870ABD8CC102CC330A0238BC3A30A6B6D1
:10AD20003A30FCE64738AACA0C4B8A3B384AD3086B
:10AD3000EE41A43DA43DA4AA0A559CEE530C3BEA67
:10AD400049A4E5A4D6E63342EAEAEA22E2E697C657
:10AD5000EAAD3CD86A8C8346425366985846704B9D
:10AD6000C63673A2A2B3AA62620DA48308AD3C8466
:10AD7000D8064891900AD8662702331B061B04AAFE
:10AD8000464223666262E6E6E6E61322CAE641A48C
:10AD9000EDA47CC63CFAFE8D8C59A4CE7C8D8CE54E
:10ADA000A4D8840C1388D88D8C980A7596190856E7
:10ADB000A08A16CCC3468B02A6588C3B84980638D2
:10ADC0004A4B0638AACA237D900A499646BBEAEA4E
:10ADD000868638E2AAE2270DA48B462222421B6611
:10ADE00053A2A23B047D905841A470986627023379
:10ADF0001B061B08AA0DA45697E6567FE68AB0AA42
:10AE00000C1322EAEAEAE63C8D8C9825961C903CCD
:10AE10001E98EE6A21B0001CF61B101CEEEA3CEAFC
:10AE200023BE2F7B3CEAF358845C4E7050FADA9CC8
:10AE300030583A30E6575CDA22A3E5E200D0881CAD
:10AE40003A308C97E63A30C61FE663E60EBC427C89
:10AE5000A67CCA70BCA6F6F6F6A33A3A0E303C1EA3
:10AE600078AE7E3A3A306A677E8E8EFE2F4A2F4445
:10AE7000E34A97BC631C06461F4EE030DF0647C618
:10AE80003C020ABC059AA6FCCA221C70BC0E98AEF5
:10AE90007A30EA8304D88C1B8408D86A3F8E8E0CE3
:10AEA0004F4A777C8C173C019A4ACF48B09C108C53
:10AEB0009F0E3C7A7AFAFAFADAFAFA9C98FAFA9C35
:10AEC000901CAA08E0781C101C0A70383CE6359AE1
:10AED000D5883ED37C62588ACAFCCA0E4DA459A4B8
:10AEE00098EE6E6E1CE5A46E1C6A578E8E986258A2
:10AEF000E24B4A871CCE7C0ABCA34ACF4670CE7C6C
:10AF00000444E0441CCC1F4C3BF80E38AA7CEAEB0E
:10AF1000C8E247C4EAEAEAE66FC628AE4A7CE8F827
:10AF20004666E8890AC6369B4E7048D3C44CA0F8E2
:10AF300046E8CC5795A43C0AED184435BEA918DB69
:10AF400036AF335836C7369903CC1F4CA349A43DBE
:10AF5000A41DB43C3E6B980E4670110C1B19088C56
:10AF600060D91CB8492676C321067858EE319EB8C0
:10AF7000AAA81598EEA19268B806FDBCEE3BB80EE3
:10AF80000801AC1B95BCB806EEEE787CEE0CFF78A1
:10AF9000AE3CEE1C4DA459A4C1A46E1C6AA06E1C4C
:10AFA00058EE8D8C1C98EAA0AE4670855201AC0C10
:10AFB000604ECAFCAA3C7EEE1DA0EE3F706E85502E
:10AFC0000982705838EEF0982606C3E08E85506EE0
:10AFD0000801AE41A4CC2F46CA4602B8AAA8E08C0C
:10AFE0009F061CC3300B0604B898A8A63CB0FC1CF6
:10AFF0001086BC5C221B29CA30E6D3E000000000AA
:10B00000382338F338C3389338633833387CCA3C34
:10B01000B3FCCA7C933CCA7C737CCA3C537CCAFC9C
:10B02000333CCA7C13CAF01CE03CEA7C23D588225E
:10B030003803389338633833380338D338A3730070
:10B04000385B3833381B38EB38BB388B387CEA3CFC
:10B05000EB7CC2D63CF0AA0A6E701C1BFCEA7C7327
:10B060003CEA7C537CEA3C337CEAFC13EACA47F0B6
:10B07000983EAE4670E011A0EED3A5A461A47C1D5D
:10B0800088E6132E698C980A3C1C2376DCDC76E378
:10B090004E70786E682E70E638E66670E6F0E6264A
:10B0A00066A7E6AEF04EAAAE38AEF09870384AF019
:10B0B00098A9A6980A4329A44685A47E58FEC74CA1
:10B0C00013C809824E1C70786E700638EE2F30C09F
:10B0D00006A04EE0CC8795A43C0AB18C41AA2DA8CD
:10B0E000669FE68BE841A4CC2FA1A4D84A2709503B
:10B0F0001B29A4EDA47CC4483BFCCAAED851ACD8F3
:10B100008AAE06B7662F02976A833CC9AABC08308C
:10B110007A76EF3C7E45AAA3583C0A4DA4EDA49C48
:10B12000D08D8C98E041A4AAD8A1803C1BD588D8AA
:10B13000063F6660021F62607C8ACAFCD83E67D800
:10B140003CCA7CD8447EFEFE1348E6170A4ED8E07F
:10B150004E70381CCC17E20AE01CAEE6BD9E5A26A3
:10B160008F263B301D7C44D1026666FC084DA8C585
:10B170000278101C0A703988E62709503BD5883EB2
:10B180006F4DA4E5A47CE21FF6D3B06ADB11A0EEFC
:10B1900009829C101C3020F0B070660A38D88408F0
:10B1A000D8F04E70786668C4B18C0180BD9CC10235
:10B1B000CC53AE0EBC30E04DA459A4AA0A707C302A
:10B1C00021FCE0C6C2A0BB1CCCB76262627186CC17
:10B1D0008F1C23A237A2A22FA2E0A2A2A2A2A2AEFB
:10B1E000E06EE0469C5845A4AE58707C9C98E61CE6
:10B1F0003084FCE0C98C8ECE5C581E99A49EFE5B08
:10B200003E3EBBF5A891A4CDA883FE95AAFEF75CAF
:10B21000224BFC261CE2CF8D8C8B22A70422170820
:10B220008DA4300F0C2391A453F5A82691A48DA4CE
:10B23000CDA841A459A49DA4698C7C698C0C63FCA5
:10B2400061A40A4DA4DD8CF846E8C502FEFE37CEA7
:10B25000DC95A4BB5C62439CE2B790FC5DAA628370
:10B260009CE26FD0BB8DA4FEFE33FC261CE20FD007
:10B270001DA45378EEA091A478CECE68C330F0AE72
:10B2800058782366CECEEEE798AEE0F8261F66E04B
:10B29000044E6EA05CE070CCA795A40C133C52D871
:10B2A0004A431BD5883E33E6DF09503359A4E5A451
:10B2B0007CC4488AD80EB0CA70AED851ACD832AE71
:10B2C000724B06AF662F028F627BAEE3A9184EAABF
:10B2D00058AA0C41A4B0AAD80E442BE5A84C3F7242
:10B2E00098121B0ABFAE707C066550A01C4C60A66D
:10B2F000E8B00ADD8CF8E0C41BC488CC27E5A403C1
:10B30000AABC3A30F6EB3A3076EF7A76E11B488CFD
:10B31000A91A7ABBA24BAA626266700A387CA27C28
:10B3200082E2FB2222A0F62BF61BF64FEACA8DAC76
:10B3300082E25322223BF6ABF69BF68B29A43CCA51
:10B34000E0E2EBE2FF36EF36DF8C258F8DAC8DAC83
:10B350002237484C6029A429A48C173988ED1AE2B9
:10B360008B8DACA253AA101C66700A38FCE0A27C3C
:10B37000E0E22FF66051AE7660EA8DACEA76DB0350
:10B3800004781C10581CFCCAEE30BF26AED8666B81
:10B39000D8AE7070383E437E1E1C6A237C6AE74A32
:10B3A0007F1C8A8AA6B63CCA087C7E137CF03B0CC4
:10B3B000234A3CB33CD84670D8E0B083D813AEFCE7
:10B3C000EE707C1C0A3988E6CBD5883EDBFCAA0EE1
:10B3D000584DA4E5A48A1CDA7C0AFC6AB74A574691
:10B3E0001CDA707C0EB0EE730C33466E8D8C3B987D
:10B3F00008231C980A7C8B3020061CF86AF3B8E0FE
:10B400007F61626364650060060405010C1D7E0DAA
:10B410004EF05C90308C3C0EE5A41CEA5730051CC5
:10B42000426AB7C1B06B3CC1B0E02B6E30051C4224
:10B430006A9F9E301F0C23E8BE3726BE1FE8EBE054
:10B4400020DE6DBA5E270C71B049241CE5A43C8E49
:10B45000D91C7C5675B0AB3080A330C08B0616303B
:10B460003A66AB302C66A3302E66F7304006B8D86B
:10B470004C5F8C4FD8DC101EDE7E3353D8E8302072
:10B48000DE237EBE7E70E8E0163020069730600630
:10B4900073A6D844D806B03070A646A0061B4E5CF2
:10B4A00090101C30663322E3303A5B3C56363B0E3C
:10B4B00041A4C1A41C426A60FC5C021DB48E9C586D
:10B4C00006164670307F66851DCE0E1C7C66DD8FAD
:10B4D000FC0E1DB48E9C58467051B473E0200C6075
:10B4E0004C3FC8CC37486D00CC603080E666FBE04E
:10B4F00030107030FDF09C4ADC909C905C901C9069
:10B50000282828E049246E1CCCE5A66EC9A6381C64
:10B510003CEA6D591C387C0EF87C0AAE28B87C0ACF
:10B52000AEE8787C0AAEA8AE9C9868E0E6251CE6FA
:10B5300056069C58B87CD804D83CA8F6F62F468707
:10B540008CE70C23300BE08C273077E03087E0303D
:10B550001C66273054E09D580CC92289BA84B898DB
:10B56000A82B88B898A80CA78CAB307F069C98E6CF
:10B570008D2666AF652083B83CD808D87CA8D92032
:10B580007924BD2025241D0239B478FE37FED91C4C
:10B59000B81B09B8469875B031B8638C41BB41A45B
:10B5A000198C4E70D92041A41E8EE5A41CEA2B6E86
:10B5B0008DA41E46700C1B29B8E05CA078A0FE7B11
:10B5C0009E60FEDE7E5B8C4BFE301A31B8B37E602F
:10B5D000FEE0D4577822AF145762DC5058D4A099BB
:10B5E000A4130C778CC37EB77EA7C314B794A70CA3
:10B5F000931CA0301B31B878F65329B83BA08DA41A
:10B60000042BA08DA4088D141D02301C9C5899A6F3
:10B61000307F66937846977EFE2F410CBD8AAE8DB3
:10B620008C29A44670AE68633E236520E3AE99A4DE
:10B63000BE008B1E41A459A4BE1EFC1CD08D8C7E66
:10B640000723781E9ED91C5EA0BEB8E3301FE830E9
:10B6500020DE7E6F1E3E5E23E8BEE346F07068E0AB
:10B660005ED3B8580C373CD888D87CA8469C98063E
:10B67000307F667F781CEA3FDC10FED91C1B09B8BE
:10B6800061B6851CDC10FEC1B051B6C98C9C9870A7
:10B6900041A41E30F19C5899A4B09C5899A4AE7E48
:10B6A0006815BA4E705C105CD0100EB8B03C06FA4B
:10B6B000FA7C4638BCA606583C28E0E6174E7009CE
:10B6C000503344A180AA70040A4DA4EDA4D80C27DD
:10B6D00004D8330804D88D8CB00E3988E603D58899
:10B6E0003ED7AA0A704DA40CEB08EDA47CA24BAA8D
:10B6F000626266700A387CA27C82E297E2EFE277AF
:10B70000E263DDAC4BB0E60F700C4B41A44E70E829
:10B7100028DD8CB8584CA0D5885FE27FE217365FF1
:10B72000364F59A4E5A47C22D7E38DAC0BEDA47C65
:10B73000563C8D8CE5A41C4AEECE8D8CCE7C63E508
:10B74000A41C4AEECE8D8CCE7C1BA6FC586E1DB47C
:10B750001C980120C3AEBCD91C0C733A3A3006A623
:10B760003C2EEEB9BC04D5124D140912D91CB9BC3B
:10B77000CE3C061EA114B81CD0E8661EA11463A618
:10B78000EE1C1084101C421F02889C1BDCDCB6EBF4
:10B79000E6161FDCD64E94602213E2B6F30EF88C48
:10B7A00017B858B0E0EE2798022398AE4EF0E0CEDE
:10B7B00070989801207B0C3FB858B0AEBCE06E4D3D
:10B7C0009CCE0592810A4404040C4745A4E5A45983
:10B7D000A42B6E2DB46E66E66ED91C4CD9B0D9126E
:10B7E0000C23EE58EE04D80C23080408D8E0BD1C46
:10B7F00018120F0D20E000000000000000000CB93E
:10B8000062204038238038C4F800C4039D1033D42C
:10B8100010D0CC0C0011802C2E122151C04411717B
:10B820003333809043A21A1F0035802093C1477F95
:10B8300020C4A3612032E2CCA3C838491C524981FC
:10B84000304443C8C64304224B1204F1EB003038A5
:10B850008431000000A00091869B8CE3321070D0F0
:10B860002A8348F420B806B3F836E2C90F0A92805A
:10B870003D86330033E3C94D03DC50C1832303000D
:10B88000440400300C00C07C373B280C0A5359CCD0
:10B890008A6892C4BDCC0431BD4C0C0E04E2A07881
:10B8A00038E00326143003DA203E180470483C4B7D
:10B8B00040E000002920CD9C84FC92EE2E4F87C0F2
:10B8C000804CE14430D00F461263E483E0384E10E0
:10B8D00086E1330334141258D131B2348A104D400A
:10B8E00004C0A0A20894D3206A153E053D0BE132A6
:10B8F0002138FCD7913944E6109943648E7A557209
:10B90000B4EBE27EAA2FAEEF8804E9AB701248C414
:10B91000C87675C4BED2C4D03CC8E4E8E2E1121ACD
:10B920003180CB4E02C258F8F06F8E0808A57D6DAD
:10B9300041C308EA1433A4015FE083F2604382004C
:10B94000C02C50CE0743710E6E4C8FF7C40C0D0601
:10B95000211895C54C4851A37B8DCE8DD7D40C139F
:10B960008A5A851332020C836C3854C8030C2CDEBF
:10B97000D1C404F37FC49C46D74D41334CCC3C0F1B
:10B980006195D01805C2D2A0C47A84C1E3121ECD3D
:10B990004EB838910C51A57DA23EBE8C3DD2704F61
:10B9A00060813B152E2DF67C3C70BC08A456179484
:10B9B000824F240AE00A40330108CF23F240F808FE
:10B9C000BA08D92008553CE038ECA8FA0C5021C43C
:10B9D000722208C7805E0808CFE1608E388E16623A
:10B9E0000B622F880833C20F01E7A0080328232227
:10B9F0006060FE084B0087B8C3913F2759227B0047
:10BA00000400008C00444400C820CB0DC4CC8C281A
:10BA1000C404008C0C4AFA0011110088093E06404B
:10BA200088508FEFB82BA0880F0260824D3180B90B
:10BA300008E01A12CF000522EE0741338C3C00418A
:10BA4000F0F3DFD43ACAD5C843078D40F3F3004979
:10BA5000515BECD038508380486C28C91C1132806F
:10BA60008C2CCE8CC094688C8B3B003040FD0C49F4
:10BA7000520D500D40145D55373324C34902C3188D
:10BA80004A4C50D8821B6449133184331103820419
:10BA9000D0C03C09CC4B0EE0394F8EBBB33EBE0745
:10BAA00049EFF1E22100414403880F230F051024E0
:10BAB000F3F30F015540C544CD03013C13FC0C4882
:10BAC000E4EEAE11E1816ADC861EE11086D2ED2340
:10BAD0008788181116CF704444301ADC878313B856
:10BAE0004C01847421983DCDF02034C9E0868D014D
:10BAF000008580438D30C40C208103604861F4FFD1
:10BB0000000000004C71B204FCE0180143C461BCA9
:10BB100013D30422336110447C7C4CF4217B0C1F32
:10BB200042FCC4C470D7F14CCCE3313821E310306F
:10BB300081F11008040CC2DEF228DFF9611C20300C
:10BB4000D50148E23A7B1D76D411D30434F777351A
:10BB500000B1C4714C2C48F0C74F128D33C2FD0D9B
:10BB60003131A0301310B1108010200B030A302A9D
:10BB70000A3204AC608A38CC3C23C2CC4C800A32F6
:10BB8000C1141333F18E22020C2222327131E443AC
:10BB90006ACCF771203937EBFCD4DF4C312DCE1055
:10BBA00032CE880C41CC30830236DF5B91D1B8C1F4
:10BBB000E4008D3C4D0F140E4A4C2007AA71DB5156
:10BBC0001DA342A0C3FB102632B21ACA083200BC21
:10BBD0000C008F0002D0805EC834233310F30F7343
:10BBE000DB2E0DDFCFF152F7D84B123A30000FC5E4
:10BBF0003043CBC810240C3341B4E43F000E004066
:10BC0000193F0097013B01C60A430AD2057C01D2C5
:10BC100001520A19008809B409AC0D5B0D630C16BA
:10BC2000016907F7037206B20E6205730E3606ACA1
:10BC3000080B0A7B0A85010303AF02B5068600B133
:10BC40000DE403490F530F5B0EC30EBA062D085FB8
:10BC50000E690E2F08050F2C0F350173035703C013
:10BC60000C0400AC009D03B809A300E306A20B2F4F
:10BC70000AFC00F7012001290132023C02CE066CC9
:10BC800000009319050B0C030B8045628432200ED3
:10BC90000306201418052D8D0F0F1213010B80556C
:10BCA0006A8E0306201418052018032D851A09131F
:10BCB0001001C870F868385C581C0E38AA28B044C7
:10BCC0005D5C385CD8284C9B5D1CCC274C09820DF0
:10BCD000FC0E0F20120F0F0DF1FE80BD6A981209A5
:10BCE000040D0581408001620DFC04151020060C36
:10BCF000F1FEBF0705124E78BC067CC6007DC68EDD
:10BD0000130110A9D09868F8F67B0DFC0B051903F8
:10BD10000F0405D9FE009D0E809D66BF0E0E3D18D6
:10BD20000B802D4ABF0E0E4D180B805D4ABF0E0EC4
:10BD30003C180B808D4A870E050C01F9C41379C499
:10BD40000C1B06434E3005EA6DCC66A606E0980F44
:10BD5000140179C40C1B2E53468D8C9C985606F505
:10BD6000C4B94A851A09130C068889E8B08BBF0547
:10BD70001A0913C15C4E70783CC62B0E1B841E3012
:10BD8000107046F0A1144E708C60DE9C7E7E2726DB
:10BD9000D4E30A061E5C422FFAA6E30E8EE0E1C44D
:10BDA0000459A4EDA456E63F3005426AAF089C58FA
:10BDB0001C38FCAA0A7C28E04E703830081C901C05
:10BDC0000A838D150E0179C40C600B801162940FEB
:10BDD00012010B80696660B0307CDADAFC3A307CA4
:10BDE0000B00E00B00E0D05C3066603AC60E300617
:10BDF000A075227E477E59F37E19637E0D4EEDDAE3
:10BE00003CFE4E66A63A5C105C223730C6E3692ED3
:10BE1000D05C30C6D7CC2B71CC66D3550E7C1C3091
:10BE2000060E7A30EA592FA6D3CCDD0E5D1C4CDF0E
:10BE300071CC66BFE92EBF0E0E3D3C180B80714AD7
:10BE4000F80E30E82BF80E3000E6AE6150600E566A
:10BE500037300306E3AE8D080626D3E07E7E895395
:10BE600060065E46FAA056607CA647FCA62FFCA69C
:10BE7000B5A2E10A814081C866BFE6856813A36662
:10BE80003168C66687E61568D34BD05C30E613E0B0
:10BE90007CE046E098E0D91C788C2B84D8842388F9
:10BEA000D888D8F0492660A0D91C783CD888D8FC1E
:10BEB0009B81130F100B80096A0B80F96A0B802598
:10BEC0006A0B00CD9E0286C6E0BF0E0E3E180B80A8
:10BED000C54AD91C30126A5F78D88C1F881384D861
:10BEE000F06330706A63411C30186A9D7E4EF00525
:10BEF0007E78E2D3411C4CC76100D1441BC17E193E
:10BF00007EC676C3A5D00C60C6762330EE13469667
:10BF1000864686AE0E7C0A85D026E61C4E8223A677
:10BF2000A2A2A21F26E386EA02AA0AEAEAEAAACAAB
:10BF30002AE0856813E0A6062658D944E0EB5D1C8C
:10BF4000214687010C060C0312B830FF3CEEB94ABB
:10BF500087010C060F14130B80FD6600203C56066B
:10BF60009CE23BA0005D1C21463087E099050B1444
:10BF700005070B801D6681408488ED64BE58300241
:10BF800089408808AD402570BE981D608CA7FE1FB3
:10BF90000E5B0E300555703BA00EAE00D164EE89ED
:10BFA0004C690208A140257088A393100C03100B64
:10BFB00080696E9807120C030B80C162863E3C18A4
:10BFC00015C845CCB87CAA3CA845CCF5C4CEE871D0
:10BFD0001E5CE6A616E61376A6E6E6E6C6A6D4142A
:10BFE000A3E09828C488C4FD7E3E4E302C5808300B
:10BFF0004070387CE0304070387C063CA6BCF0E0F5
:10C0000059A413A63040562B3001B6166660A5D051
:10C010000CA01C4A2A704E5CAA0A7C9C4AA606F018
:10C020007C70383CA606BCF0FBAE0E7C1CAAFC0E55
:10C030003040562B3001B6167030EF06383C662380
:10C040007666471C4A2A703866F308AE0E7C1630B6
:10C050000156BF0670F038665BA6360670F038668B
:10C060001B062B1C90D0061CE076173670383C66F9
:10C070008B3001763F2BEDA45626E66630075A1327
:10C080003AC6F306E6BCE2667CE62B4E2E1CEA8539
:10C09000D04666064B66861C82A0A2A27BC666A519
:10C0A000D046A063044E70F8EECE71C8700439D04B
:10C0B00006B0BCA6700C1F08B30C60783C06B03C00
:10C0C000063C068C3BB958BC70B95A3C70E06EA077
:10C0D0005627FAA6F330030C1B6608468EAE608D19
:10C0E0000A304056A03001B616E0041308081B04BD
:10C0F000044E7038DC901010102884444E5870386C
:10C100001CFCEADCD0BEEB59A4EDA48A1CEAAB0A05
:10C11000302C6A1F48B3885E5BBE980C23AA3C1B78
:10C120007CAA581C6A3005426AF78A985E630C2B19
:10C130003C58BEC37C1C9010CB2E5F1C38FCCA7CC4
:10C14000288C6F0C0B0CA0CC23D5886A41A47B0CE7
:10C15000A0986815980EEE734C670C771C9DA47C14
:10C160000E7C0AFD1A0DFC0E010D05D9FE83051289
:10C17000140507884B8305120C031201840B80A160
:10C1800052E54C0CA0983C063C4C3B0C17060C139B
:10C19000463CA63C9C4A0EA04E2F8C7B5C628E6671
:10C1A000665C1BFAA642EB8C13BE600D544924F862
:10C1B00028AEE8B5BCFD5A064C2B48B03C06CE7CF8
:10C1C000A6FCEEB0FC061C0201D08408CEFCAA0A34
:10C1D0007CEEEDA456E6C6762697CE7C4C1F261341
:10C1E0006603047CAA0ABCC6BCEE8CC3B07CA6263F
:10C1F0005F0C4FA646BC26BC703A4BA626E6EDD097
:10C2000063FCEEE626E6EDD00C604388983CAA7C01
:10C2100058E0CE7C0698E6B07C463C70B0FC70BC22
:10C22000A63C66063CF0E09301051601130B8099CD
:10C23000568891D04E70F80E300255701BB5A2AEE4
:10C24000BCEE514C4E70783C06F8C4FE1388CEF616
:10C250001348A67C9C4AFE1348A63C583154BCEEB9
:10C260008940A808B156BF0E0E3D3E180B80A14A6A
:10C270004E75F0EE600DFC0E0F200412091605F14C
:10C28000FE8C06130F1049F0F9C40B80E6E956BD89
:10C2900056585D1CCC604C6060B03AE08D0F0F12B8
:10C2A0000D050B809D5A8215131405074433901415
:10C2B0000507480B80594200BCA8E04E0070446856
:10C2C000780605BCEE59DE785E3E683C06660401E1
:10C2D000AC0EC1B01C0C0742271D145BAE012063DD
:10C2E0000C77AEBC4D14DDAC4924E304B1BCC36E85
:10C2F0006EC9A46E085346F059A4E5A459A4046677
:10C300008E060404D91078065830301C622B30B0E9
:10C3100062275613B6D91CB8B81C101C8C3342B80F
:10C32000302DE876B63CA23C3E1E7E7E8518492420
:10C330005DBC99C844785CE291DF3084CC2766EB21
:10C34000B371CC663F785C62683DDE309366FBC8B3
:10C35000CC2FC8CC0D541C101C02784CBB426F76FD
:10C360005B6267A21C10101C021776A268C34E5CA9
:10C370006244D302FDDA3668F6F65BE2E21FF6337A
:10C3800078562268E201DAFE435CE2234830F02B63
:10C39000C1B0BD1C03011420050D101419DDAC083B
:10C3A0000170650E4E9C90CC67601B7A1F7ACB881B
:10C3B00059C8550E1CA020E2F9CFD91C7858492441
:10C3C000300501ECC27012C38700233BB313BB0DD1
:10C3D000549B8CE378068605BC95BC66866608018E
:10C3E000AC4359C85B785C42688859C851DE8CEB15
:10C3F00048C393011405070B80ED520000000000B4
:10C400009805160113883398140507843DF0B0068B
:10C410003C2606F9FBE6C622BC70067CF03DD04EF9
:10C4200070F8AE708C2F38EEB94AAEF0E048F9C41F
:10C4300046C10238467CA65849F0DDD4B0E622FC5D
:10C4400006023DD08A983C0A05CC98420C172E0A69
:10C45000F9FB4EB07C5CD070FCE090051601130B2C
:10C46000803D6A4CE57A040D7CF57A0B80694606BE
:10C470007038F61366663C1EE0D09C30583A1C3A81
:10C4800030E63A30C64FE63F5C50D0D0F19AE60E27
:10C49000BC427CA67CCA70BCA6F6F6F6E33A3A0E1D
:10C4A000303C1E78AE7E3A3A306A677E8E8EFE2F22
:10C4B0004A2F440B4A97BC430E98AE7A30EA830465
:10C4C000D88C1B8408D86A3F8E8E0C374A77BCFD07
:10C4D000E24AE748B19AE6C532308306CE3C56665A
:10C4E00037B85CE2E2E2313238FC9CA262CF1CA297
:10C4F0003C28352EE0DCA0DCF2C156A00EAE1C724A
:10C50000CD564EEB514CD1C8E653D144E0C4F57E34
:10C510007D6813BB664670385C5228A658BDE0BEE5
:10C52000EF983CA6BCBE580948EEEB86983C7038A4
:10C530000EC67066E6386E33EE773A6E5F300406EC
:10C54000983A7EB75826371568A30DFC0E0F2013B6
:10C5500015030820010C0DF1FE266F29E60948EEAF
:10C56000DB33D1C8E62B4670F828B8EE4670CEF023
:10C57000F1688E1C527C706944E86E754CA8987006
:10C5800038F6274E70AB98267038463C05688D709B
:10C59000CE0EDC52BC702626694468454098803D2A
:10C5A0006A84050B800172840C0612038443930194
:10C5B0000C0612038801C8E6B5A2DC908C133E6815
:10C5C000BDD00881F08CA1C34E70780666263DC2AE
:10C5D0005AEEAE3C700698F00DD0A6065870CEF01C
:10C5E00070088C6366700201D030FF8D8CA658985D
:10C5F0000E0DD0A65870B0662F704EF09B0C234ED7
:10C600006EF0C102847E1788B0FC580670BC9C4A4C
:10C610001CBCF004738C060C033EA5E8B07E7E2B98
:10C6200089F63E8C1B78EE55F2BDD07DF20DFC12E2
:10C63000050320140F0F200C0F0E07F1FE920803C4
:10C640001010018408B5E00CAFCEBC06B07C8C2F76
:10C65000A63C707C26E6CEFC0AEDD0AE7C0E980699
:10C66000CEBC4630FF063B3CAA8D8CB03C0698E61B
:10C6700071D8849803920803130E09884349EA830A
:10C680000512130E0904B5E00CA7B03C51D8CE3CFE
:10C690000E889826587C9C0A7C1C0AAE7098E6EDA1
:10C6A000D0B0AA7C0EEDA4AEFCAE8D8CAE7C0E7C20
:10C6B0006A93846262901C622751EC02AE8C2FFC5C
:10C6C0000E888B987C0AFC66588C9BB383051210ED
:10C6D00010014404B9E049D8987C0EFC2BEDA45914
:10C6E000A4AE7CAE8D8C01D098663758AEFCAE738C
:10C6F0004C6030FF8D8E8C061A1305120B807D4A1C
:10C700005ABC1A203C06B0303AE62366DF461AE0EF
:10C71000411CF53E30EFB616666F3001B670387CBE
:10C7200006562306B66666E09819050B1405070B36
:10C730008005427924B5BCC10208D8284E2E687005
:10C7400088C4651C0488ED0600000000000000009D
:10C7500000000000000000000000000000000000D9
:10C7600000000000000000000000000000000000C9
:10C7700000000000000000000000000000000000B9
:10C7800000000000000000000000000000000000A9
:10C790000000000000000000000000000000000099
:10C7A0000000000000000000000000000000000089
:10C7B0000000000000000000000000000000000079
:10C7C0000000000000000000000000000000000069
:10C7D0000000000000000000000000000000000059
:10C7E0000000000000000000000000000000000049
:10C7F0000000000000000000000000000000000039
:10C80000810F1418F8EECE7EFE595A15C89C58397F
:10C81000B69209040D052E009170A56CBDCC06469C
:10C82000BCA63CF0BDCC26BCF0883E4E5859F08CDE
:10C8300053C1B01C4E901A987C5875B0BAD33020B2
:10C84000E8B03000E6E6C67EE3E8B0DCD00EA11426
:10C850004924385E285DBC8001529CC22B387C661E
:10C860003B0D54663002C61306F5C44E708CB551AC
:10C87000EEE8D5CCA6A62FB5BCFD5AC1B0BD1C04B0
:10C88000091220050D101419DDAC080170B902DC85
:10C89000901BDCD0FE84480453DC501BDCD0FE042B
:10C8A00044848404040E30407030BF0638661B0890
:10C8B000634C537C66B5F7EE7CE6FCEEAE0E3CA610
:10C8C0003C263C0E0C7F7038AED86E1788D8AE2E42
:10C8D0006F8C1B6E582DD00CE7A6067038FCA60690
:10C8E0007C7026E63DD00C6F4C278C5F83CE7C6637
:10C8F00037FCEE4B84AE0E3C06704E6EF00C278C6F
:10C900006B8485D0C6A686A6A5D0469330EEA62613
:10C9100086065C424F9B880C2FB0BC16DEBCDEF353
:10C9200076E30DFC060C2014191005D9FE0DFC064B
:10C930000C200E0F1420060F150E04F1FE1C3040C3
:10C94000704C57AE0EBC06387CA6BCF00CA04E2E28
:10C95000BC30BFF0E09208030C0504884383051245
:10C960000C05048449F08808E9D48CF9FB8C7B4ED3
:10C970007001C898A658CEBC06B07CC6E698A6063C
:10C9800027C6DB0686A6467098C60658CEBCA6C645
:10C990003CAA8D8C98E63C0AEDD0987C83B07C460E
:10C9A000707C707CF0CEFC0AD9D0CE7CAA0E84EDCF
:10C9B000A4F0664BB0561C2A13886A1CF0AE7CAEFD
:10C9C0008D8C8C60A293A63040562B3001B6166633
:10C9D0002F70383C06A2A2A28CAFAEFCAE88338C7E
:10C9E00006121510A068A5E88EB05A580881F09874
:10C9F0006E46262642EA4E7078063DC3BDCC46BC44
:10CA0000F0AE0E3C0A3DD0BA3CE6A670A638EE70F9
:10CA1000EEF0DA3C66A084A63040562B3001B61604
:10CA2000661FA5D0668C27887B981205160113888F
:10CA30003B9812140507843DF0B0588891D0B00699
:10CA40003CC61306BCA606BCD870E63C4626832628
:10CA5000E698A658B0FCA61C223DD098EEDB9214B6
:10CA60000507843B920516011388DC90FE95E8C10A
:10CA70005C4E70783CC6A660E6B006978C730DFCE1
:10CA8000050E04200F0620060CF1FE66A6C686BC25
:10CA9000A6BCFAB0FC060DD07AB0FC70BCC626BCB1
:10CAA000F0AE7084448C57A67CA63CA6700488B374
:10CAB00008849B90011713070512484B85160F0D2C
:10CAC000070512448491D0E6136670063C063C06C6
:10CAD000B958BCB958063C0627883C70B00E3CA635
:10CAE000BCA670840404B07C7038EEB07038EEF0F0
:10CAF0004C33B07C70CEF0B03C66603C048C7F8CD4
:10CB00001B661326700C600CEF3C080C9B700E2DFE
:10CB1000D0B0A68BAE7C0EB0E622FC06023DD08AD9
:10CB2000AE0E3C0A05CE94100B050513844B811400
:10CB3000100B0505138889E84E7001C8FCFA1E7EAB
:10CB40007EB0FC70BCA6063C463C7080C15A941076
:10CB50000C031284438114100C03128889E8B03C42
:10CB6000A6F5C4CEF07C06F5C46EA05A233003C6E9
:10CB7000B01D60EEB94ABD1C20051212DDAC0801E3
:10CB800070ED8AA188C1B0BD1E492404CDB4734E96
:10CB90005C90D0D010309C6262BDC06B49A43DA4B3
:10CBA0008A3DA4E5A4581C22071CAA588CDF6AED14
:10CBB0001898EA6DCC3010701EA114D91C7E9EBE50
:10CBC000B8BEF37EBAFC8518F90E46F070B85CE288
:10CBD000E2E24660E21BAE4BAEBC067CA63CA63C45
:10CBE0005EE0000000000000000000000000000007
:10CBF000000000000000000000000004320605E80C
:10CC00000000000000000000000000000000000024
:10CC10000000000000000000000000000000000014
:10CC2000000054000000009001000000042AD08899
:10CC300022282280008051018045028001C05504D5
:10CC4000C02422006024110054005001400500243B
:10CC50000204100D2002C05000000C0C00E0344F04
:10CC6000C8834F8A4F3C372C8E20C13B08E16810A7
:10CC70000D204E064065F3B8144DBFF48308922290
:10CC80000159C91D744FCC78E4452FC2F1020054FC
:10CC9000D450C1D8C430FD3A06FE876130164E41EB
:10CCA0008660434BC43D898BBBD1D3BB031011516C
:10CCB000D100034035312DE212133131D5C172500C
:10CCC00031E04C0005D10444151E50455D4C762FD3
:10CCD00003005C000000194207C9C4004066021648
:10CCE000F6460522501012B4CD460A001900740011
:10CCF000318F4F40384454F37F2B4147888714E0ED
:10CD00004331410F3C4A349009941140314166301F
:10CD1000CD2823514ECA60CAC01F8FC2E72F080119
:10CD2000B60501C2C8105D07FC2210301100FB04DB
:10CD30002244448C738748E0C4073D03A3064AA4F9
:10CD400080C1084B31C1142013044B03D60F1B02C2
:10CD5000023D0CC1E724E20051086000800000524F
:10CD6000D147842000923374CDFD6405C1111104B4
:10CD70000004F04020800661761402C404640012AE
:10CD80000012EE450D0511A0803900102148410028
:10CD90005238B18C40225015F70500549C0B0060AE
:10CDA0000020409A25CE660040050002205D3EA985
:10CDB0002686E8B534D00C004033C14149C223A3D4
:10CDC0007463C71333CDEFD27188521027BAD2E300
:10CDD000C4B84EF9F3B5A78448F623C2BAA24521D8
:10CDE000A28D6CF63300004E32C884B83260301D1C
:10CDF0000100104CE98608B7203B2AE10E0019001B
:10CE00000008804278001A0A820280078F442200BC
:10CE1000215410E1417004001D65155D2275F3B8C1
:10CE2000E322C140244354689FA88F2F638F854B12
:10CE30008B3D1F4FBCA244C05C357A9F2B0896D413
:10CE4000C515724F45A1214505910921A130E24444
:10CE500029BD290000603C981F8E04884668819196
:10CE6000089282470BA9C55401110002008620A236
:10CE7000833C683D40964089240204500189800724
:10CE80003A8A500A640200E8C0A48C0800006000DE
:10CE900080C1612444020555582C00146001800EA5
:10CEA00000040F80996110440009001073CD003C0C
:10CEB0007D840900500011C8000049C01D000074A5
:10CEC00094D4CA63114113480DD4000051DC70980A
:10CED0001913000000000000000000000000000026
:10CEE0000000000000000000000000000000000042
:10CEF0000000000000000000000000000000000032
:10CF000000804A0C00404613912302090D54171D5E
:10CF100053B58F34215E94A01611043630C5D10C60
:10CF20000080938C20000802F01246CC800200148E
:10CF3000482734878189904020227082815389025A
:10CF400031057041D43D5124230060080000601079
:10CF50000215828F8403800080427218468451C477
:10CF60004820514800511110204241B420B02C00FB
:10CF7000F0514CD008550B3C00094048A4803E03BA
:10CF800052098180487F314103FC038000A0104298
:10CF90000451019D4400480420002800E0D43022C0
:10CFA00000008640040480620208117C1F0000001B
:10CFB0000088488851C41004C14B02824022380CBA
:10CFC0008838C693C014400854000003000C184071
:10CFD00081124404C000C0000454E0440030809337
:10CFE000CCCC4406F5BF5A318CBC41400484CC40C3
:10CFF0003708C25EF501D4080C00000000000040B4
:10D000001A24005D0B6E08060F380B670B5F02D702
:10D0100002E202EA02F306340407010002C102C878
:10D0200001790089016E0122011701350B010423EA
:10D03000040F0B440CE5056009FB00EE09410054A8
:10D04000006902D0007A007100610000850D0914AA
:10D050002018032D83322020050D09142D9410175C
:10D0600013C5DA810D0C010C0341E68D0C010C0394
:10D070001289E6930D0C01120C03C9CE00000000CA
:10D08000000000000000970F0404A140F944694823
:10D0900063C1B0981E7E3570DDAC6564983102586E
:10D0A000300370C158CE6152814084D54CF88C1346
:10D0B000B86ED330200C3330188C1326E6A18804C8
:10D0C000B17022D91CB8C6E86564ED8A389C4AE084
:10D0D0003E3E3E8A1E4E62EFCECAD47EC31E4EAA8C
:10D0E000E05830107030FBF0E8E0850D0914D96885
:10D0F0008E7C5E61446948BB6ED9708B85140104D7
:10D10000D968754C694843C1B008F548656498EE24
:10D11000B94A97130C0312514C04E5449B86010C49
:10D12000031295445B514CF8BC6944FEA0DC50E00E
:10D1300097130E1512514C68E08940A838A0FE1BC9
:10D140005C8A0E9E1EB1644E46D95C5C19688D7077
:10D15000CE0E5C7CEACED95C5C4AFA1F4E5BA00E18
:10D16000665C1BFAA642EBAE0E60E099040DB8BCFB
:10D17000D844D87CA8E0990D04B8BCD848AB0E8E32
:10D180008EA04E5C504E4E9C3E3ED05C4140603C7A
:10D19000E00408E0DCA046F098067038F6136666F6
:10D1A0003C7E60BCA6BCDC100EC1B0AE5C900E46EE
:10D1B000F03C70380C435C04F2277CA2E370D91C6D
:10D1C0008EB07C7075B06E8E5E4B5CA2A39CA2AFDD
:10D1D0007AD30CE361009CD2BB9CD2A0C1B0DC101E
:10D1E000FE04041B300B3C0E1CF86A1FBEE3B8495A
:10D1F000243E616A856869547008A968E60670383B
:10D200001CFC6A6A1E6A337E7E98A658B08148ED7F
:10D210004E6954BE3E0165DB000045DA00000000A7
:10D2200000006954F693E0DCA01CEE982670380EDE
:10D23000A0F2A65EEBA6728940387C323200003242
:10D240001F12EF662792B2939260981D68A6049809
:10D2500070CE1C42F0861E81487E98C6BE6066EB8A
:10D26000F613263C5E9E9870380C134E7098532629
:10D270007038A670A6F066A60626AFC670B0F0BEDF
:10D2800033E0300870A6DCD09C1E387C4A3CEE604F
:10D29000A6BE60A6067038BB8940387C4666E6A606
:10D2A000260E4B361CE2172AA6496870383E607E6F
:10D2B0001C128B1C42F0935C0A6029FEAB05140122
:10D2C00004D9CE93190104048DCE980D0C010C03E2
:10D2D00011E6B2310B0C03DD48449828E0B4320B60
:10D2E0000C03DD4848AB940B0C03DD48846B8414BD
:10D2F0000B0C03DD488823514CAD72754C46178EDC
:10D3000030020C6BE01CA01C50509C30057217665C
:10D31000884884DD6C0C0BDDAC4E30200EB8B8B8FC
:10D32000662F7EB86623D888D8E8492438D91C9C53
:10D330004A9EF9447E3570492659CA85683389402A
:10D340004EA8E0454A93000099CA08C1B04944007C
:10D35000B9620058894068F858A8B80E4EA07A60A3
:10D360006E1F8CA0A84E2828A82828E8E828E8A83E
:10D370002828E8A8E04970136BDD48A00E3CAA7C81
:10D38000C6A670663004062B301246BA9A4EA6BC6A
:10D3900001700EB01A9A70DAA5709A7C2B816CA07D
:10D3A0000E0E4924389C0AAE284A7C0E4E5C50D0A2
:10D3B00010101090504E5CD0905090DC4140AEBCAC
:10D3C0000E389C4ABC70BAA57070BC0E4E1CD010B2
:10D3D000903A5C49404E5C100E2BCE7A1A23AE7CFC
:10D3E00006B0A6705A0170BC30120EB0BA5A7A66F6
:10D3F00006237AA646FCDA3C5CAA7C0EDD48694628
:10D4000094030512120F034843850D0914051344B4
:10D410004E7D4070CD6C49503C2EFCBB8514010400
:10D420001405134E7E708140EEB5A258CD6C448435
:10D430004950704570380EB0284CD3492478AECE90
:10D440003010956078AE68CEF0AE5C4E138A0A302C
:10D450001095607858B075604E3004583A3024BC4E
:10D460004960709544A0EE1FA01B2D60B02560EEB2
:10D470003961216CC4F57C856813E061481CCAF9E8
:10D4800072E0AEBC0EA01C30120A334A2356134A77
:10D4900016E004E0DCA005688EB03E777E4970138C
:10D4A000730950EA0A4BAE3C0E1C12D1501B84ABE0
:10D4B000D8EE271CD2D3D54CB540EE4D704E1C5043
:10D4C000501C0A1BCD4290901C0AD36E816C4E0EEC
:10D4D0008D70CE4EFD50A0980EE09ED95C4D70131D
:10D4E00063D95C8A8A4B30030455701B616A8A8A4F
:10D4F0008A1ED95CA04E9C909C0A931C3C0A73A087
:10D500005C99704E5CA5700E0E60E00E695013EBD6
:10D51000D95CDE7098067C6627B00E2B6670C15809
:10D52000CED95CFE23A03E2B6E6D50234C670BD9E9
:10D530005CDEA05CFE138A0EB0FE138AAECE5E6F78
:10D540009E2146307A66FB61020404981D5C5AE114
:10D55000080698467CA6BC58E01C987038E09713E3
:10D56000783CE64EC67CC63CEE514CC4780ED1E207
:10D57000B1640E681CE260CE3C58B96C6100CCED21
:10D5800057080C7F44E544CCCFE05CB5708C171C89
:10D59000D85346F0987CB95844CECC37FE2BA03EE9
:10D5A0007E538C2B2D548B234970630460B1702201
:10D5B00008D91C495C638ECC4FE01C214CCCF55C37
:10D5C000A0CCCF6089406C9BF89CE27B4970CC1D5D
:10D5D00070CC4F89403031E8F9561CF8EA23A8385E
:10D5E0000E98BC62EBCCAFA2023C580CAF0844AE24
:10D5F000F544CC47214CE05C115C3B6046F03013B5
:10D60000716487138474348575358676363718824D
:10D61000C21283C37300230B36363636363636369F
:10D6200036134B237BFBFB6B53306E66FBF1568B43
:10D63000030F0C039170E5EE995ABB05D40D5449C4
:10D64000248142115AB95A855A0DD49170A56CA003
:10D65000F9CE73AB8C374C73195C061C62131C42F9
:10D6600062315D33D38940F81C0CFFEABF4EA82815
:10D670009B4C8FB570A88C1B281368580C2555F34C
:10D680008C178C1F883B842B4CD73032155CA08CB8
:10D690002FA6FB415E66134660315C315488E54C31
:10D6A000AB8C9F4C8F0C1F0813042D5404434C3734
:10D6B0008C370CCF08A55A044C1F481344989C4241
:10D6C0001C4258C3155C044C374666B64893367600
:10D6D000DF1C862233A24C47C62B629C86A24431B3
:10D6E0005C4CCF3154BB4C778940A838700C255521
:10D6F000987CB958B004F544987C70AEF0C8CC7BE7
:10D7000008488C2D55C8CC3BE01CF55C46F0983C95
:10D71000A02660F61348315C7C26BC588CE54D6130
:10D7200000987C26167616577038AE98F038AEF012
:10D73000986E4971F9560CA04C43C8CC60A060208B
:10D74000E0CCED57E006983C0CA03CE03C0C173CCC
:10D7500058E0302E0C1B303DE830128C1B3004E8B2
:10D76000195CD95C065E3E4C1B3E234C17E63030FC
:10D770007CB6163C761B301FE8E67EABE0A0C1B05D
:10D78000600C495CD95C6EE00C2B5E4BD43B5E13A5
:10D790001C4C135C2BE01CA05E0EC1B03E04885CE8
:10D7A000421B3EC3EAE0DCA07EBB830491704C4F79
:10D7B000D8C9705C422F3E33D8885E3EFED91C78B3
:10D7C00068786860E0EAA09C9A5E339A509C029068
:10D7D000DEDE1790D95C13D07EF3D0D0D0D0D0D07D
:10D7E000D0E0DCD08C7F0A9417904C276210135045
:10D7F00050DC0210CA683828380AAE28A046F0E08B
:10D800009401030D0C017D681B796666A65E3E5887
:10D81000C4440D54E0C170843D6404CDB47B758C68
:10D82000E06564E04871682B65644164E04544EB61
:10D83000B068CDB42BE5AC88138478703D64E065A6
:10D84000443B8CE5AD3D6413208C758DE020843322
:10D85000985E580D54214C492498FE2BCC6F1568C6
:10D860004330FFCC3766EB235162203C560630181C
:10D87000662D5A308766D3309366FBC8CC6100FBB7
:10D880004E9C90CCA7601B7A1F7ACBF55A894858DA
:10D89000C17085641385644B1C20E2B78C73E54C22
:10D8A000300671643470C28412C300133383533B57
:10D8B000DBBBD14413037966E168E09C83016442D9
:10D8C00049621B985E3E4962E54C2B3008716480CA
:10D8D0003482C2848712C300CB033B3B6333538B38
:10D8E00073EB1568E365203BF168E05CE17084410F
:10D8F00062F168C1B008ED48B3447168008B294EED
:10D900008568668698663315C84D68CBC658E02092
:10D9100030F1CC256366E3E0E008017201EE884156
:10D92000DE9870C4F57CB058E0000000A09C4ED09A
:10D9300090CEFBE0B87CD88C6089028D0C011A195E
:10D9400018300289407D4070514CE83888084D50AD
:10D950007C46EE173A70842689400EEE6B8899500B
:10D960002B301AF1424E360ECFAE7C466860094825
:10D97000B0300446068C1B66367066A658851406C1
:10D980009806678826260613848568238C97A188C5
:10D99000C1B0BD1C0E0F20120F0F0D38F8214286AA
:10D9A000C626704E7EF0C6704EDC90901090F0044B
:10D9B000A96858B0C6260E2568869806B05568989E
:10D9C000A658A670660638D87066D8F026ABC67022
:10D9D0002658B0F65BF04670780E98702658AEF078
:10D9E000B09C629F0948EE173AD87026D8F0BE3F27
:10D9F000A6667006388BD152982B148140CD6C2EC0
:10DA00005899501BB5A2A0DE1B8E0E70984E5E3347
:10DA10000ED164AE734E9C501090D05010D090AE8A
:10DA20000E874570380EB00E286B8606B05568C656
:10DA30007038FC1CAA0C2F0A3967134A7CF026A602
:10DA400004A568A6A6E0A6496870381C3E607E1250
:10DA5000B3E0067038F61366663C46FC0606E051F5
:10DA60004C4EF0E0DCA030C0085C905C0E13664EBB
:10DA70007078067BA60670383EAF7E62A0FC5646E4
:10DA8000EE770CA0A398496870383E6F98A658E0CE
:10DA9000894833D144E07EA060B03AE06954F69BF7
:10DAA000982670383C05688D70CE0EBC555CD91C2C
:10DAB000B83B4C604EBB514C894038339870384667
:10DAC0003C0E0430059C5A109010DCDCDCDCA0FA23
:10DAD0005A13229AF33A0C534C2BC8CCA023CCED0A
:10DAE000576627D4BA73945BFA5A5CD0905CFA46B6
:10DAF00026139423FA10C3FCAA0E60E086011405D5
:10DB000013514CE838288140EE8349701B4E5BDC92
:10DB100050AEFC1E1B261FE6EBBC89403CA8E8E08B
:10DB20004EDC5050501090E084E80444D828E8308F
:10DB300029E8E0EE514CE8380E4E70AE68A0E09750
:10DB400013140513417013339E048D501BB5A24D61
:10DB50004C98DE1BA08E28E0B432050D0914018418
:10DB6000887B850D091401843B8514010401888498
:10DB700044417013CBB87C1C50600691704C23D884
:10DB80008813D8492430260213A222D888D88C7B47
:10DB90008662271CEAEA0604E948E2B308A3068C79
:10DBA0004FC9705C4267DC906B095060AE3C0E134D
:10DBB000FA4C47DCD0A25D6C6E4BD91C9C10D0A2F5
:10DBC0007CE89CA2BB8C608C603020616C30414C46
:10DBD0001B3050616C304D6E5851B6B6A31C8C7F13
:10DBE000A25390909C5D6C6E167693D090BBA2CFA2
:10DBF000302F0C4B664C73B8D848D81B4C3BE84BC5
:10DC00000EEE0E0EEECEEE0EE0CE30046944A0E035
:10DC100081400E3001A0A65C4636616B7606138A01
:10DC200066F3E0A0A01CE0DCA04EB2CEEE4EEEE02B
:10DC3000F16804E09C23E09C08A0C1B0AE707C5E5B
:10DC40000EAD5C0C60D91CF8F8B00EED4A7E7C1A63
:10DC5000FA5AA57013150E0D0F0E141505170504AD
:10DC6000140815061209130114B01A30E83ABEE37D
:10DC7000E09806C44924B8BCF6F6F6A088E004C5CE
:10DC8000703059D866F31BC570301E0C1BCC8766EC
:10DC9000DB2308C570302DD80C1BCC1F66D3C458AD
:10DCA000A60658E030107030FBF0A838238940F801
:10DCB000D8E0AE8444BC0E30121C0A776A53A0CA66
:10DCC0000A374A881B563348234ADF0660AE3C0EAB
:10DCD000E00E4E7078EE894078A0AE8E0E68E09728
:10DCE00013100F1413514C28E060FCB07CA0EE0E12
:10DCF0001CD09050A636369C133AA2F38E76E3AE33
:10DD0000BC0EDA3CDAB0BA5A707A9A4E5C109C417A
:10DD100040AE3C0E3C5A4E1C50D010509010AEDA23
:10DD2000CEFC70B01AE05D1C0C13C88498A8150CCA
:10DD3000711EE1688CD972E0C97020E0894038A07A
:10DD40002E2E60E000000000000000000000000037
:10DD5000000000000000000000080B6CBB8CAB0E44
:10DD60004E70B89CA2A8B5708C1B585B4C43C1B0D8
:10DD700048042BA16C044484617604588940594CB2
:10DD800038580CC76C2F4C517EDBE8F8D84C4D76D8
:10DD9000D80C1F4CC34670B83CD80C738C674C57DA
:10DDA000D80C7BC97491704898A828E8381CEA57A9
:10DDB0008CA30568EA274E907BF83CFECFFEBF603F
:10DDC0003D5BCC4B3B4E36682B854044E804D8A8DD
:10DDD000288940BD6C88044408844484608940F8E4
:10DDE000D88C3BD83038E8FD7E0C27D8D57E5848F3
:10DDF0003031E8757A980670389C62CFF613666603
:10DE00003C1EA6067038AE7E1B4E23267038AEE050
:10DE1000DCA05CEE5D7AF237B2EEEE7CD37C0630AD
:10DE20005EA61C6A873C5CB27C0E4EB2EEEE521BC4
:10DE30003CD31CEE25510E917004E6C61CEA4BE063
:10DE400008F174A8E8557E3C305E6A478E8E8CBF20
:10DE5000CC87A3FE97C68C7F4C6FD844CCD3655437
:10DE6000D0F0F9700D7EC6A16C49240C37B8D844A7
:10DE7000D8A8AE6841683B8DE2F174A8E8CC9974EB
:10DE80005D1C0C330498A809B8BC5884983CA87849
:10DE900058EE091E44D5420C676554D0F09888BCF2
:10DEA000983C589974E020F97098BC584C93C1B0D4
:10DEB000BD1C14090D051220010C01120D20534543
:10DEC000441333C17098BC5846F06666FB610098F5
:10DED000DC1044E05830F1CCFF66EB2030264C2BB0
:10DEE00008FD7046CC9F66EB987E4B4C1F482B4834
:10DEF0008C979170A56C6B2020441C583C1C0A49DF
:10DF0000CA30C36A8B2E4C4544000D54654400460C
:10DF100066CC3766EB0D54411C4C5F9C985606301E
:10DF200072665F4CFBD57E8C6B480D7CCB4168BB29
:10DF300098E3970F0E0D0C01514C88C4084860857A
:10DF4000684B2315684389400EDB6631687038E6FC
:10DF5000463C0E8940F9740E630C474C3F8C271CDD
:10DF6000C217D5764C43F8D88C1B58E058AEA8E8B9
:10DF70003038E84C60E00C132049244CA7CC091F32
:10DF80008C8B91704C37D88C53C502603D5BC97443
:10DF9000F90C9170048498A82860A05D1C98CD9E0F
:10DFA00058B8EE514C6C9B385888989CC2285D1C20
:10DFB000089842A84B4D4C38580484D91C783C89A9
:10DFC00040A8FE63084E2B00E080E02E6889CE4C0E
:10DFD000EBA56C33587D6813DBDC90F091708CA757
:10DFE0006148D6F970736576817ED968C97071BA57
:10DFF000D57EE976008B93CBD3DB0003320D14CEB4
:10E000000000000000000000000000000000000010
:10E0100000000000000000000000000004000000FC
:10E0200000006C454C54434D613076314C4C8C4C67
:10E03000C1CC34CAAAF4BD031FC60F60481110003A
:10E0400066C4781400404503401794EB00D4DF28E1
:10E050001B505047BB402060CD3D3930B30FCCDC66
:10E060004B45DA6707C225523BE40D172330723364
:10E07000300173171992E4E3C4793F7D6055402461
:10E08000A348451455922000508E404ADEC7B14245
:10E090007CF45845324211EDE291008482183D62D1
:10E0A0001F2246E435C9C708060B94B8FC3838006F
:10E0B0000400020000C07503700D700EC07999CD88
:10E0C0002144688C43D910FDD3B31F8E505448713E
:10E0D000300DD21847374FA8C3E0129BC4139A489B
:10E0E00043315140140AA790161A425812250507C9
:10E0F00029C05104E961838D01501188137A71564A
:10E100000080008018642B00006242E4C615594864
:10E110001122B05884214406012921804253B16D57
:10E120004D79CC4C3C7220125843C53149500611F0
:10E1300036063D6474670E11D01311F643423C3E1F
:10E140005190798704E5501A90281C3EE16288F4CA
:10E1500054B848C554429F0C0388D434242344F255
:10E1600025D28109C71972A2320444064DC1405D0F
:10E170009C371CB6DD05353DD50E91263405A61C11
:10E18000040000000050AAAA5645851700069754BF
:10E19000CC998911501ED521961D5B33B72DF316EE
:10E1A0003E7719A53409564948885810C210C00452
:10E1B000914520A1BF00E353659537581944293E86
:10E1C000393D501CAA504A92A43442826DD5F227A0
:10E1D0007F17CE091D12C7C44521481C9311EF3388
:10E1E00052043033002134C623334E16DB03830C34
:10E1F0008040CF1708042E12308010011F0004F059
:10E20000005050605B1294719219441A681820E40F
:10E210008111732E51556463F4782414576CF98B73
:10E22000C8843851445398464100C080724C06D18E
:10E2300054587410000004BC600A0664D978675C06
:10E2400015CDD4F479B92790C444030AF5B70B006F
:10E250008419356F23B2967C84E1336A844D124968
:10E26000CD3A57333300601F288AA82014585154E0
:10E2700084469A8F868896862C26A619685C8051DB
:10E280001DA01835109015047F850914C2808618CA
:10E29000554C09EE9F488D763112ED113E24EE4328
:10E2A000DE5422D1C4DD6625291E6D36DF5C0709E8
:10E2B0005684F52F6017F2F3C92F10050EB0E40055
:10E2C000D4644280818877CE08D907773035213AE7
:10E2D0000004744025CA00C000C0003010CE99C5AB
:10E2E00070D4E03F4F1F1610D8239810837030036E
:10E2F0007F3CC745C405403EC11F34DE01F237FCF8
:10E3000065BD1FE556C86AC2BE84C0D5260232204C
:10E31000990FD365550000000000E4DBDF31D55FC5
:10E32000A54E458C539531BEF4617C1C0F553C6362
:10E33000134C7C428772483200D44B0852E8D43BDD
:10E34000858100E561462545102EA32F6192F48753
:10E35000EA0000000000D44C786C333009D95757DC
:10E360009D83357303E17F541319DF2C724270488B
:10E37000F5601CF11D6D0B1ECF01C13581952C522E
:10E3800047828002B226FC5FF03B073FBE930987BD
:10E3900012DA311F4E3030565B05853C8F46104AED
:10E3A00002FCF4B3398AD6461379D53003000088CD
:10E3B00001D5AC4BA6C5F82D15E3B97866D406DCBB
:10E3C000C4805107BE57C0500C94531B0100D56246
:10E3D00081719009D8D108CB7EC0F383013B4738C7
:10E3E00063304C4561FE89344D7D7F24CE57FBE47C
:10E3F0001D40B70D9315ABF6665D665456FC0B8851
:10E4000000F8615044FE1348260E7676B5A3D91C59
:10E4100078D88484D88C1326F046F009C886E64B59
:10E42000309EA62BA058F142CC2766EBA3D91C78CE
:10E4300058203C56069CE21B4EAB3012664761C822
:10E440006686A568E330C4064FC64ED0A646263C75
:10E45000A3E6761C4E906AC6FB303162276A13A68B
:10E4600062AA3C26048C2B08A07E60585D1C98BCD8
:10E470009CE22B0602A2E6C602A23003622F1C42D7
:10E48000136230088C270C237B0C134630555EFC3E
:10E4900006BC30E61BF61B2E03068C2FC16813C387
:10E4A000A60EA05A7C1AFAFAFAFA56233C3AFCEE67
:10E4B0001A46BC26260E55C4604C61008859C8789F
:10E4C00028B86898A859C4EA005ABC1AB0303AE68D
:10E4D0002366DF461AE0BDD065F04C2FA18002DB39
:10E4E000CC3F4E70B8584C7BCC6795A43C0A59A4DD
:10E4F000E5A4D88C1744A180FD188A8514064E70B7
:10E50000CA685878A6C6026A6DCCB05E3C062B5D20
:10E51000C4C830DA7004B07C0E01D0EDA4AE3C6605
:10E520007F7098AE59A48D8CAE7C6606FC5843046F
:10E53000987C1666C3084E70980E78061BA66878FD
:10E540000E59A430C08D8C4DA4468D8C4E587078D9
:10E550000E4C23C4BD8C783C667BEDA4D884D88D4A
:10E560008C29A429A4AE0E584E70780EB8BC5884DD
:10E57000E0DCA0DC1050121C8AE5A43C5CF2CB7EEF
:10E580000F02FF1C8A4DA4EDA47C6A22D398AA69CD
:10E590008C0A588C574DA459A4468D8C980A29A4EE
:10E5A0001B1C6AF5A89B623C5888821B59A4468DA7
:10E5B0008C42D762101C021F023BA666700A4EF006
:10E5C00098AA698C7038989C50F09806467078A686
:10E5D000682E063B6670EEF0EECB4924F85A5EE8F2
:10E5E00030BF2684A80E78AE66CB70380E4670AE6B
:10E5F0003E8B1C8C137CEA330EFDBC95BCB88C1F83
:10E60000884B781C0A29A429A4B8AAA8A1801C397F
:10E6100088E68F0C2F59C4F0000DFC03080B13156E
:10E620000DD9FED5883E434670AA680A4DA4E5A4DC
:10E63000AA704670785816468386FDBCEE4B66B8C5
:10E64000FCEE0825AC1B95BC780EE3D1486E2B5927
:10E65000C42E1659C41916D1486ECFA3D1489D486F
:10E66000FE738BD1486E4BBBD1486E439D48FE2351
:10E67000FBD148CB4E3E304C0EB87E5B81C806784D
:10E680003C06B9586E63AE6E7F3A3A3A3A3C7038FF
:10E690000E8E844E70F8E030546E9B305A6E736666
:10E6A0006E53666E33B5A20EA04E3E7EC37E7EA034
:10E6B0007ECE7E574E43EEA0663346F6A0BEE04EB9
:10E6C0005EE76EE0CE7E1B5EE0E0DCA0DC5EEE1F6F
:10E6D000237CF2F3AE5EEE1F237CF2F30E03E0A583
:10E6E000CCBC0E4670AE6881F04E70789A66AE680B
:10E6F000304070AEF03E55F04E7084B07E7E7E2F7E
:10E700007E89F68801C8E6B5A286B0668DC61C066D
:10E71000A54FC678A6063DC358B0FC06707C26E619
:10E72000F002223DD0AED8E63C7006023DD0B0E605
:10E730000CC38604304006A5D00C49D1C676431CD4
:10E740000A6AA5D049D066B0E6C67038A670A6F0B1
:10E75000986666776651ECA606704EF09866BF8D97
:10E76000C68451EC8C276688D326E67022FC06020C
:10E770003DD0A658B026E6FC063DD098BCA6588CE5
:10E78000A3BA44DDD47AFA9A983C0698767FA60616
:10E79000BF0DFC060C2013091A05D9FEA5D00C9755
:10E7A00098762BA5D00C5F98E63CA6B0FC707CF068
:10E7B0005DC40A3EE6B006A63CA60667BC704E7075
:10E7C000F8FE2F66A6067038EE472DD0983C66AF4F
:10E7D000BB0000000000000000000000000000007E
:10E7E0000000000000000000000000000000000029
:10E7F0000000000000000000000000000000000019
:10E800009CC2FFCC574626FBCC2F5DC4243C71CC68
:10E810006653309066FBC8CC6100839C4262E2A5DF
:10E82000684E9C90CC5F601B7A1F7ACB5DC4E01071
:10E8300071CC664FA5689C228859C87BA568D91CF5
:10E8400078583012662761C8CB30C266AF46F08C6C
:10E850005B59C8BDCC66E627652073BCF05DC42952
:10E860003C26662F8865C82B49F08804E9D48C2B98
:10E870005DC47E3E4E70088C2B4540061BF9C430AB
:10E8800018A6C6B07CEEBCA686A6061F04A666988F
:10E890003CC658B03C0671D84E70B87CD8040C13F6
:10E8A00008D8BCA898668DC77C0EEDA4E601D0AE52
:10E8B0003C58C69C584E7051B41C53BDD0C1D85E54
:10E8C0003E2DE0DDFCB1C0BDD04C1BE9D071F0B0F5
:10E8D000FC700602385AF051FCAAAE3C58C9C099E7
:10E8E000C0980A01D098AA0A5841C480E68741C45A
:10E8F0004C5780E6AB708D8C987C0EB004D88C138E
:10E9000008D826CABFAE3C580AB066577001D0413D
:10E91000C4808D8CAB0C2341C4804B081304980A2F
:10E9200030FF8D8CA156C1D8BDD04CD9C85E7E7E3B
:10E93000FE39E098EEB5F604DCD01EB07E7E2F08DE
:10E940007E29E331F40C533E85E0B05E3E7095F0D5
:10E9500059C0B0CE46CE6E6E68BDD071F04E7078A4
:10E9600058B0FC060201D0EDA48A0456705C0A0679
:10E9700076265766D88C1B086AD86A6A98AACAE7AE
:10E98000AA581C4699C4B0A1C46AB0664F7001D0A1
:10E99000EDA4A1C4B30C7B46A1C45B0830FF99C4AD
:10E9A000640530FFA1C469D095DC0C554AF9FA38EA
:10E9B000BCA6BC288804E9D48C434E30913CEEE9D7
:10E9C0005ACEBC06B07CC698BC1ABCEE4E70385C01
:10E9D000AA581C06BC065F3C0EEDA459A4E6AEBCCA
:10E9E0000EEDA4AE5884C61C6A17881C987C66E697
:10E9F0001F8CAF8CFBFC580A01D098AABCDBE156F7
:10EA00003BB03C263C463C7098E63C0AEDD02E8458
:10EA100049D463BC6658CEFC0A01D0B07C263C7059
:10EA2000983CAA7C5806D3B0FC707CF05DC45E3F75
:10EA30007E2F06ABF0837E7E89F788480DD4CE58B2
:10EA40004E70F80E8C2BEEC3F9FA3DD00698BC063A
:10EA50007F0DFC050E04200F0620120503F1FE6653
:10EA6000B03C065DD8554AA5CC06BCA63CF081F06A
:10EA7000D5CC663002C61306F5C459C42E12000068
:10EA80000000000000000000000000000000000086
:10EA90000000000000000000000000000000000076
:10EAA0000000000000000000000000000000000066
:10EAB0000000000000000000000000000000000056
:10EAC0000000000000000000000000000000000046
:10EAD0000000000000000000000000000000000036
:10EAE0000000000000000000000000000000000026
:10EAF0000000000000000000000000000000000016
:10EB00000000000000000000000000000000000005
:10EB100000000000000000000000000000000000F5
:10EB200000000000000000000000000000000000E5
:10EB300000000000000000000000000000000000D5
:10EB400000000000000000000000000000000000C5
:10EB500000000000000000000000000000000000B5
:10EB600000000000000000000000000000000000A5
:10EB70000000000000000000000000000000000095
:10EB80000000000000000000000000000000000085
:10EB90000000000000000000000000000000000075
:10EBA0000000000000000000000000000000000065
:10EBB0000000000000000000000000000000000055
:10EBC0000000000000000000000000000000000045
:10EBD0000000000000000000000000000000000035
:10EBE0000000000000000000000000000000000025
:10EBF0000000000000000000000000000000000015
:10EC000081C8E6B5A2064540B9CCA6BCA63CF048F2
:10EC100085F08C5BB0FC2670381CEE77709BD5CCF1
:10EC2000A04E70EE59C4EA003CEAF30E4E70AE6896
:10EC3000B01E4E3E1CBEBE33501050903B10BE2B3B
:10EC400010105003BE2B5050D0D3B046FC06F5C474
:10EC5000A3F85E5AE8A878E630C0062663A60670D8
:10EC6000383E334E7EF066A3A1803CD5883E7B7053
:10EC7000AE0E584DA459A4468D8C980EB0E66F7018
:10EC80005DC414218A4E6E56DC90688DB8BC08981D
:10EC90003C28441C6A8AEDA45606303A067B303084
:10ECA00006AF3020469C58DD201C6A4E30056A5B5A
:10ECB00059A46A4C8FEB48783A87783A8DC7B83CAC
:10ECC000D808D87CA88CB5515DC4333B3045663F2D
:10ECD000783A27301B83302B66832666378C7F304B
:10ECE0001A23266627301CD32666678C9F4C435315
:10ECF000F8EECE71C8700439D006B0BCA6700839E1
:10ED0000D0E6172606B0BCA670783C06B03C063CA0
:10ED100006B958BCB95826703C063CE64EA670A60B
:10ED2000F0B02606C78DC60E66176629C6BC069CBF
:10ED3000E2D330901C02AB30316A8B30460217664A
:10ED40009C024B501C62276A136AA6A606C6E6A25E
:10ED5000065E233008465DC46A27F9C40C2F70157F
:10ED6000C8E68DC606F8FEB0C6FB46DE1BA6C6A6E4
:10ED70007079C4AA58B0665F701C980AEDA49C58BC
:10ED8000461C8D8C51B47B4E1C10CC2F6EEB4E4B21
:10ED9000203C56069CE21B4E5330C4064FC64ED054
:10EDA000A646263CA3E6761C4E906AC6FB3031622E
:10EDB000276A13A662AA3C26EE61005DC42E1230BB
:10EDC000FF06F8BC66470EB8A6AEA88DC6B8BC66EE
:10EDD000B5A3840895D0302B06B006273C061B81CE
:10EDE0000A06B8BC13EEA6F30EB03CE630A8AEEEB1
:10EDF000176668A69C583508B0063C260677BC7096
:10EE0000783BF87EFE5F5C10EEAB1C7CEAF33C3393
:10EE100015C83C9C4A7079C40C2F8AB058EDA4AE3A
:10EE2000D87C1C846A1788D8AE987CEA1F8CBF4EA9
:10EE300030051C6A538C2F6A59A40359A4034E70E1
:10EE400030913CEE3B79C46DCCF5C459C4EA00BDA9
:10EE5000E0DC101E46FCBE77E6A670066638EE7053
:10EE600066EEF0BEAB5DC4EE00307A66FB61027800
:10EE7000E8380E38D81CAA28E09CA01C380EF8AA46
:10EE80007CE8AE7C280EE0D4948DC7A0EA73E267DC
:10EE90009846AE283B48084EDDE04E300BAAA0FA5B
:10EEA00060E6133AA6CB3C30030E51C45DC42E126B
:10EEB000B87CD83C30300693302E66370C60A6A65E
:10EEC000E0300D664F302D06E0303A066061DAB171
:10EED000D0AE0E3CEECEFCEA6DCC666686664E3059
:10EEE00007A63AC6F346703CEEBCC66804044CE183
:10EEF000C4E9D00881F08C4BB07EFEA1C3A1F4839D
:10EF00004E70780666263DC2EE4E9CCA1C3E70AE20
:10EF10003C06027098F00DD0A60670B0F07A4670EC
:10EF2000CEAA7C0EE5A4E6AEBC0E01D0C68D8CB098
:10EF3000A626A67A2770AE5B7001D0B08D8C0DD05E
:10EF4000A6704E6EF05DC4F000492438FC7006389F
:10EF5000FCA67C70E04670387CAA0A3C28E00404D9
:10EF600084E9D4983C1C0A0451FC4A2A2AE0306007
:10EF70000698467004261C7C4A300AFC58B8A6A89D
:10EF8000E0D91C78D8E0EDA40616D91C303A6643C7
:10EF9000302C6623302E6661DAE0B1D08E0441A4B5
:10EFA00044CE0637662FA20217484ECA686A054645
:10EFB0000000000000000000000000000000000051
:10EFC0000000000000000000000000000000000041
:10EFD0000000000000000000000000000000000031
:10EFE0000000000000000000000000000000000021
:10EFF0000000000000000000000000000000000011
:10F0000088DCD0FE95E84E705C380AB0AA2845D856
:10F010001388D91C78468C1326F0256C88080404C4
:10F02000E9D40C5B44DDD4CE7C06463BA6265DD8F5
:10F03000705B7C0A556CB03C46BC70C57E256C0488
:10F040004670387C1C0AEDA4563CAA7CEE3BCEFCF4
:10F050001C0A556CDABC06B07C063B86BC065DD843
:10F0600070DA7CE6917AAE4670CE68C1B0E0B07CD2
:10F0700006300B0697300D46DA7C06333017C63E55
:10F080009306301806BBB03C061EA114F87E7E9E87
:10F09000066646F098A6581CB07C26E6CE7C0A048C
:10F0A000EDD098E67CAAFC58CE7C0AEDD098AA5800
:10F0B000CE7C0AD9D0DC101E9E9E1C98AA5804084B
:10F0C00093EDA48A06D91C79B01CCCE746F06A01FE
:10F0D000D0987C6A6F98DE586A8744D91C987E2F36
:10F0E000581EA9763020E805768A48196C4479B014
:10F0F00098DE1EFCDC901E1F5E1BBE5E3C5883ED3E
:10F10000A48A06D91CCC33D9B008357679B01C6AEC
:10F1100046F001D0986A63DE3FFCFE9B0C8BFEDE5E
:10F1200004F3D91C0CE37E9EBEC7F8BEF3A3D91C22
:10F13000B8F8568A063040C64B46F06A196C1B79FF
:10F14000B0980C37FC1E9E3C1E3C9CE2042030F024
:10F15000E6E09CA0443020CC697766E3C666797708
:10F16000E699C8D91C9C6282B8A2F34C1B98F3069E
:10F17000E094339C98A60658A0D88444D84C77C60F
:10F18000A69C58301F6617260698069CE8D09C025D
:10F1900082B8A2F34C5177485576203CF64BA568CF
:10F1A000711C5DC4E01078581A7A7A4E203C5A1CC3
:10F1B0005D001AE000105B504B903BF3D023000041
:10F1C000103C56063044668F788C1B84138884D894
:10F1D000F0A5680C6973517626669FB07C06668C34
:10F1E00023300B4686BC0646F05DD8C97A26667782
:10F1F000B07C0646268C1B300CC653064349247847
:10F20000FC5CEAEE9C300842A17CF6DD7B30088C89
:10F210001F4200957C068C47C1681BC17A7C5898B8
:10F22000A6588CBB796C4A57C1B0BD1C0E0F20127A
:10F230000F0F0DDDAC78D884D8F049246D586100EB
:10F2400030FF66675ACCE3203C0630C366DD7A693E
:10F250007288489806C96C25E8E3CEBC06B07C6687
:10F260002326E6CEFC1C0A04EDD0988D8C0666861B
:10F27000B03C0671D8C97A3008957CE6EFDABC0656
:10F280001C3001667FE6CEFC0AEDD030608D8CB07C
:10F290003C9D7EB07C667766C6E6A658BC065DD807
:10F2A0007C26E633C626E6A658CEFC0A04EDD098A6
:10F2B0003CAA7C58066611F4D3F6278C557B1C06B5
:10F2C000300825400E7E9B9A0507088700D36B3BCC
:10F2D000E3FBEBD323DBB17E75F44670387C0AED9B
:10F2E000A4567626A3617E056C8C1B8413883D761C
:10F2F0006520056C8498F0A568F572796C0AA17B8D
:10F30000B96CB0684829E84670787083BB843BFBD1
:10F31000796C0A5788CEFC0AD9D0B03C26BC70ED77
:10F32000A456768CEBE6556CC6263FAA7C5CCAEEEA
:10F3300083B96CB0FC5CEAC41C59E8056C8498F095
:10F3400046F01B056C8C1B84138898F0C97AB03C7E
:10F35000E6C17A6606265DD8056C8498F0A56869D2
:10F3600072267F556CB03C06265DD80B4666E68853
:10F3700059C804C1B0BD1C07140F201E7E7EC63CB8
:10F3800030033E1B30017EFCE8BEB3DDAC0C3B46D7
:10F39000F0C6E10803A5684E5C10901ACC4F26EB2E
:10F3A00099C8BACB7976300B01ECC3847434857577
:10F3B00035867636370023363636363636363636A6
:10F3C0005B65209300000000E080E006C61C224739
:10F3D0001C8622279C860882CD7EC61C222B1C22DE
:10F3E000DD7B02A29F8C174230555EFC06BC30E0EC
:10F3F000000005CAF3EBE3DBD3CBC303180D14679E
:10F40000308AA630BD8B72201165E34F0B1D10238F
:10F4100050C604A89C60C74C81496A521BF515F37D
:10F4200014124485B60825C6205B15EBA2262A0ACD
:10F43000400C50AD3C362203820F003532388184B7
:10F44000D80400CCC040819010038074D184F5B002
:10F450004DC000A409302333CC5068BB881F88FB03
:10F460000D8C8C84D4CC0035C0A803033C3181863C
:10F4700021F25B38338A1CC3A1362321B22485E8EC
:10F480002ECD8843480C08000638622380C71082BE
:10F49000B02066CDC040FD657EFDF5E6D61831D1C1
:10F4A00018C0A82221727CBCEF43E2F030E363BBBA
:10F4B000EF0C2320EC20ECFF10A2A0802122282AB0
:10F4C0008221C0C3953C412282101102821108CCD6
:10F4D00004002088310089FD0CCF0B1042084991AF
:10F4E0009D3055C3080018E00D7800880350F08166
:10F4F00034242AF102000000000000000000000097
:10F50000C9E0331053FE72482113E20331158A35E6
:10F510001D23C6B0CB28320EF88A423203980C4025
:10F52000102131411204B81BCE392500C520F0044A
:10F5300052D9C408182044D915449146A603153D54
:10F540006D50210009076954011693A150421A4ACF
:10F550001B050452C7AC8EA0418010409A4F5D112C
:10F56000040481004227644114441785A2244348BF
:10F5700061542468441EC98009CD33A1DC50106A4F
:10F58000821041C1B30601194525880333D6404393
:10F59000482331E50800000610D014294304310047
:10F5A000000000000000000000000000000000005B
:10F5B000000000000000000000000000000000004B
:10F5C000000000000000000000000000000000003B
:10F5D000000000000000000000000000000000002B
:10F5E000000000000000000000000000000000001B
:10F5F000000000000000000000000000000000000B
:10F600002134432432A02C3222037A488414111767
:10F61000C54108160E3BD19008DA2308D40C50B827
:10F620000320AAC428201417170E003183AAAE7332
:10F630007F3703F17A18EB40E8C42EE340E044E062
:10F6400088114C2046211420D24F22D41E7F7C8C5E
:10F650003FCF143D4D34004238019D1008E1503237
:10F660000030344E4207C404A89C60C74C81C84097
:10F6700045D3F0D0801231CC44D401412433841BD3
:10F680008E32F62E61200609FD73B40CC10CF38C8A
:10F690002108C44098186081620F848B9EC008279F
:10F6A00008C70FEEC5174060865D2403B731315C93
:10F6B000C744C7CB50005044642384930C32E88C79
:10F6C000683D00088509240A6002040084C0000027
:10F6D000880E841800A3512E4891801E8508048945
:10F6E0004F2F313131B13C1432C3085200000000B9
:10F6F000000000000000000000000000000000000A
:10F700000B801A2838215A84720934015C0504954B
:10F710006824000054180D059034E248C5443411A3
:10F72000140F3113C411249811405844587841C41F
:10F73000084D700CC447E3244571A11991368087A8
:10F74000D0CC54010C8D2B033B0371330F45304655
:10F7500034D6061D20F4E668C8003744C8516C4B07
:10F760004C8C214BDD14E55131D0141E6300C000D8
:10F770004931CDEC56540E954414C339144A34879C
:10F78000064767C5C435C67D44753300E0B41B2306
:10F790002DBC141F595580D10A901110105C9C612A
:10F7A000C4004500148D4105090941465124C9444E
:10F7B0007155591055508296A0968978626E514DB8
:10F7C00085094A4DF5430186E051080816C68CB1FB
:10F7D0009C01B0079E01E6167941C088F20C200515
:10F7E00021A1F70C331654E3D21600000090AAAA08
:10F7F000884077282F3FC5A2474B85F630FF3F88CA
:10F8000000000000010000000200000003000100F1
:10F8100005000100050101000800020109000201C4
:10F82000090102010A0000020B0000030C000004A1
:10F830000D0000050E0000060F0000060A0000077C
:10F840000B0000080C000009584E55543020005899
:10F850004E5554312000584E5554322000435846DE
:10F86000554E300054494D45522000435846554EA0
:10F8700031004164764C31200041647655312000DE
:10F88000416476553220004D6174683144005374F0
:10F89000617431420046696E616E63005A656E7232
:10F8A0006F6D005050434C20520050504355205231
:10F8B00000436972637569005374616E6461004747
:06F8C000616D657331006B
:10F8C600414C504841005052474D00534849465418
:10F8D60000524144005553455200444547001A1B07
:10F8E6001B1B1B1B1B1B1B1B1B1B1B1B1B1B1B1B62
:10F8F6001B1B1B1B1B1B1B1B1B1B1B1B19007C2009
:10F906004275696C742062793A204D652120202069
:10F916002020202020202020202020207C007C2049
:10F92600496620666F756E643A20696E666F407030
:10F93600617865722E6E6574202020207C00171B6E
:10F946001B1B1B1B1B1B1B1B1B1B1B1B1B1B1B1B01
:10F956001B1B1B1B1B1B1B1B1B1B1B1B18004255AE
:10F96600494C543A204E6F762031312032303235B0
:10F976002031373A35373A3139005645523A203038
:10F986002E393035004A414E00464542004D41521F
:10F9960000415052004D4159004A554E004A554CBF
:10F9A6000041554700534550004F4354004E4F56B3
:10F9B600004445430053554E004D4F4E00545545A7
:10F9C6000057454400544855004652490053415497
:10F9D600004D454E552000444953502000424545B0
:10F9E600502000434F4D20200053504545440049C8
:10F9F6004E464F2000534C4545500056494557202A
:10FA0600004D4F52452000524547532000464C4179
:10FA16004753004D4F445320004144562020005286
:10FA26004F4D532000434F4E462000532E494D471D
:10FA36000052414D20200050524F47200053495A52
:10FA4600453A0052414D204D6400202D2D2D2D208C
:10FA5600002D20202D20202D00726573746F726991
:10FA66006E672E2E2E0052756E20204379636C65CC
:10FA7600733A0044697370204379636C65733A0086
:10FA86004B657920204379636C65733A004465625F
:10FA96006F756E636520542E3A00426174742E2091
:10FAA600456D7074793A0050582D34314358004EE4
:10FAB600414D452020506720426B2047700042414F
:10FAC600543A00534E3A00020C010E0B00444953BF
:10FAD600500A00454F460A0057616974696E6720EF
:10FAE600666F7220646174612E2E2E0A004F4B0AD7
:10FAF60000505834310A0052414D0A004552524FC7
:10FB0600520A0044495350004245455000434F4D68
:10FB160000535045454400494E464F005649455707
:10FB2600004D4F524500534C4545500052544E002F
:10FB3600455849540044554D50004C4F4144000926
:10FB4600204F4E0009204F464600384D485A003196
:10FB5600364D485A0032344D485A0033324D485AD1
:10FB660000314D494E00324D494E00344D494E004C
:10FB76004E455645520058595A5400584100585956
:10FB86000058005245475300464C414753004E45E6
:10FB960058540050524556004D4F445300502E3095
:10FBA6002D3700502E382D46004144560055500042
:10FBB600444F574E00494E430044454300005447C6
:10FBC6004C00524F4D530041444400454A4543546E
:10FBD60000434F4E4600532E494D47004F4E004FAF
:10FBE60046460052455345540052414D0045784D16
:10FBF600454D0052616D4D640050524F4700314CE7
:10FC0600494E4500344C494E45003120534543008A
:06FC1600322053454300BB
:020000021000EC
:100000001640008F00A60299009E026600950247E6
:1000100003370309031E032602EC02F90451052FDE
:100020000557056A0577050C059104800485048A47
:10003000048F05B104630456045C046A047705A5C3
:10004000059A05D205A005C204E70504051204BE01
:1000500004C904A904DF04D004D7051604B0049E23
:10006000049704B704EF05CA054605290522054F84
:10007000056405710583058A05BA05360608066319
:1000800003B400008220160E0F03201604012DE099
:100090008E091805084830088B8E0914030F300F9D
:1000A000438E090E0902300244E6B83C5804CC1FC6
:1000B0008C2BC4840C5F04C1B0301F682668C668EE
:1000C0001E2B6520610049244E00309D3CFA7EB80D
:1000D0003C98FC6D1C3C587EFA7A6F605B0C2F08D4
:1000E0006B0B133C7A17FCCC8B0C67793C2E3812C7
:1000F000C6C3837711C08070301084743485753521
:100100008676363700E3E323DB53B300C3666666C7
:100110006666666666666666666666661B693CACAB
:100120004CE733FB300A06B34CA7DB5E23793CDE99
:100130002146A3B87CD84C1B441348D83CA8A34CF8
:10014000EF8B4C1B446B485B5E2F6100410EE0D986
:100150001CB8E6F8302006A8B8B856A66617B8A6A8
:10016000E826E8C6E8BE5E2B6D8CDF005D1C3C58BF
:10017000200BE066D91CB8569C5806E223E2E20642
:10018000A2263B66F8693C2403DC904C1B7E7E066D
:100190007E9BFEB806B8300A664623302F0626E856
:1001A0007E3E23C666E8E6E89C98E8EB5E6BD91CC9
:1001B000B8E63020E86606B8B8B8566613F866A602
:1001C000E8E6E84924793CC8B01A5A300CBC1A70E9
:1001D0008DBCF10E8498A8793CDE5D1C1106E0D937
:1001E0001C0EB89CE2337E7E4C137E7E302FE81CC2
:1001F00022A6F8B0E21B62DFA0FCCAF61F226656F8
:100200005ABCBADEFA7EF35AF8B0E2736263601E3B
:100210003009065C422FFAA6E30E6EC1B04924B83D
:100220003CD808D87CA8208CB55188EEE8E04E2058
:100230003C063018BC1AB0303AE62366DF061AE0F6
:1002400097050916180508F8AE6D8CDF8C3008008C
:10025000E66D8CDF3A5C005AD070088DBCF10E97C9
:1002600005091614030FF8AE6D8CDF8CAE0E9C00E2
:10027000E21B8902DCE2E7E2D7E05CA01C4EA202AE
:10028000E2EEEEEE3CBAF2BAA2DCD493300FE669AD
:100290003C51970509160E0902F8AE6D8CDF8C4EA5
:1002A00000BA1A3CFA1B8902E6EFE6DFE05CA01C0C
:1002B000BAF2F2F2BA42421322A2DCD4A33002E62E
:1002C000693C51B8AE6D8CDF8CAE00F06D8CDFE711
:1002D000A600F0EE3004EE465BCE1C58DC9886C3D8
:1002E000EE66F3BC463CE09918140F12793CC370DB
:1002F000793C43B0CBBF140902793CC33CD88C276E
:10030000D8B95AD8655A840E01793C43B0BC463CF2
:10031000BA6D8CDF6C6E008C9102A902920F793C51
:1003200043705B920F18793C4358AEB0D8AEAEB074
:10033000AED870D3940F0EF888AE6D8CDF8CBA00F7
:10034000BA005BF88458B8AE6D8CDF8CAE00D8AEC6
:100350006D8CDF8CD800E00B00A188C1B080B0307C
:10036000063000E6465D003CA6BC300656A87A562C
:10037000D3492408000170ED8A0B00C1020B00B9BB
:100380004A0B0089520B00B5A20B0089020B001921
:100390005A0B00810A0B0009828814010D201604F3
:1003A000012DE08D1614201604012DE00B00A1880C
:1003B00080E00440CC00F3004D50A631F27F3A6952
:1003C000111B1342A631F27F3D85C2032F0270C676
:1003D00000F600534952544EA605C8012F0470C6BA
:1003E00000F400535A3FF653495A453E3DA631A802
:1003F0001997738B9BF37585C8032F0000000000CD
:10040000050E04200F062001121201190E0F1420F0
:10041000011212011920060C0E010D052005121201
:100420000F120E0F20120F0F0D04090D20051212CE
:100430000F120E0F20182D0D050D0F1219150E0499
:1004400005062001121201199812140D201604013C
:100450002DE0AB14010D4EABAD14010D308073AA2D
:1004600014010D30203BAF14010D30A0D8793CD9D8
:10047000038D090414010DF86150753CD6CFAB090A
:100480003016F3AD093056CBAB0A3036A3AD0A3087
:10049000767B810A09130D30053B8A09130D301153
:1004A00058F86150EB8A09120D3013ABAB03130DF2
:1004B000301273AB12130D30323BAB03120D30927E
:1004C00058753CD606AD03120D30D2ABAB12120DEF
:1004D00030B273AD12120D30F23B810A09120D30A9
:1004E00007FB85160F0D0DC4483B900117130DC473
:1004F0008808F86150B80E785150753CD697BF0502
:100500000D010E0D793CDF22BF0D0904793CD62286
:10051000920DC433930DC4608848793CDFD0BF127C
:100520003E12C448C3923E3C12C493833E3C03C473
:10053000085B832B0319B86150C40888F8615075B3
:100540003CE5CE96091008048B820118010D1204B7
:1005500043820118010D030808844884F86150EBB8
:100560008D120E1204338D120E0308846B8D151339
:100570001204338D1513030888448404753CDFF19D
:100580008D1513883B82010D151384843B8D120E4B
:1005900006888844A3820118010D84845B8E090DAE
:1005A000882B98010D8488480804793CDF428D2A05
:1005B0000D793CE56793100E1214793CDF49960ED5
:1005C000090D793CE5259319130D793CE5EA94056D
:1005D000040D793CE58EB030CBB030F6F6366BB01A
:1005E00030F636F63BB030F636F636F61336F613FE
:1005F000363A70DADADA3ABC80E000000000000037
:100600000000000000000D50CA00F6004D454449AE
:1006100054A81B10A5AFCF66A90AA819A5AEAB199F
:10062000B6B2018BA5A8AC0AB6AA87A5BFA5A59BA3
:1006300073AC08B997F27F3FA9178EA5A57179A56C
:10064000AC9A73AC17A5AC0AA596B12A09A8157E79
:10065000BA0BCF6F06AC071DF34D5452A5A4C40CC2
:100660002F1F10C401F700434D45444954A81B07F0
:10067000A906A59283F74E4F542043505868124B59
:10068000638E75691A10101245A806AC06B1874B27
:1006900067B1838EB72701A90A73CF661242111A78
:1006A00010101141A819A5AEAB19D07D8F02AC0A6C
:1006B000D0778FE06683F352452EA5BFA5A59B7327
:1006C000AC08B994F27F3F8EA5ACAC06B98AA5966A
:1006D000A594A5ACA597A59509A815AC087EE03B07
:1006E00083F3494D2EA5BFA594A5A59B73AC08BA6D
:1006F00091F27F3F8EA5B0AC06BB8FA59554A5ADFA
:10070000BB880A7EA596AC06B25D0BAC0AD01A8FE8
:10071000AD06A596AD09A595B26D04A5A8111A1050
:10072000101140124385CF6FCF0FAC071DF34D540E
:1007300052A5A4CA1D2F2150CA00F6004D415452A3
:100740005801A902A81BF5524C2043588ECF68CF00
:1007500069CF6AB114CF67A802CF66F74F524445FC
:10076000523D3F8E616883AC024030511140A6215A
:10077000AB198E2083F152111B1C134240A59DC260
:100780000AF4004D5452CF6F02A908A907A815A872
:100790001BFC2041204920445420422053458EB266
:1007A0001904F152A5A0F44445543D9B737EB22830
:1007B000CF7BA808CF66F152BFB9CF67F152A5A28F
:1007C000B23ACF68AD02B4279F00B244CF6AE02DA1
:1007D000829A73F2522C9B73A5B2B254CF7CF15221
:1007E000AC029F00AD02A5BBB262CF7EA808CF6964
:1007F000E00B820FA807AC02A5BEA5BD03F152A570
:10080000926883511140A63175A819A59DAA198532
:1008100074401140A6218ED0926FC2162F3D30C079
:1008200001F4005A5E4E8030754F205371204271A2
:10083000054E01AC0485A815F2553D9B737EF2561A
:100840003D9B727E85C605F5004D41475A4FA81560
:10085000F2523D9B73AD047E85CC02F400655E5A76
:1008600081554E80B134CC01F4004C4E5A814F502A
:1008700080B141CC01F6005A5E312F4E8030131604
:1008800010714331754F20686053712068437104C3
:10089000E061049700B28185024F71214071B4116B
:1008A000C606F50053494E5A81325A7133E04C8ADC
:1008B00042225923E0518B4280B100CC03F5004322
:1008C0004F535A8132597133E0318A4254225A23AC
:1008D000E0358B4280B100C004F50054414E5A818E
:1008E0001242325A71124233E01D8B4023E00C8ACF
:1008F0007143762259714380B1000B83835871553F
:1009000043715840BD850C558360400D124385C02E
:1009100008F400615E5A7532717450427622421DAD
:10092000F3655E5AC003F5004C4F475A5034758149
:100930004F5024957195727580B100C403F6005A2A
:100940005E312F57327533753151713051402071FE
:100950004354762171432322C204F4005A5E578126
:100960004F504F75754F7175427540744E554E809E
:10097000B100CA03F300432B71067540754074B192
:1009800000C202F300432D547154B613C801F500A0
:1009900043494E56E00482B100034F607154714EDA
:1009A00085C003F300432A4F75754F757571754205
:1009B0007540744EB100C003F300432FE024021DC4
:1009C000F2432ACC012F5B70C600F400504C591240
:1009D00013A621AB198ECF6AF84445475245453DD1
:1009E0003F8E1245D00F6A71121146D0166A71A857
:1009F00000A903A905A9069116911506E04B8C974D
:100A000015B608E0448CCF6FA815A81BFC465820EB
:100A10005254202020204E45578ED0156FCF66A906
:100A200006901691157183838397159096AC059562
:100A30007342E1E18E9073909642AD0571F4463CAD
:100A4000583EE18B8FD0406F0DF1619015A631F3C8
:100A50007F3D3F778E919585CF67A619D0576FC898
:100A600015F40052545312141A11AC069117AC0528
:100A7000BB9390161141911590960C95959715BCC6
:100A8000079500A8050B2036213722382339243A50
:100A90009016121040A819AE73F34E3E358E85CFD6
:100AA0001911101A10101691149115E12E902DE0C5
:100AB000DC842A11E17191E16E91E16B91E1689121
:100AC000CF18289112543827911129911342269159
:100AD0001014424137901214429013514190104229
:100AE0009011514136A900E06397AA038503AA0239
:100AF000B1882D29453D2D2A453D0190133C129585
:100B00000C950D2D51901041661000111B1C1845BD
:100B1000E0358675523F2C2D4290111243416711EA
:100B20008361433E2C519012412D12424052940E4B
:100B3000A800E00287082C2E543E40372D2F543F4A
:100B40004036E02796850771777185CF17181A1000
:100B5000101691149115E08390AC03852DAC00E044
:100B60002C842811E0C191E0BE91CF162754124386
:100B7000838351264166B1A2524039AC00E00E8415
:100B80007476413AAC00E00584A9028505F4524F21
:100B90004F54E03B8F77E02C8D850154523B742BF2
:100BA00054AC00E00586A802850774F155E0208F5B
:100BB00074F156E01A8F74F155E0148F74F156E019
:100BC0000E8F850EAD068591979617917385CF0F81
:100BD000E00E0DF27F3D9B737E85CF10103D268386
:100BE0006167B4D0433E7690956140566811405796
:100BF0001146713C0A1110950C2E543E092D2D2CD6
:100C00002E42403D78858383E00B8E67852E4266B9
:100C1000B916BA200F909540429715BF099095409C
:100C2000901491157585CF119715012D424090951F
:100C30007191958504A803103D27362837E0D41616
:100C4000B300C0452F2320C201F600444946455158
:100C500019A621AB198EA815F54E414D453F8C8E36
:100C60009A07F74F524445523D3F8B8EA901977327
:100C7000A801FB535445502053495A453D3F8E121D
:100C80004331F458303D3F8E32F459303D3F8E337E
:100C9000AC01E02D800A2322E0958135E06B84369B
:100CA000E06784920683402340222183403440E061
:100CB0007E81254026834040134324E05482BA2B92
:100CC00001F559302E3D3F8E340B242322E0608104
:100CD000353021E0498636302120244025E0448506
:100CE0009206834030218340E034862683404025AD
:100CF000401343244034762625401343402183404B
:100D0000354276E00C82BB3F052340222140B29E53
:100D10000392027192038F980298037F8507202423
:100D2000402006124324407442234022744002AE05
:100D300087082142CC212F3A50CA00F3005643A91C
:100D400004CF6FA815A81BFC4450204350200D2051
:100D50004D2055568EA627D0176FCF7EA62DF16455
:100D6000CF14F27F3D9B737ED0286FCF7DA62FCF0F
:100D700068A62CF10DD01614CF6BA62AD03C6FCFED
:100D80007BA629D0068FCF7CA628CF0FAC04D04EEF
:100D90006FCF7FF2583D9B737EF2593D9B727EF27E
:100DA0005A3D9B717ED0656FCC0FF60043524F5376
:100DB0005383CE023042CE022342CE01947171940D
:100DC0000342742042234121744190712241CE712B
:100DD000A62785CF67A623D04E0FCF6DA624D09E21
:100DE0006FC208F300565361686877139474967461
:100DF0000F7591F496740F7591F496740F7591F4C4
:100E0000757585CF6EA625D07E0FCC05F3005652A2
:100E1000686175A627741342134090F3977290F29D
:100E2000977190F185CF66A626F3444F54D0CE1427
:100E3000C605F400444F54214271224240712342BE
:100E40004085CF6AA62BD0BD0FCF69A62B74F14D7C
:100E5000D0F114C005F30056453175327533757500
:100E600085C002F300562D1C11A62EC601F30056B4
:100E70002B920175920275920323222185C802F4F8
:100E800000565859CE0175CE0275CE03757585C8CA
:100E900002F30055564F90714F917077114ECE70FE
:100EA000754E85CC02F300560DA62BA62AA62BA6BE
:100EB000265D85C402F3005644A628A62B7485CA75
:100EC00001F300562A9470947142C8012F2030C05B
:100ED00001F30054521117A621AB198ECF6AA91B3A
:100EE000FA5A302C59302C5830203F8E13A62477D4
:100EF000F5524F540D3F8EA90567B198A805911082
:100F00007311CE71F7632C622C61203F8EA62B12D9
:100F1000A624CF6F01A81BA815A901FC5E4E205E78
:100F20004F202020204E45578EB117CF7DA622CFCF
:100F300066A801A630D008FFCF67A901A630CF7FF1
:100F4000F2583D9B737EF2593D9B727EF25A3D9B57
:100F5000717EB140C013F3004354AD01B38813A6B2
:100F600025A628AD058503AD05B2B611A62412A6A7
:100F700025A6239010AD015459A62E1130A6259018
:100F8000105A9300A62EA62914A62412A62511A64F
:100F900025A6269400A62A20A62E14E00783AC01DD
:100FA00085021304A625A629C00C2F00000000000E
:100FB0000000000000000000000000000000000031
:100FC0000000000000000000000000000000000021
:100FD0000000000000000000000000000000000011
:100FE0000000000000000000000000000000000001
:100FF0000B00D19E000000CBC30000311604011885
:1010000000000000000000000000000000000000E0
:1010100000000000000000000000000000000022AE
:10102000020000C0001800100010F223E3F3C4CE49
:10103000201214C16F3C5888FFE6EF080000000042
:10104000006804545555554D1CF1EC4CE30DC03D62
:1010500006CC23E2CCD14F333B3713F22B3353541E
:101060000D4FAB28CF1D48E80DCEB33713DBCF1C97
:10107000734C456417FC24E2F05112F1F2F2BA28E5
:101080000479EF2FD173C3C4FD7D138C14D5CA63CB
:1010900000004C444C10D705000013542274334018
:1010A0005513ECC10800C0041122DD0C5430B20706
:1010B000234C101304C12CD07530002333008C3C1A
:1010C000C300CC074CD033303F30E7E1B4003341AC
:1010D000220713141335CDD4650D74EC47C9D01015
:1010E000D0109010D01000003000C0348D0110419D
:1010F00041111462000011620010004444512100AB
:1011000001000001000001001000040010000004B4
:10111000000000000C0000014000104F02003301ED
:10112000114410410440001033000400014000103D
:101130004F00C40031400C4008C001C0CB1033093F
:10114000009300D330B0330D70000CC002C02CCC23
:10115000246000800080910C00022000088064134D
:101160000000800060008000024839054C0330090F
:101170003005300530D9744967746618DA6F050098
:101180000080010044111111511151444404515483
:1011900044441145114500116200004411050054FA
:1011A00055014544455114154011111441101011B9
:1011B00011411111111145140444444404454414CF
:1011C00051115104111151045015110144880100AD
:1011D00014110045444444004055541551454045C0
:1011E0000010454404000050141140141111111155
:1011F0001111111144101111111111114111114549
:10120000541545445551106200505555551441141C
:1012100044050014414405005511005445000015D3
:101220005455555541445515010055055541450046
:10123000405541554145004055554105555551557D
:101240005551555500505555000100555544450020
:101250000055555555550140555555551100555595
:1012600004401501004154550540555555110041A4
:1012700040880140441401005441515044444441C9
:10128000441011010000144444544544144414050E
:1012900010044544404511410010101111155144EE
:1012A00044545555114504540440445050411004D1
:1012B00051545154544545455145101551555554B7
:1012C00044454540415545555515551511545555FD
:1012D00015545504101144455041105555155504E9
:1012E00055114405101454554510550445500445F6
:1012F00050514414411015551555545555455455E4
:10130000555541551145454411155115454555054E
:1013100011620000451401501100501111000050DD
:1013200015400550115441414154555550555510E3
:10133000054055055550550551554155555555557F
:101340005510551545514455555555555421064090
:10135000444400000045101111444144440411412B
:1013600044101111441005511005010014151551B8
:1013700054551515514410110440551115511115AE
:10138000554410005554151111450404014055559C
:10139000151144144100545505404400445154056E
:1013A000005114550014451555004444540044544C
:1013B00000441462004444110100404501501411DE
:1013C0001501004511454400000045444404111135
:1013D000411444411401105144544451444445457E
:1013E00014114551444451105511210000000000D2
:1013F00000000000000000000000000034C003E016
:101400001839F738F77FF3A2007B00BC00CAF3CF8E
:10141000F81FF845F859F866F873F8A0F8BBF8D744
:10142000F90FF924F93BF958F972F981F98CF9A10E
:10143000F9B6F9C8FA5FFC470DDE0E280E3F0EB470
:101440000ECF0F5CF3DFFD39FDA8FDE1FE0AFE3093
:10145000FE53FE61FE6BFE7DFE8FFEA3FEB3FEBF5C
:10146000FECFFF540FB7F3AB0B900C350CA40CC19F
:101470000CE40D21000085160C0F1308793C2C6834
:101480004670F87030C070381CD0F0A04E68A8B01C
:10149000E80E4924B8AE4EEED74E9F30C7704E5C72
:1014A000229CD08628E806706048658C015C621B2F
:1014B000A2A230C770AE738705140E0904793C2CC4
:1014C000A8898C00900F0F0C0913CC37793C92C47B
:1014D000E0793C3BEEA038588C4F0C27693C924C8D
:1014E000E733784C270CB3B846FC064924F81E7E37
:1014F0007E37793C92895270A6A687A647A6B7A6E2
:10150000BF898C5DEE3B0E658C32EE2F58658C21C9
:1015100070658C3A898CC5898C50793C92793C1ADB
:10152000120503151213090F0E898C881E7EF87E92
:1015300023B87E37793C92895244793C3BEEA338FC
:10154000580C270C63AB8C9F884844CC13488843C5
:10155000084404CC13080898F04670B87C588C876F
:1015600088983CA86D8C9F580C1F04138498F04CED
:10157000471348300B0C1F301E06793C65E6534C70
:10158000C36D8C9F580C174B793C92793C1A0E0F07
:1015900020120F0F0D898C884E58793CD36AF3DCEA
:1015A000901E1C793CE5E698E6D63C58BEB31C98E4
:1015B000EA1F3CEB58681598EE1B4C33793C92813E
:1015C0000A5C420A0C23AA62231C29A430C3704E71
:1015D0005CAAF04D9CCC67B8584C474EE8380E0AD0
:1015E000AE28B80A30C370387CAABCF04E705C10CC
:1015F0009050105090105050D058681598EE1B4CD9
:1016000023693CBCC80C17C40E1C1DA4BD8C4D9C8A
:101610000E30C37038BCAA7CF0E0A18888C1B0BD90
:101620001EBA60A67066A638E67066E6F0A3BA60D9
:10163000A67026A638E67026E6F0A3E0DCA0467089
:1016400078E630C0067026CB38EEB33E8F7E5C1253
:10165000DC90905C726B5E725BFC560643A6262B98
:101660004EE0E026E046704EA668793C3BEE43A68D
:101670000670264338EE2BFC5606B3668646707815
:101680003CC6BC68860630C070383C1CCA60164632
:10169000A0A6262746E02B66E6C60A3C0A7CF03662
:1016A0006630C1464670783CA6C6A65ABC1A783C3D
:1016B000066626A666A6793C21A6E066866D8C9F06
:1016C0003E13664670783CC6BC682626C61B46E0BC
:1016D00030C00670383E23A626CB30C01E7EC646DC
:1016E0001F661E46707826467CA63C66683C06A6A9
:1016F0008630BF46BC265E1726463C5ABC1A667921
:101700003C21467078E67C0630C0704EDC9090FC40
:10171000A6B606167CE6F67CF04E68A830C00666D3
:1017200070383E274E7EF04626E0044460793C3B0C
:10173000EEA038588C13488CE30C8B084C3F0448BF
:1017400098F0B833844498F07858FB7858C44C1318
:10175000C88CBF6B0C1F4EE0B858C40C13C80C5794
:101760004670B87C5884983CA84670987C1CEAA0C7
:101770000E6D8CBAB858259E4924B0E888793C2A69
:101780000C27793C954C534924B87C588C1F450252
:10179000C502793C2A793C3BEEA0A6067026433868
:1017A000EE2BFC5606B38630C00670383C56062633
:1017B0000670385CEA273E1366A6066686A65ABC03
:1017C0001A6630C0E6793C2E662643A67026064E81
:1017D000F0C3E04E1C909C101C0AE5A456E6603055
:1017E00005426ABFE01CEDA43C3005426A1F1E1B87
:1017F00059A47CE000000000000000000000000090
:101800004408918C6B30C170385CEA1CBC0A46708D
:10181000793CBA5C6AC44213C81CBD8C4C091FC118
:1018200002793C95F858793CAB6BB058793C9558A7
:10183000793CAB793CA2F0418C78793CA8EE2769E1
:101840003CA10EB05EFE23693CAF1EA0BE1D6160D0
:10185000FE1FEE27693CF3793CA5EE63793C9F1CA3
:1018600002D0761613B6F0793CA86838E8F828B0AC
:10187000A8B80E793CB53A356060793C1D793CF2E8
:10188000EE9B793C6A0E793C1A793CB52626BE253A
:101890006160FE574E5C2226260E793C1A793C99EF
:1018A0000E38AEA0BE1D6160793C1D793C79793C53
:1018B000A2A0256060793C1D793C56D85EFE6B790C
:1018C0003C52A04E3E6EA03D60A5500E60793CFD9E
:1018D000EE9F793C56793CA2A02560A550600E7918
:1018E0003CFDEEFBF8700648693C00793C524E5CCA
:1018F000223AA3793CA5EE37B068693C71793C9FE8
:10190000F627693C6A76F0793CE7793C1DB00E79A0
:101910003CA8A0BE1D6160793C52A04D6060793C3E
:101920001D793CF2793C1D793CEC793C06A0BE1E49
:1019300060793CE3793C81793C990EF8AEA0BE1DFC
:101940006160793C063ECE63793C0EA0BE1E607994
:101950003CDF23793C5A793C87EE67793C5A793CE5
:1019600087EE27F8E82BF84EEED7793CA858793C5B
:101970009558793CAB793CA2F04670B0E8498C2A86
:101980000C27498C95B95AA04E5C66503D6030C812
:1019900070382560A5500E30C770AEE80E384E6026
:1019A000E0B0A84E68793C99E8064870693C00B8F8
:1019B00068380E793C99AEE884B0A8F8280E793CD6
:1019C00099A0BE1D6160793C1D793CA50EB8A0614F
:1019D000604E5C223ABE256160793C060E793CA2DD
:1019E000A01D60A5500E60793CFDEE87793CEC7936
:1019F0003CA2A05CFA37BEB626228B5E37FE373A91
:101A00005BBBFEE762FA1B2213667A00A5500E60EC
:101A1000793C99AEE84EEE27693C2A7870F80E7949
:101A20003C994EEE27B08C53AE0E06664870693C6A
:101A3000000E793CA85EFE23693CAFA0B8AE6160A1
:101A4000096060793C1D793C990EF8A0BE1D61606B
:101A5000793C52A0496060793C1D793CE7793C6A49
:101A60000E793CB5BE1D610E60793C99AE680E7969
:101A70003CD3BE1D6160FE9B793CA55E680E793C3F
:101A8000D31D6060793C1D793CA50E793CB51D6085
:101A900060793C06793C1D793CD386BE2561FE7396
:101AA00060793C52B0A0BE3D61BB793CA50E793C4B
:101AB000D386BE1D61FEBB30C970380EB0BE356125
:101AC000A5500E60793C99AE6888693CB9B026266D
:101AD00026BE77793CB5666666E0A0316060E07945
:101AE0003C5AC3793C56A3793C99F823793C990E2A
:101AF0003833793CA50EB8A0BE1D6160E0793C99F1
:101B0000AE0EE8384EE0793C52A0756060E0793C5A
:101B100056C3793C352B793C52E32E7A0B30C0709A
:101B20003868F828CEBE1EE8B8BA9CEAEAEABAA835
:101B3000AA8A8A8AE330C070EED8B81A9ABABABABA
:101B40001CEAE6A8F8EE38E87828BA463CFED8EE5B
:101B50005CE030C39C4330C41C2330C59C7038EE1D
:101B6000D8B8D4CE14EBFEAED83B793C52A0756009
:101B7000A55060E0AE0E58CE23793C56A049606077
:101B8000E030C070B83CA6BCA830C37038BE5CEA78
:101B9000F0E07038E0793CAB0E30C7BB30D0A330FA
:101BA000C08B30C87330C95B30CA434E707828B8D8
:101BB0006898A85CE04E5C22A0E01C38AAFC0EF8F5
:101BC000FCAAE8AE28E0B0A0FA274626765C5A5E6A
:101BD00050EE4670B87C0E9CA2467C60E6E6A0AE55
:101BE0001C2666E21B4213A6B67FB66F58860646D1
:101BF000B6504626561B26986E466030D070E000E0
:101C00004924F870B80E30D0704EF0F0586D8CAB9F
:101C1000AE5830C07098E8A0BE1D616030D0704EE4
:101C200028E8DA2F58693C3E793C5B30C070F825D3
:101C300060706006481344666630D07038F0EE5825
:101C40004670B028EE7004793C6B30C270658C0829
:101C50006D8CC6AE68F8F0E80666693C506D8CC6BF
:101C600078A01D6068B80EB86160AE0E58CE4960AD
:101C700009604EBE50503D60606D8C1D30D0707854
:101C8000A03D6030C070B82560A830D070F80E302C
:101C9000C07038F01D6060793C55B0FED830DE7001
:101CA00038FED83160606D8C1D30DE7038A6F07E55
:101CB00030C070CE284E900E30D070B8A01D60A8F5
:101CC0000E60693C0A30D0704EE86D8CC6B068304A
:101CD000C070AE6830D0705C4E90A830DE70385E58
:101CE00046F030C0704E28A830D070F80E78A01D95
:101CF000602830C070F80E30D07038AEBE1D61382C
:101D00003D60A550F05C4E22A80EA0B8AEBE1D618D
:101D1000FE2B60693C55B86960AE0E58CE4960E84C
:101D2000B80E1D60B82560F83D60B869604E6690D9
:101D3000503D607030C070F80E60793C62B03D601C
:101D4000700E30C070F81D60F00E60793C62E806DD
:101D50006660693C36B80EA0BE35612830C070B8E8
:101D60000E30D070B86160F030C070780E30D07036
:101D700038616030C07078BE2561B0256060793C04
:101D80005B78256068606D8C5230D070F870B8A0B8
:101D9000696078BE2561B02560606D8C1D30D070A3
:101DA000780EF0A01D60386960606D8C35A03160E0
:101DB00060793C5BF02560606D8C1D30C070787080
:101DC00030D070B8A0FA23DA50260EA8356009602A
:101DD00058606D8C95B0AEA06160B0256068EE462D
:101DE00070B80E78A846703868EE2E7A606D8C0652
:101DF0006D8C52A03160709E30C070CE2830DE7085
:101E000038A606F0B0BE256158380E30C070AEA8B6
:101E100030D07098E8780EB0AEBE1D6128B06888EA
:101E2000084E6830C070B84AFC0E4E1C50A8901C7A
:101E3000029C48021BAE44F08C1F04138430D07007
:101E4000780E4E5C10A035604ED0256068F80E30DC
:101E500007E66030C070B8AE26AE7038A0BE1D6117
:101E6000382560A830C070780EE0DCA01CF2525E0D
:101E70001B669230D070B85EBE1D61FE7384083060
:101E800007E66030C070B80EB09C02EB26AE70AEB4
:101E900038A0BEAE60267038A01D60783D60B8697D
:101EA000604E90BE2561FE1B88083007E66030D08A
:101EB00070F80E30C070B8A626A670AEF0B80E78D6
:101EC000A06160F82560E83007E6C66030C070B8F1
:101ED0000E0C33B0AE9C22A80227693C38B80E4CD9
:101EE0005730D070F826AE70AEF030DE7038A03EBD
:101EF000137E46F060693CE2F858606D8C9530D0F6
:101F00007038586D8CABAEA0BE1D6130D07078704B
:101F1000F858606D8C81980EB0A01D6060793C55BA
:101F200070606D8C521E30C07078A03D60B0FA4376
:101F30005A5E5066D414EB2560A550F05C58606D75
:101F40008CABB0A0A550F060D44B30C07038D888AE
:101F5000D8F0418C786D8C52A049624EA05C6650DE
:101F60003D6230D07038AEA0BE1D636630C10C1724
:101F7000267038FC9CA2023CF0A0B0A550584670D8
:101F800098F068A8E87060E0DDAC0170ED8A5470EC
:101F9000C600F40054564D1110A621AB198EA900AD
:101FA000CF7F773132333435D00BEF0FA815F27F66
:101FB0003D9B737ECF6FA81BA916FF204E2C204996
:101FC0002C2050562C504D542C46F27F568ED01B50
:101FD0006FCF7B111242CF66F14E31AB16A634BFE4
:101FE00036CF7C111243CF67F14932AB16A638BF0A
:101FF00046CF68F2505633AB16A635BF52CF69F3C1
:10200000504D5434AB16A636BF5FCF6AF2465635F4
:10201000AB16A637BF6BCF7EA815F3454E44AB0079
:10202000A800AC00F5424547494EF67F204D4F448D
:10203000457ED07F6FC817F2004E2267B49B111BFC
:10204000124336E02F8864BBA32864B29705F624B8
:102050004552524F528ED0A36F042325402467B5BA
